:10000000EC68040000000000FFFFFF00FFFFFF009E
:10001000FFFFFF00FFFFFF00FFFFFF00FFFFFF00EC
:10002000FFFFFF00FFFFFF00FFFFFF00FC020000DB
:10003000FFFFFF00FFFFFF00BC020000FFFFFF000B
:10004000FFFFFF00FFFFFF00FFFFFF00B001000008
:10005000FFFFFF004A030000FFFFFF00FFFFFF005C
:10006000FFFFFF00FFFFFF00FFFFFF006E02000029
:1000700020020000FFFFFF00FFFFFF00FFFFFF0067
:10008000FFFFFF00FFFFFF0000010000FFFFFF0078
:10009000FFFFFF00FFFFFF00FFFFFF00FFFFFF006C
:1000A000FFFFFF00FFFFFF00FFFFFF00FFFFFF005C
:1000B000FFFFFF00FFFFFF00FFFFFF00FFFFFF004C
:1000C000FFFFFF00FFFFFF00FFFFFF00FFFFFF003C
:1000D000FFFFFF00FFFFFF00FFFFFF00FFFFFF002C
:1000E000FFFFFF00FFFFFF00FFFFFF00FFFFFF001C
:1000F000FFFFFF00FFFFFF00FFFFFF00FFFFFF000C
:10010000FFFFFF00FFFFFF00FFFFFF00FFFFFF00FB
:10011000FFFFFF00FFFFFF00FFFFFF00FFFFFF00EB
:10012000FFFFFF00FFFFFF00FFFFFF00FFFFFF00DB
:10013000FFFFFF00FFFFFF00FFFFFF00FFFFFF00CB
:10014000FFFFFF00FFFFFF00FFFFFF00FFFFFF00BB
:10015000FFFFFF00FFFFFF00FFFFFF00FFFFFF00AB
:10016000FFFFFF00FFFFFF00FFFFFF00FFFFFF009B
:10017000FFFFFF00FFFFFF00FFFFFF00FFFFFF008B
:10018000FFFFFF00FFFFFF00FFFFFF00FFFFFF007B
:10019000FFFFFF00FFFFFF00FFFFFF00FFFFFF006B
:1001A000FFFFFF00FFFFFF00FFFFFF00FFFFFF005B
:1001B000FFFFFF00FFFFFF00FFFFFF00FFFFFF004B
:1001C000FFFFFF00FFFFFF00FFFFFF00FFFFFF003B
:1001D000FFFFFF00FFFFFF00FFFFFF00FFFFFF002B
:1001E000FFFFFF00FFFFFF00FFFFFF00FFFFFF001B
:1001F000FFFFFF00FFFFFF00FFFFFF00FFFFFF000B
:100200000200FA003600F800801F7800200020006D
:100210000C000900B01F7800C01080006200600070
:100220004101DE006000510040003A00C010800033
:10023000610160003B003200E0108000000F780098
:10024000020F200060004700100261000209200038
:10025000020052001A003600E00247001500780044
:100260004500DE00650050004101DD0080F92000FE
:1002700002024000546388000500780010007800F6
:100280006F016000400620000010B800000A7800EE
:100290000500780010007800700160000400320052
:1002A000F0FF2F00606388005C0104000000000084
:1002B00010002000606388008E0104000000000030
:1002C00060024700140078004400DE006F01600007
:1002D000A00020000011B800040078001000780091
:1002E0006F00600000014100506380001008410071
:1002F0005063800010017800C0C620001091B90042
:100300005063800002087800C27C8000E0C62000B4
:1003100060081100D07C8000806388001601040012
:10032000000000009C01040000000000D2FF2F002C
:100330008021200010086100F2EF2F0060082000EB
:1003400010086100A00120000C0009004F10780087
:100350004F0078003600F9000080FA0000400600E7
:100360003600F800801F7800200020000C000900F3
:10037000B01F78007010800062006000C102DE00D3
:100380006080520022003A0070108000E10260009C
:100390001D00320025C7200020CF2000908242009F
:1003A00090108000804A780090678000E102400051
:1003B0009567880002082000110009008282D80099
:1003C0000100780090678800E102400002082000E8
:1003D000110009008282D8000100780046CF200079
:1003E0009602500006003A0010002000B067880016
:1003F00000002000A06788000000200090678800AF
:10040000C4010400000000000E020400000000000F
:10041000D5FF2F00E020200010886200F5DF2F00BC
:100420004008200010886200A00120000C00090094
:100430004F1078004F0078003600F90000400600A9
:100440003600F800801F7800200020000C00090012
:10045000B01F78005E61AE003802040000000000AA
:10046000E00A8000010020002A02040000000000D1
:1004700061E62000C8A2AE004802040000000000AF
:1004800080087800910098006002040000000000DD
:100490000001780011005100C06788008000EB0067
:1004A000D1678800E16780000100E00004003A00A5
:1004B000F16780000100E00001003200C00E8800FA
:1004C0008640A900A00120000C0009004F10780010
:1004D0004F0078003600F900004006003600F800B2
:1004E000801F7800200020000C000900B01F780059
:1004F0005A61AE008602040000000000C00A8000BD
:1005000001002000780204000000000021E6200025
:10051000C882AE0096020400000000008008780047
:1005200091009800AE020400000000000001780075
:1005300011005100006888008000EB0011688800FD
:10054000E16780000100E00004003A00F1678000EC
:100550000100E00001003200B00E88008620A900F2
:10056000A00120000C0009004F1078004F00780017
:100570003600F900004006003600F800801F7800C1
:10058000200020000C000900B01F78004661AE007A
:10059000D402040000000000200A800001002000B6
:1005A000C602040000000000A1E62000D422AE0034
:1005B000E402040000000000800878009100980028
:1005C000EE0204000000000000017800110051005C
:1005D000206888000000EB00306888008480A90053
:1005E000A00120000C0009004F1078004F00780097
:1005F0003600F900004006003600F800801F780041
:10060000200020000C000900B01F78004261AE00FD
:100610001403040000000000000A80000100200014
:100620000603040000000000E1E62000D402AE0052
:100630002403040000000000800878009100980066
:100640003C0304000000000000017800110051008C
:10065000406888008000EB0051688800E1678000F6
:100660000100E00004003A00F16780000100E000B2
:1006700001003200D00E88008420A900A0012000D3
:100680000C0009004F1078004F0078003600F90088
:10069000004006000200FA003600F800801F7800D3
:1006A000200020000C000900B01F7800001480001A
:1006B0006068880010148000706888002014800032
:1006C000806888003014800090688800826880000C
:1006D000CF91DE0040D12000101841001090490059
:1006E00092688000CF91DE0080D120001018410078
:1006F00010904900E068800061024000E4688800D2
:10070000823E20000200520028003500E26880008E
:10071000CF91DE00A0688000B16880000002EB008D
:10072000A220070044C520001401500002079800D1
:10073000F2688800E2688000CF91DE00C068800027
:10074000D16880000002EB00982007000069880053
:1007500000002000CF80DE00C0688800D1688800DB
:100760000000200001002000A0688800B168880017
:1007700000002000E06888000E0190006000510039
:1007800002003D0000002000F0688800F268800050
:10079000CF91DE0020D220001018410010904900B7
:1007A0001200200060D2200010484100F27F2F008C
:1007B0004008200010086100A00120000C00090082
:1007C0004F1078004F0078003600F9000080FA00E2
:1007D0000040060001002800C020200010887000A2
:1007E00001402000E020200010887000000006007A
:1007F0000000FA00711080000010200000806000EE
:10080000C800DE000100E00002003A00FA03040024
:100810000000000068005700104078000080FB00D6
:10082000801088000080FA00000006000000000030
:100830000000000090108000000006007010800092
:1008400061006000000006007110800000102000B0
:1008500000806000C800DE000100E00003003A00F4
:100860000000000024040400000000000000060056
:100870000C00FA00803F20004069880060412000A1
:1008800050698800E04120006069880040422000F3
:1008900070698800A03E200080698800C055200053
:1008A0009069880000002000601088000000280087
:1008B0007010880048000700000F780011079800AA
:1008C000823E2000CF91DE003A32070020079800D8
:1008D00031079800000F780011079800660020008B
:1008E000CFB3DE006A02570034017800A40178001B
:1008F0000603E900030035000201D0008381D20025
:10090000FBFF370042079800530798000002EB00F6
:10091000FA1F07002E029000BE0290004E019000C8
:10092000DE0190002007980031079800040078004D
:10093000850078000002EB001C200700000F780003
:100940001107980012002000CF91DE004E009000A9
:10095000DE00900000027800810278000201E900C8
:10096000030035008502D1000482D300FBFF37006D
:100970002E019000BE019000040051000580590036
:100980000500360012002000CF91DE006000470015
:1009900010184100109049006001470032007800B3
:1009A000A200780061005000E0805800000F78003D
:1009B00011079800A0108800D2FF2F00E02020002F
:1009C0001008610083FF07000D0007000C000700FE
:1009D0000080FA00000006000088230011002000BB
:1009E000000006000100280060212000108870002F
:1009F00001402000802120001088700000000600C7
:100A0000E0462000801F7800A0072000801F7800AB
:100A10005A2F07004F00B100000006000000FA0046
:100A2000C11080000010200000806000C800DE00BF
:100A30000100E00002003A00100504000000000080
:100A400068005700104078000080FB00D01088003C
:100A50000080FA0000000600000000000000000016
:100A6000E010800000000600C010800061006000FF
:100A700000000600C110800000102000008060000F
:100A8000C800DE000100E00003003A0000000000A2
:100A90003A0504000000000000000600F1FF2700F6
:100AA0006021200010886000F1BF2F00802120000D
:100AB0001088600000000600F1FF2700C020200021
:100AC00010886000F1BF2F00E02020001088600037
:100AD000000006000C00FA00E05020004069880089
:100AE000C05220005069880040532000606988008F
:100AF000A053200070698800204F20008069880082
:100B0000E05420009069880000002000B0108800A8
:100B100000002800C0108800AFFF0700000F780019
:100B200011079800823E2000CF91DE00A13107001E
:100B30002007980031079800000F780011079800EF
:100B400066002000CFB3DE006A025700340178004F
:100B5000A40178000603E900030035000201D0007B
:100B60008381D200FBFF37004207980053079800AB
:100B70000002EB00611F07002E029000BE029000F1
:100B80004E019000DE019000200798003107980088
:100B900004007800850078000002EB00831F070046
:100BA000000F78001107980012002000CF91DE009E
:100BB0004E009000DE009000000278008102780074
:100BC0000201E900030035008502D1000482D30050
:100BD000FBFF37002E019000BE0190000400510081
:100BE000058059000500360012002000CF91DE007C
:100BF0006000470010184100109049006001470054
:100C000032007800A200780061005000E0805800B7
:100C1000000F780011079800F0108800D2FF2F0015
:100C200080212000100861006EFF070074FF07009C
:100C300073FF07000080FA00000006004003200058
:100C40004015880040042000001588004041200025
:100C500010158800301020002015880000002000AA
:100C600030158800B01C200050158800B0FF2F0000
:100C70003016880000002000A0168800F0FF2F002A
:100C80009016880000002000C01688000000200098
:100C9000F016880000000600F1F32F00E02020008D
:100CA0001088600001022000800920009080680008
:100CB0000007200080806000800920001088680004
:100CC000F1DF2F0040082000108860000120200084
:100CD000C008200010887000F1F32F008021200050
:100CE0001088600011002000000A200010806800B9
:100CF000E7006000000A2000108868000110200052
:100D0000E0082000108870000000200030088800F3
:100D10000001280080088800E00420007008880096
:100D2000000020005008880000012800900888007A
:100D300001002800002A200010887000F17F2F0099
:100D4000400820001088600001802000C0082000BA
:100D50001088700001082000A01520001088700085
:100D600011002000A015200010806800E70060003E
:100D7000A01520001088680001022000C009200092
:100D8000908068000007200080806000C00920007B
:100D900010886800D1FF2F006008200010886000D4
:100DA00021002000E00820001088700001082000C9
:100DB000E01520001088700011002000E0152000D0
:100DC00010806800E7006000E015200010886800CF
:100DD00001202000C00920009080680000702000E1
:100DE00080806000C009200010886800B1FF2F00DB
:100DF000600820001088600041002000E00820000A
:100E00001088700001082000201420001088700055
:100E1000110020002014200010806800E70060000E
:100E200020142000108868000102200040092000E2
:100E3000908068000007200080806000400920004A
:100E400010886800D1FF2F00400820001088600043
:100E500021002000C0082000108870000108200038
:100E60006014200010887000110020006014200021
:100E700010806800E700600060142000108868009F
:100E8000210020006009200010806800E700600059
:100E90006009200010886800F1FE2F004008200043
:100EA0001088600001012000C00820001088700038
:100EB000000006000000FA00F1FB2F0000222000D5
:100EC000108860000011800062006000C100DE0038
:100ED0000100E00002003200620704000000000090
:100EE0006800570010007800201188000011800071
:100EF000E100600002003A007607040000000000F4
:100F0000201180000080FA00000006000000FA00B6
:100F10000100280000222000108870000080FA00E4
:100F2000000006000000FA00F1FF27000022200068
:100F3000108860000080FA00000006000000FA003F
:100F4000A0752000A069880060782000B069880042
:100F500020792000C0698800680057009000780060
:100F60006A005700908070006C00570090807000FD
:100F70006E005700908070007000570090807000E5
:100F8000720057009080700074005700108170004C
:100F9000F60057002022200011087100F1FB2F00FD
:100FA000002220001088600001002800002220009C
:100FB000108870000080FA00000006000A00FA00A5
:100FC0006000470041442F000900090031587800B3
:100FD000E0222000801F7800D0032000801F7800CE
:100FE000E62D07004F00B10060004700801F780029
:100FF000081D07002F00B100E0462000801F780088
:10100000A0072000801F7800DC2D07004F00B100F2
:101010006800570010007800A01088000080FA00D7
:10102000000006000200FA00F0FF2F00000F780019
:101030009467800043CF2000130052000E0032005E
:1010400023C7200040CF200090814100134078004A
:101050000080FB00000F7800A0678000E1014000E5
:10106000A367880002082000110009008281D800CF
:1010700001007800A06788001E0078000080FA0058
:10108000000006009167800040CF200010805000D3
:1010900002003A000000200001003700100020008C
:1010A000000006000000FA006C0157009240780032
:1010B00010002000124910000104E0001D00320061
:1010C0004EB897009040780060C050000700320092
:1010D0003EB997004EB897009040780012C050007B
:1010E00002003A008A08040000000000CEB8970011
:1010F0003EB89700104178000100780090407800D9
:101100008180FB000281FB0002007800008050001B
:1011100009003700110020006800570010884000C7
:10112000110020006A005700108840005408040095
:1011300000000000000020000080FA00000006000F
:101140000400FA00680057001000780010079800AB
:1011500000002000000F7800620047009000780037
:10116000608050001100360011002000620047002E
:10117000108810001E017800110020006000470058
:10118000108840006A0057001000410010417800AC
:10119000C10220000140510002003200BA080400E0
:1011A00000000000AC080400000000001E007800F1
:1011B0000080FA00000006002A00FA0070004700D4
:1011C000E1442F001300090031587800000020008E
:1011D0003007980000002000010020004007980020
:1011E00051079800D0CC2C00C1DC23006007980088
:1011F00071079800000020002017980000002000D0
:10120000000F780060004700100178007300510063
:101210001C003D0068005700100178006000470086
:101220001000410010427800D2022000024052001B
:101230001400390068005700100178006000470072
:10124000100041001042780092032000024052003A
:101250000C003E0070004700E0024700150240000D
:101260006800570010017800050078001000410068
:10127000104A780010002000950A4000020904007E
:1012800000000000F00247006002470014814200A5
:101290000000200000497800040078001000780069
:1012A00010079800040078001000780020079800CC
:1012B0000500780010427800D2022000024052005F
:1012C00002003A0010002000300798006600470036
:1012D00010007800000F78006000470010027800CE
:1012E000620147001200520018003D0070014700E3
:1012F000600047001000410010427800E202200028
:10130000024052000C003A006001470012007800D1
:10131000200798000200780010027800660147005C
:101320001200520002003A00F0FF2F002007980040
:10133000A609040000000000120020006000470021
:10134000100841006C09040000000000F4FF2F00A9
:1013500064014700120012002A00320064004700B6
:1013600010017800600047006108510060004700EC
:10137000100278006601470012005200210035007B
:101380006E009000FE009000020020000312240076
:10139000622D0700301798004117980060079800E9
:1013A000710798007001470060004700100041007D
:1013B000104178000281FB00000320000000510072
:1013C000CF80DE000081EB00F92C07003E11900079
:1013D000CE119000512D07006802470034017800BB
:1013E000A4017800222E07004007980051079800BA
:1013F000120020006000470010081100B609040028
:10140000000000000000200001F8230060079800A1
:1014100071079800620047001000780061025000D8
:1014200064014700120012003D003200F4FF2F005B
:10143000640147001200120003003A0066004700F2
:101440001000780020079800000020002017980066
:1014500066004700100178006000510002003A0069
:101460001000200020179800640047001001780049
:1014700066004700100241004202200002014700BE
:101480006000470012084200600047001002780028
:10149000620147001200520021003D0002002000BE
:1014A000031224006E009000FE009000A62E07009C
:1014B000301798004117980060079800710798004E
:1014C00070014700600047001000410010417800A3
:1014D0000281FB000003200000005100CF80DE00ED
:1014E0000081EB00B22C07003E119000CE1190005D
:1014F0000A2D07006802470034017800A401780033
:10150000DB2D0700400798005107980012002000CB
:101510006000470010084100440A04000000000079
:1015200066004700100178006100510007003A0092
:101530004E009000DE0090000200200003F82B0017
:10154000F62C070040079800510798004E009000C5
:10155000DE0090000080FA00000006000600FA009D
:10156000CEB89700114078000080FB00000F780093
:1015700002022000E00047001100110006003200C6
:10158000600047009000780069805000020032003F
:10159000D60A040000000000110020006800570077
:1015A00010884000B00A0400000000000000200085
:1015B000100798000000200020079800D2022000A9
:1015C000E00047001100110008003A00110020005F
:1015D0006400470010884000110020006800570098
:1015E00010884000040B040000000000B20220003C
:1015F000E00047001100110003003A001100200034
:101600006800570010884000CEB89700114078005D
:101610000080FB00000F780060004700901F7800FA
:101620001A0007002F00B1000000E0000D0032009A
:101630006202470094007800A00020000089B900F1
:10164000010320006000470010801000000A4100E4
:10165000110020006800570010884000040B0400AF
:10166000000000002E0090000000E00004003200A6
:101670006200470010007800600010000100370091
:101680001E0090000080FA00000006000000FA0032
:1016900092032000E80057001100110008003E00EE
:1016A00002032000E8005700110011000400390077
:1016B0001000200080407800640B0400000000004F
:1016C00000002000804078008180FB00010078004D
:1016D0000080FA00000006000800FA004EB99700EA
:1016E000124078000080FB00000F78000402200008
:1016F000600147001200120006003200600047003F
:10170000100178006900510002003200940B0400BF
:10171000000000001200200068005700100841007F
:101720006E0B04000000000000002000CF80DE00EF
:10173000100798002107980000002000300798004B
:101740004EB8970010427800D202200002405200AA
:1017500008003A001200200066004700100841000F
:10176000120020006800570010084100CA0B040056
:10177000000000004EB8970010427800B20220002E
:101780000240520003003A00120020006800570097
:10179000100841004EB99700124078000080FB000D
:1017A000000F780060004700901F7800B7FF070027
:1017B0002F00B1000000E000120032001E00900077
:1017C000AE009000A200200003002000792E070048
:1017D0000403200060014700120112000202780099
:1017E000CFA2DE00620147000419400005914800C5
:1017F000120020006800570010084100CA0B0400C6
:10180000000000003E0090000000E00006003200F2
:101810006200470030017800A001780060001100EC
:10182000E0801900020037001E009000AE0090001A
:101830000080FA00000006000000FA006A0157006C
:1018400062004100904078002003200001487800A9
:1018500012007800C00088009C05BA00B00080002B
:101860000080FA00000006000A00FA006A00570033
:1018700010007800100798004EB9970032007800E9
:10188000A20078002007980031079800000020008F
:10189000000F780060004700100278006C015700CC
:1018A0001200520015003D006400470040079800F8
:1018B000B01F7800A01F7800DFFF07004F00B100C5
:1018C0001E019000000978002200200062004700FD
:1018D0001008410022002000CF91DE004E00900051
:1018E00010184100109049001200200060004700CD
:1018F000100841004A0C0400000000006C00570072
:10190000100078004100DD004EB99700CF80DE0066
:1019100012194000129148000080FA0000000600F1
:101920004E00FA0060004700C1472F000500090083
:10193000315878006600470021482F000500090053
:10194000315878006C00470081482F0005000900DD
:101950003158780072004700E1482F000400090068
:10196000315878007700470031492F000500090001
:10197000315878007D00470091492F00060009008A
:10198000315878004002200000004700014A2F0033
:10199000020009003158780000002000101F980054
:1019A00068005700901F7800E62407002F00B10060
:1019B0006200500040179800610150006800570015
:1019C0001000410010427800A202200002405200A4
:1019D0000200320000002000D502370086022000FD
:1019E00006034700160078006100500068025700A7
:1019F0001401400000002000004978000400780035
:101A000010017800060078001000410010417800B5
:101A10000281FB00000320000001510052179800D2
:101A2000690051000400340072002000A002200070
:101A30000000470010081100A0022000000047002D
:101A4000100078004400DD00101F98008002200084
:101A50000000470010007800610140006800570056
:101A600010004100104178000281FB0000032000BB
:101A70000001510052179800690051000400340021
:101A800072002000A0022000000047001008110092
:101A9000A002200000004700100178002003200071
:101AA000000047001008410000002000D0698800B5
:101AB00000002000501798000000200040179800F8
:101AC00068005700100178008002200000004700E5
:101AD0001000410010417800604051000E003200BB
:101AE00068005700100078008402200004024700BC
:101AF00014004000104178000281FB00A002200089
:101B0000000047001008690010002000140A40007F
:101B1000600D0400000000002003200000004700CA
:101B200010027800A20220000201470012005200B9
:101B30000400320010002000D0698800000020005E
:101B40007B02370050002000801F7800680057009B
:101B5000901F780060004700801F780051FD07004B
:101B60006F00B10060015000D6003A0068025700D3
:101B7000542798001400780071004000104178004C
:101B800070D220000248780004007800901F78008E
:101B900010002000801F780069FD07004F00B10091
:101BA000401798006601400068005700100141008E
:101BB00000002000004978005E20900010017800AD
:101BC00080022000000047004027980010004100DC
:101BD00064004000801F780077FD07002F00B100EF
:101BE000E0698800F1698800800220000000470059
:101BF00010007800640140006800570010014100A7
:101C000000002000004978005E209000100178005C
:101C10004E2090001000410062004000801F7800BC
:101C20004EFE07002F00B100006A880080022000ED
:101C30000000470010007800620140006800570073
:101C40001001410000002000004978005E20900053
:101C5000100178004E20900010004100801F780095
:101C60003EFE07002F00B100106A88006800570090
:101C7000901F780030002000801F780030FD0700A2
:101C80004F00B10040179800680157001200400053
:101C900062004000801F780047FD07002F00B10060
:101CA000201F9800311F980080022000000047008C
:101CB00010007800620140006800570010014100E8
:101CC00000002000004978005E209000100178009C
:101CD0004E20900010004100801F780036FD070064
:101CE0002F00B10020279800312798000200200023
:101CF000032724002E189000BE189000922C070095
:101D00002E219000BE219000D92B0700206A880068
:101D1000316A880068005700901F7800400020005A
:101D2000801F780006FD07004F00B10068015700D2
:101D3000120040001041780080D420000248780052
:101D40005E209000901F780050002000801F7800D7
:101D5000FBFC07004F00B1004017980068015700D6
:101D60001200400063004000801F780012FD070051
:101D70002F00B100201F9800311F98008002200022
:101D80000000470010007800630140006800570021
:101D90001001410000002000004978005E20900002
:101DA000100178004E20900010004100801F780044
:101DB00001FD07002F00B10020279800312798006F
:101DC00002002000032724002E189000BE18900067
:101DD0005D2C07002E219000BE219000A42B07004F
:101DE000506A8800616A880068005700901F780078
:101DF00060002000801F7800D1FC07004F00B10078
:101E000068015700120040001041780090D4200073
:101E1000024878005E209000901F7800700020003B
:101E2000801F7800C6FC07004F00B1006801570012
:101E300012004000801F7800DFFC07002F00B10077
:101E400062E52000D3FE2300B42A0700706A8800F0
:101E5000816A880068005700901F78008000200089
:101E6000801F7800B6FC07004F00B10068015700E2
:101E700012004000801F7800CFFC07002F00B10047
:101E8000906A8800A16A880068005700901F780057
:101E900090002000801F7800A9FC07004F00B100CF
:101EA0006801570012004000801F78000AFE0700FA
:101EB0002F00B100B06A8800C16A880010002000BD
:101EC0009B01370050002000801F780068005700F9
:101ED000901F780066004700801F780071FC0700A3
:101EE0006F00B1006001500028003A006800570000
:101EF000901F780070002000801F780090FC070081
:101F00004F00B1006801570012004000801F7800A8
:101F100092FD07002F00B100D06A880068005700CA
:101F2000901F780080002000801F780084FC07004C
:101F30004F00B1006801570012004000801F780078
:101F40009DFC07002F00B100E06A8800F16A88005C
:101F500068005700901F780090002000801F7800D4
:101F600077FC07004F00B1006801570012004000E5
:101F7000801F780090FC07002F00B100006B8800E4
:101F8000116B88001000200069013700500020000C
:101F9000801F780068005700901F78006C00470091
:101FA000801F78003FFC07006F00B1006001500007
:101FB000CF003A0010002000206B88006800570016
:101FC000901F780030002000801F78005CFC070024
:101FD0004F00B1006801570012004000801F7800D8
:101FE0005EFD07002F00B1005017980060015000FF
:101FF00004003D000000200050179800101004005D
:1020000000000000A002200000004700100178003E
:102010006C00510002003400C000200050179800EE
:10202000A002200000004700100078004017980030
:10203000A002200000004700100178006C00510051
:1020400016003D00A402200004024700140078009E
:102050004201DD0060D620000201400000002000A7
:102060000009780004007800100078004201DD00CB
:1020700060D6200002004000620140000000200005
:102080000009780012002000A00220000000470094
:1020900010084100181004000000000068005700FC
:1020A000901F780020002000801F780024FC07008B
:1020B0004F00B1006801570012004000801F7800F7
:1020C00026FD07002F00B100610150006217980043
:1020D0006300510084003D00C00220000000470062
:1020E000100078004201DD0080022000000047005F
:1020F00010011100421798006400510002003400E2
:102100004000200040179800000020005017980061
:10211000A002200000004700100278008202200088
:1021200002014700120052006F003D006800570096
:10213000901F7800A00220000000470010007800E7
:102140004200DD0064004000801F7800FCFB0700B7
:102150004F00B100101F98006801570012004000A6
:10216000104178006040510059003200680057006B
:1021700010017800200320000000470010004100FB
:1021800010427800C202200002405200500032008B
:10219000C00220000000470060279800100078006F
:1021A0004201DD00A00220000000470050279800F7
:1021B000100041004201DD0060D620000200400016
:1021C00040279800680057002027980010017800E9
:1021D000200320000000470010004100801F78000D
:1021E000DEFC07002F00B1004E21900000097800AE
:1021F0002E209000901F78005E2090001000780044
:102200004200DD006400400063004000801F780051
:10221000CBFB07004F00B100101F9800C202200046
:1022200002014700120178004212DD00A2022000E4
:1022300002014700120142004212DD0062D6200076
:102240000401410062014100222798006801570003
:1022500012004000801F7800C0FC07002F00B10072
:102260004101DD002E209000020878006E209000D1
:10227000100078004201DD005E2090001000410057
:102280004201DD0060D620000200400062024000F2
:1022900032062000140011000D003600C00220009C
:1022A00000004700100078004201DD00A00220007D
:1022B00000004700100041004201DD0060D6200010
:1022C0000200400062014000300620000009780052
:1022D00012002000A002200000004700100841006A
:1022E000881004000000000010002000900037005B
:1022F00050002000801F780068005700901F780071
:1023000072004700801F780066FB07006F00B10075
:102310006001500006003A0077004700801F7800F7
:102320001D1807002F00B1001000200080003700AA
:1023300050002000801F780068005700901F780030
:102340007D004700801F780056FB07006F00B1003A
:102350006001500073003A0080C52F00F107200093
:10236000002798001127980010002000801F780097
:10237000A002200000004700801F78000004200019
:1023800000004700801F780037FD07006F00B10094
:1023900020002000801F7800E0022000000047009D
:1023A000801F78000004200000004700801F780094
:1023B0002DFD07006F00B100E00220000000470083
:1023C000B01F7800A01F780020462F00801F7800E3
:1023D00060D92000801F7800D41707008F00B1005B
:1023E00060D92000801F7800EB1707002F00B10094
:1023F0005E12900012002000A002200000004700A2
:1024000010081100600052003F003400000420005A
:102410000000470030027800A002780042FF2F0041
:10242000F30720000200520003805A0036003E00ED
:1024300020002000801F780080032000000047005B
:10244000801F78000004200000004700801F7800F3
:1024500005FD07006F00B10020002000801F7800FC
:10246000C003200000004700801F78000004200007
:1024700000004700801F7800FBFC07006F00B100E0
:1024800010002000801F780080022000000047001C
:10249000801F78000004200000004700801F7800A3
:1024A000F1FC07006F00B10080022000000047002F
:1024B000901F7800C003200000004700B01F780084
:1024C000A01F78008003200000004700B01F7800A4
:1024D000A01F7800C0462F00801F780060D9200020
:1024E000801F780091170700EF00B10060D920002D
:1024F000801F7800A81707002F00B1000060FE00C1
:10250000F811040000000000400220000000470015
:10251000801F7800A01707002F00B10010002000D6
:102520000300370020002000D06988000000200050
:102530000080FA00000006000000FA00906E8000A3
:102540000000E0001100320068005700901F780082
:10255000FC2107002F00B100810220000080500004
:10256000C180DE00B062800068004000801F7800FB
:10257000811F7800810C07004F00B10068005700F0
:10258000901F78001F2207002F00B1000080FA0082
:10259000000006001000FA0060004700514B2F00B9
:1025A0000C00090031587800E06A8000F16A800070
:1025B0000200200003002000652907000000E00061
:1025C00002003C0000002000010037001000200045
:1025D0000000E00058003200E26A8000F36A8000E8
:1025E000A06E8000B16E8000592907000000E00055
:1025F00002003D0000002000010037001000200014
:102600000000E0004C003200E06A8000F16A8000C7
:10261000A06E8800B16E8800C26E8000600051001C
:1026200035003C00906E80000000E00001003200A8
:1026300057140700506A8000616A8000D06E8800DD
:10264000E16E8800206A8000316A8000F06E8800A8
:10265000016F8800006B8000116B8000106F880094
:10266000216F880080D420001042780032052000BD
:102670000240520005003A0002002000030028003A
:10268000E0DD2000101869001090690090D420004F
:1026900010427800720520000240520005003A0006
:1026A0000200200003002800A0DD200010186900AF
:1026B00010906900106A8000906F8800006A8000A6
:1026C000A06F8800E0698000F1698000611B07004D
:1026D000B06F880010002000C06F8800000020004C
:1026E000801F7800941707002F00B100F921070020
:1026F0009813040000000000C06E800061005000CC
:10270000C06E8800801F7800304A2F00801F78003C
:1027100060D92000801F7800041707006F00B10007
:1027200060D92000801F780083FF07002F00B100D0
:10273000EA13040000000000C46E8000C2C0200044
:10274000120052001F0032000000200070079800A5
:102750006E00470010017800760051000A003D002D
:1027600062D920006E0047001001410000022000E5
:1027700000497800120020006E0047001008410058
:10278000A81304000000000062D920006E0047007A
:1027900010014100000020000049780060D92000AD
:1027A000801F780064FF07002F00B1006060800088
:1027B000C06E880060004700801F78005EFF070041
:1027C0002F00B1004060800051608000A06E880042
:1027D000B16E88000080FA00000006000800FA00D0
:1027E0006A005700B01F7800A01F7800C5020700DC
:1027F0004F00B10000017800810178000000200046
:1028000001F82300152907000000E0000200350050
:102810000000200001003700100020000000E00050
:102820000300320000002000010020006D0037008E
:102830003EB89700CEB897003EB99700CEB9970042
:102840003628070020079800310798000000200074
:1028500001F82300821F7800831F78002E0190006A
:10286000BE019000BF2807004F01BE00801F780006
:10287000811F78005D0007004F00B100000F780055
:10288000110798006A005700B01F7800A01F780059
:102890009C0207004F00B100000178008101780020
:1028A000F0282C0051F32300A92807000000E000C5
:1028B00002003C0000002000010037001000200052
:1028C0000000E0000A0032001E0178009E01900026
:1028D0003EB89700CEB897009B290700801F78006C
:1028E000811F7800A10207004F00B1003D003700B2
:1028F0006A01570032007800A20078000200200030
:1029000003002000D52807000000E0000200350089
:102910000000200001003700100020000000E0004F
:102920001D0032006000470030017800A0017800EF
:10293000000020000100280000006900818069007B
:102940003EB99700CEB997007F290700801F780015
:10295000811F7800850207004F00B1002007980012
:1029600031079800B0FD200091FC2300821F780001
:10297000831F78002E019000BE0190007928070087
:102980004F01BE0002002000030028000200680082
:1029900083806800130037003EB99700CEB99700D6
:1029A0001E0078009E00900067290700801F7800B5
:1029B000811F78006D0207004F00B10020079800CA
:1029C00031079800B0FD200091FC2300821F7800A1
:1029D000831F78002E019000BE019000612807003F
:1029E0004F01BE000080FA00000006000E00FA0051
:1029F0006A01570032007800A2007800020020002F
:102A000003002000952807000000E00002003400C9
:102A10000000200001003700100020000000E0004E
:102A20000300320000002000010020006F0037008A
:102A30006A01570032007800A2007800000F780089
:102A4000110798000200780030017800A00178009A
:102A50000000200001F823003D2807000000E000EE
:102A600002003C00000020000100370010002000A0
:102A70000000E000070032001E0178009E01900077
:102A80000000200001F823002F290700000F780024
:102A9000110798006A004700801F78006000470017
:102AA000B01F7800A01F7800520007006F00B1002F
:102AB000000F7800110798006A01470012017800A2
:102AC0004191DE00821F7800801F7800811F78000E
:102AD0009C0007006F00B100000F780011079800FC
:102AE0006A00570030017800A00178000000200043
:102AF00001F82300162807000000E00002003C0057
:102B00000000200001003700100020000000E0005D
:102B1000070032001E0178009E0190000000200096
:102B200001F8230008290700000F7800110798001A
:102B300040012000400798001E0178009E0190008F
:102B40003EB89700CEB89700FF2807006002470004
:102B50006407980034017800A40178004428070035
:102B60000200200003002400F72807002007980037
:102B70003107980000027800810278006E00900012
:102B80000001780032007800A2007800040178008B
:102B900085017800312807000000E00002003200C3
:102BA0000000200001003700100020000000E000BD
:102BB00002003200F215040000000000640147002A
:102BC00032007800A2007800000F7800110798000A
:102BD000680047001000780061015000420798002B
:102BE000D5FF3A001E0078009E0090000080FA0099
:102BF000000006000400FA00600247006A01570066
:102C000032007800A2007800001A780001127800E3
:102C1000620042001001780000F827000000610007
:102C2000C701DE00E20720002EB89700028851009D
:102C3000E201420000F023001301680000F82700C1
:102C4000000061009309680034007800A400780057
:102C50000080FA00000006000600FA006A01570032
:102C600032007800A200780002002000030020005B
:102C7000FA2707000000E0000200340000002000F6
:102C800001003700100020000000E00003003200C7
:102C900000002000010020002800370060004700ED
:102CA000801F78006A005700B01F7800A01F7800CE
:102CB000D0FF07006F00B1000200200003002400D5
:102CC000162707000200200003F82300A5270700AD
:102CD00030BF9F0041BF9F001400200060014700EB
:102CE0001209120082002000821F7800224C2F005F
:102CF000821F7800801F7800811F78008B080700F2
:102D00008F00B100100798002107980030BF9F0086
:102D100041BF9F001E007800CF80DE000081EB00E5
:102D2000A32607008221270013F32300FB260700B8
:102D30001E019000AE019000CD2707000080FA0030
:102D4000000006000400FA00E00147006A01570095
:102D500032007800A2007800801978008111780094
:102D6000628041001001780000F827000000610037
:102D70004701DE006C0057001001410022BF9F0098
:102D80006000510003003D00000020000100200011
:102D900023003700F30F20006C0157001280110050
:102DA000130034006A01570032007800A200780056
:102DB0000200200003002000A82707000000E00018
:102DC0000200350000002000010037001000200044
:102DD0000000E00003003200F0FF2F00F1F72F00A9
:102DE0000F003700F0FF2F00F1F727000C0037002D
:102DF00060004700E20140006C00570010007800BE
:102E00004700DD001301680000F8270000006100A2
:102E1000930968006001470032007800A200780042
:102E20000080FA00000006000800FA006A0157005E
:102E300032007800A2007800020020000300200089
:102E4000862707000000E00002003200000020009A
:102E500001003700100020000000E00003003200F5
:102E60000000200001F823007B0037006A005700B3
:102E700030017800A0017800E04F2D00212B2400C4
:102E8000762707000000E000020035000000200067
:102E900001003700100020000000E00003003200B5
:102EA000F0FF2F00F1F727006B0037006A00570092
:102EB00030017800A001780000C52A00E12A2C002A
:102EC000232707000000E00002003C000000200073
:102ED00001003700100020000000E0000300320075
:102EE00000002000010020005B0037006A0157004D
:102EF00032007800A20078000200200003002000C9
:102F0000562707000000E000020035000000200006
:102F10000100370010002000000F78000000E000E2
:102F20000500320002002000030028006A0057005C
:102F300010186900109069003EB89700CEB897004D
:102F4000B2A32A0083FB23007426070030BF9F0032
:102F500041BF9F00801F7800811F7800A3070700F2
:102F60004F00B1003B19070030079800CF80DE000A
:102F70000081EB000E26070010079800210798003B
:102F80006A01570032007800A2007800821F7800A2
:102F9000831F78001E019000AE019000F12607000B
:102FA0004F01BE0030BF9F0041BF9F003E01900017
:102FB000821F780092002000821F7800624E2F004E
:102FC000821F7800801F7800811F7800D7070700D4
:102FD0008F00B100801F7800811F780059FF070023
:102FE0006F00B10030BF9F0041BF9F001E007800FE
:102FF0000000E000160032006A005700300178003F
:10300000A0017800F0FF2F00F1F727001327070039
:103010000000E00002003200000020000100370044
:10302000100020000000E00003003200000020003B
:1030300001002000080037003EB99700CEB9970084
:103040000000200001F82300BF270700020037001E
:103050003EB89700CEB897000080FA000000060046
:103060000000FA00020007009818040000000000A9
:103070000001BE00190007000470A70003F0A100C2
:1030800003F8A30013003A006509B10010003200F4
:10309000090035006928E100020035000100280020
:1030A0000000050000004000818048008502E90022
:1030B000FCFF3A0000000600F88F420005003500D2
:1030C0008100D1000080D3008502E800FCFF3A00B7
:1030D000000006008000EB0000000500C70ADE00CB
:1030E000F107B200F50FB20008003200E1CF420054
:1030F000020032000170A00024000500810F700062
:10310000010032000408050044000500810F700032
:1031100002003A00140005008502E90000004000AA
:1031200081C04800FCFF3B000170A00024000500A6
:103130000080FA00000006000600FA0000002000EF
:10314000000F78006A01570032007800A200780072
:103150000200200003002000C02607000000E0005D
:1031600002003200000020000100370010002000A3
:103170000000E000030032000000200001002000F9
:103180005E0037006E01570032007800A200780020
:103190000200200003002000B02607000000E0002D
:1031A0000200320000002000010037001000200063
:1031B0000000E000030032000000200001F82300BE
:1031C0004E0037006A01570032007800A2007800F4
:1031D0000200200003002000A02607000000E000FD
:1031E0000200350000002000010037001000200020
:1031F0000000E000220032001EB89700AEB8970031
:1032000097FF070010079800210798000001EB00C6
:103210006725070000027800810278006E015700E0
:1032200032007800A200780004017800850178005F
:103230008A2607000000E00002003A00000020009B
:1032400001003700100020000000E0000300320001
:103250000000200001002000280037006200470025
:103260001001780060004700610861000200200042
:10327000030028006A0057001018690010906900C8
:103280006A005700B01F7800A01F780072FE070088
:103290004F00B10030BF9F0041BF9F001EB9970093
:1032A000AEB997009D25070030BF9F0041BF9F002A
:1032B000801F7800811F7800DBFE07004F00B100FF
:1032C00030BF9F0041BF9F001E0078000000E0005B
:1032D000080032006A00570030017800A001780031
:1032E00000002000010028000000690081806900C2
:1032F000020037003EB89700CEB897000080FA0071
:10330000000006000000FA006A0157003200780051
:10331000A200780002002000030020004F260700D2
:103320000000E0000200350000002000010037002E
:10333000100020000000E000080032006A00570082
:1033400030017800A0017800000020000100280072
:103350000000690081806900020037003EB89700D4
:10336000CEB897000080FA00000006000A00FA00BC
:103370006A005700B01F7800A01F7800E1FF070027
:103380004F00B100100798002107980002002000AC
:1033900003002000312607000000E0000200320098
:1033A0000000200001003700100020000000E000B5
:1033B0000300320000002000010020006B003700F5
:1033C0006200470030027800A00278000000200070
:1033D00001F8230004017800850178001F2607000A
:1033E0000000E0000200350000002000010037006E
:1033F00010002000000F78000000E00007003200FD
:103400001E019000AE0190000000200001F8230092
:10341000CD26070010079800210798001E00900095
:10342000AE0090001E019000AE0190003B25070009
:10343000300798004107980054002000841F78004E
:10344000E4502F00841F7800801F7800811F7800CF
:10345000B60607008F00B1001E019000AE0190007B
:103460002E25070010079800210798004000200033
:10347000801F780060522F00801F78006600470090
:10348000B01F7800A01F7800A80607008F00B100C9
:1034900000017800810178001E009000AE009000CD
:1034A000A926070010079800210798001E00780041
:1034B0000000E0000A003200B6FD200097FC230067
:1034C0006202470034017800A40178000600780009
:1034D00087007800A32507001007980021079800AF
:1034E0006A02570034007800A4007800020020002F
:1034F00003002000D92507000000E000020035008D
:103500000000200001003700100020000000E00053
:103510000B0032006200470030027800A002780001
:10352000000020000100280000006A0081806A007D
:103530000003780081037800AA1A0400000000004C
:103540006202470034007800A4007800000378008D
:103550008103780006007800870078001007980043
:10356000210798001E009000AE0090000080FA0035
:10357000000006000000FA006E01570032007800DB
:10358000A200780002002000030020007025070040
:103590000000E00002003C000000200001003700B5
:1035A000100020000000E0000A0032001EB9970061
:1035B000AEB997003EB89700CEB8970062260700D4
:1035C000801F7800811F780068FF07004F00B1005E
:1035D0007D0037006A01570032007800A2007800B1
:1035E0000200200003002000592507000000E00031
:1035F00002003D0000002000010037001000200004
:103600000000E0001A0032006E015700320078001E
:10361000A200780002002000030020008F25070090
:103620000000E0000200350000002000010037002B
:10363000100020000000E0000D0032001EB99700CD
:10364000AEB997003EB89700CEB897003E26070067
:10365000801F7800811F780044FF07004F00B100F1
:10366000B2FD200093042400812507005600370096
:103670006A01570032007800A200780002002000A2
:1036800003002000752507000000E000020035005F
:103690000000200001003700100020000000E000C2
:1036A0002A0032006E01570032007800A200780034
:1036B0000200200003002000682507000000E00051
:1036C000020035000000200001003700100020003B
:1036D0000000E0000D0032001EB99700AEB997005F
:1036E0003EB89700CEB8970017260700801F7800D5
:1036F000811F78001DFF07004F00B100B2FD2000C0
:1037000093042C005A2507002F0037006E01570044
:1037100032007800A20078000200200003002000A0
:103720004E2507000000E0000200320000002000EB
:1037300001003700100020000000E000030032000C
:10374000B0FD200091FC2B001F0037006E015700D8
:1037500032007800A2007800020020000300200060
:103760003E2507000000E0000200320000002000BB
:1037700001003700100020000000E00010003200BF
:103780006A01570032007800A20078000200200091
:1037900003002000EE2407000000E00002003C00CF
:1037A0000000200001003700100020000000E000B1
:1037B00003003200B0FD200091FC2300020037001E
:1037C00000002000010020000080FA000000060038
:1037D0001800FA00506A8000616A8000B2FD200083
:1037E000930424004D2407000200200043332400EA
:1037F000D5250700000F780011079800206A800087
:10380000316A8000B2FD20009304240043240700A5
:103810000200200043332400CB2507004007980016
:103820005107980090D420001043780074052000C0
:103830000440530005003A00040020000500280061
:103840006000470010186A0010906A0080D42000C1
:1038500010437800340520000440530005003A006E
:1038600004002000050028006800470010186A00C6
:1038700010906A00C4002000680057001022B800B1
:10388000A0DD200004024000040F980034007800FE
:10389000A4007800B2FD2000930424001F24070038
:1038A0000200200043332400A725070020079800CA
:1038B000310798000E089000640240003400780040
:1038C000A4007800B2FD2000930424001324070014
:1038D00002002000433324009B2507006007980066
:1038E000710798000400200005002400841F780060
:1038F000851F78006803470036027800A60278002A
:103900000401780085017800962407000200200059
:10391000030024008C250700801F7800811F780099
:10392000A60507004F00B100801F7800811F7800B6
:1039300001FE07008F00B100200F9800310F9800A2
:1039400068004700B01F7800A01F78003806070005
:103950004F00B100000F9800110F98006C00470055
:10396000B01F7800A01F7800310607004F00B1009B
:103970000E0A90009E0A90000401780085017800EC
:10398000E6230700000F9800110F980000002000A8
:1039900001002400801F7800811F78006400470028
:1039A00030037800A00378006002470034017800FB
:1039B000A4017800060078008700780069240700D9
:1039C00002002000030024005F250700801F78000C
:1039D000811F7800790507004F00B100801F780033
:1039E000811F7800D4FD07008F00B1000E0A9000FF
:1039F0009E0A90000401780085017800C723070023
:103A00002E0A9000BE0A900004017800850178001B
:103A100097240700801F7800811F7800F3FB0700C0
:103A20004F00B100801F7800811F78006BFB0700FA
:103A30004F00B1000200200003002400B72307005C
:103A40000200200043332400B4230700B2FD20000D
:103A5000930424003C25070002002600A3762400DE
:103A6000AE23070062E52000D3FE2300AB2307004E
:103A7000D06F8800E16F880004002000050024005A
:103A8000841F7800851F7800801F7800811F7800D0
:103A9000A9FD07008F00B100000F9800110F9800DA
:103AA0000000200001002400801F7800811F7800A2
:103AB000020EF800040EF8009FFD07008F00B10011
:103AC0000E0A90009E0A900004017800850178009B
:103AD00067240700801F7800811F7800C3FB070060
:103AE0004F00B100F06F8800017088006800470047
:103AF000B01F7800A01F7800CD0507004F00B1006F
:103B0000000F9800110F98006C004700B01F78005C
:103B1000A01F7800290507004F00B1000E0A900091
:103B20009E0A900004017800850178007B2307003D
:103B3000200F9800310F980068004700B01F7800F0
:103B4000A01F78001D0507004F00B100000F98006E
:103B5000110F98006C004700B01F7800A01F78007C
:103B6000B30507004F00B1000E0A90009E0A9000B6
:103B7000040178008501780068230700000F980091
:103B8000110F98006400470030037800A00378000C
:103B90006002470034017800A40178000600780034
:103BA00087007800EF230700801F7800811F7800CE
:103BB0009F0507004F00B1000E0A90009E0A90007A
:103BC000040178008501780054230700000F980055
:103BD000110F98002E089000BE089000821F7800F8
:103BE000831F78000E0990009E099000DD230700D6
:103BF0004F01BE00801F7800811F780064004700DD
:103C000030037800A0037800600247003401780098
:103C1000A40178000600780087007800D12307000F
:103C2000801F7800811F7800E40407004F00B10076
:103C3000000F9800110F98006C004700B01F78002B
:103C4000A01F78007A0507004F00B1000E0A90000F
:103C50009E0A900004017800850178002F23070058
:103C6000801F7800811F780042FE07008F00B1009E
:103C7000020020004333240028230700B2FD200067
:103C800093042400B024070030708800417088003D
:103C90000200200003002000F02307000000E000E5
:103CA0000200350000002000010037001000200055
:103CB0000000E00009003200347080004570800090
:103CC00000002000413B24000401780085017800B9
:103CD000E723070030708800417088000080FA00F8
:103CE000000006002A00FA0060004700A1532F00E0
:103CF000040009003158780065004700F1532F0097
:103D00000E0009003158780026032000A4E02000AE
:103D10007400470014084300680057001002780040
:103D20006000520011003A00607080000000E00066
:103D30000C00320000002000607088007400470012
:103D4000901F7800700B2000801F7800F50107009D
:103D50004F00B10060004700801F7800291C070059
:103D60002F00B100F4210400000000006470800006
:103D70006000520010003A001000200060708800BF
:103D80000000200080708800000020007070880013
:103D900074004700901F7800700B2000801F78008F
:103DA000E00107004F00B10065004700801F780068
:103DB000141C07002F00B1003EB897000000E0007F
:103DC000660132007461800085618000127080009D
:103DD00023708000040078008500780061230700CC
:103DE000300F9800410F980000027800810278009F
:103DF0003062800041628000040178008501780013
:103E0000962307000000E0000200350000002000BB
:103E100001003700100020000000E0000600320022
:103E20003062800041628000300F9800410F98009E
:103E3000541F0400000000003462800045628000CE
:103E4000000020000100280000036A0081836A004E
:103E50007600470030027800A00278000600780063
:103E60008700780004017800850178003823070076
:103E70000000E00002003C000000200001003700CC
:103E8000100020000000E0000700320036628000D1
:103E900047628000040020000500280076004700EB
:103EA00004186B0005906B003E089000CE0890004F
:103EB000D2608000E360800098220700700F9800B5
:103EC000011798000002780081027800906080005D
:103ED000A160800004017800850178005F2307005D
:103EE0000000E00002003500000020000100370063
:103EF000100020000000E00006003200906080000A
:103F0000A1608000700F980001179800C21F040084
:103F10000000000094608000A56080000000200088
:103F20000100280000036A0081836A007E004700C8
:103F300030027800A0027800060078008700780040
:103F40000401780085017800012307000000E000EB
:103F500002003C000000200001003700100020009B
:103F60000000E0000700320096608000A76080003B
:103F700004002000050028007E00470004186B00A4
:103F800005906B00746A8000856A80005061800033
:103F9000616180000401780085017800EC2207004F
:103FA0000000E00002003C0000002000010037009B
:103FB000100020000000E0000A0032005261800082
:103FC00063618000706A8000816A8000DE230700E0
:103FD0007E0990008E11900050220700700F98000B
:103FE000011798003470800045708000926A80004C
:103FF000A36A80000400780085007800D9220700B9
:10400000500F9800610F980000027800810278003C
:10401000000020004133240004017800850178006D
:104020000E2307000000E000020035000000200021
:1040300001003700100020000000E0000C003200FA
:104040007A00470030027800A002780002002000C9
:10405000433B24000400780085007800C12207005B
:10406000500F9800610F98006A20040000000000C3
:104070007A00470030027800A0027800000020009B
:1040800041332C000401780085017800B02207003C
:104090000000E00002003C000000200001003700AA
:1040A000100020000000E0000A0032007A00470003
:1040B00030027800A002780000002000413B24007C
:1040C0000401780085017800E9220700500F98006C
:1040D000610F98007A00470030027800A002780053
:1040E0001062800021628000040178008501780060
:1040F000DA2207000000E000020035000000200086
:1041000001003700100020000000E000060032002F
:104110001062800021628000500F9800610F9800AB
:10412000CC200400000000001462800025628000A2
:10413000000020000100280000036A0081836A005B
:104140007A00470030027800A0027800060078006C
:104150008700780004017800850178007C22070040
:104160000000E00002003C000000200001003700D9
:10417000100020000000E0000700320016628000FE
:104180002762800004002000050028007A00470014
:1041900004186B0005906B000200200043332400DC
:1041A0005E089000EE0890006723070032618000EF
:1041B00043618000D921070010179800211798004B
:1041C0000002780081027800F060800001618000C8
:1041D0000401780085017800A02207000000E000BB
:1041E0000200350000002000010037001000200010
:1041F0000000E00006003200F060800001618000F5
:1042000010179800211798004421040000000000B6
:10421000F46080000561800000002000010028009B
:1042200000036A0081836A0020022000000047002A
:1042300030027800A002780006007800870078003D
:104240000401780085017800412207000000E000A9
:1042500002003C0000002000010037001000200098
:104260000000E00008003200F66080000761800076
:104270000400200005002800200220000000470064
:1042800004186B0005906B007E0047003002780038
:10429000A0027800A2708000B37080000400780053
:1042A000850078002F220700B2608000C360800084
:1042B0009A2107006714070090708800C61220003A
:1042C0000602500004003400C012200090708800E4
:1042D00078210400000000009670800044ED2F005B
:1042E0000400530002003D0040ED2F009070880054
:1042F000200220000000470030027800A002780071
:10430000D2708000E370800004007800850078009F
:104310001422070012618000236180007F210700C2
:104320004C140700C0708800C6122000060250001E
:1043300004003400C0122000C0708800AE210400C8
:1043400000000000C670800044ED2F000400530000
:1043500002003D0040ED2F00C07088009470800086
:10436000E0E02000301798001002520032002000D8
:10437000110009000202D8003E1290001400400013
:104380004017980070708800C470800000E1200021
:10439000301798001002520032002000110009006E
:1043A0000202D8003E12900014034000867088007C
:1043B000E4C420004E1090001484B90000C5200011
:1043C00010B3B90004D02000601D200014081400B0
:1043D00084CF2000801D20001408430084D02000DA
:1043E000A01D2000140843000080FA000000060011
:1043F0000E00FA0080C52F00F1072000400798004A
:1044000051079800506A8000616A8000000F7800B0
:1044100011079800206A8000316A80002007980008
:104420003107980080D42000104278003205200027
:104430000240520005003A0002002000030028005C
:1044400064004700101869001090690090D42000A3
:1044500010427800720520000240520005003A0028
:1044600002002000030028006000470010186900C7
:10447000109069001270800023708000106F80001F
:10448000216F8000FA210700F213070060079800EF
:1044900020002000801F780060004700801F780007
:1044A00068005700901F7800A31007006F00B1004C
:1044B00020002000801F780064004700801F7800E3
:1044C00068005700901F78009B1007006F00B10034
:1044D00010002000801F78006C004700801F7800CB
:1044E00068005700901F7800931007006F00B1001C
:1044F0006A00570010007800600798001000200044
:10450000801F78006C004700801F7800680047001B
:10451000801F7800881007006F00B1000080FA004B
:10452000000006000000FA006A005700901F7800A3
:1045300068005700901F7800E0542F00801F78001B
:104540004B1A07006F00B1000080FA00000006005F
:104550000800FA0060004700F1592F00040009002C
:10456000315878003000200030079800E007200024
:10457000801F7800E0012000801F780010020700F3
:104580004F00B1006A005700B01F7800A01F7800EC
:10459000B0552F00801F7800351A07006F00B1005A
:1045A0006A00570030017800A0017800F0618000B7
:1045B00001628000A92107000000E0000200350030
:1045C0000000200001003700100020000000E00083
:1045D0000F003A006A00570030017800A00178000F
:1045E0005061800061618000592107000000E000F7
:1045F00002003C00000020000100370010002000F5
:104600000000E00002003A00102304000000000057
:104610001000200030079800142304000000000060
:10462000300020003007980050072000801F7800DD
:10463000A0012000801F780060562F00801F7800A6
:104640000B1A07006F00B10050072000801F780090
:10465000B0042000801F780000572F00801F7800D2
:10466000031A07006F00B100B0072000801F780018
:1046700080052000801F7800A0572F00801F780041
:10468000FB1907006F00B10010082000801F7800A0
:10469000B0042000801F780040582F00801F780051
:1046A000F31907006F00B10010082000801F780088
:1046B000A0012000801F7800E0582F00801F7800A4
:1046C000EB1907006F00B10060004700801F780001
:1046D000CC1907002F00B10066004700901F78003A
:1046E00080592F00801F7800E11907004F00B100AA
:1046F00000002000801F7800A0052000801F7800A7
:104700006A005700B01F7800A01F7800370007002C
:104710008F00B1000080FA00000006000600FA00D9
:1047200060004700815B2F000500090031587800C8
:104730006A005700901F780068005700901F7800AB
:10474000405A2F00801F7800C91907006F00B10080
:104750006E005700901F78006C005700901F780083
:10476000E05A2F00801F7800C11907006F00B100C8
:1047700060004700801F7800A21907002F00B100D9
:104780000080FA00000006000000FA006A005700EE
:10479000901F780068005700901F7800E05B2F00A2
:1047A000801F7800B21907006F00B1006E0057003B
:1047B000901F78006C005700901F7800805C2F00DD
:1047C000801F7800AA1907006F00B1007000570021
:1047D000901F7800205D2F00801F7800A41907002B
:1047E0004F00B1000080FA00000006002000FA002F
:1047F00010042000000F7800500B200010079800D4
:1048000000002000400F980030002000500F98005A
:104810006E005700100278006000520017003A0046
:10482000EC02570015027800680047006208420059
:1048300005007800100078006500400050079800DF
:10484000200F980090618000A16180000113070093
:1048500070079800F061800001628000FD1207007F
:10486000000F98005061800061618000F91207001C
:10487000100F98006A24040000000000EC025700AA
:1048800015007800400798000500780010027800B5
:104890006A004700630842000500780010007800B5
:1048A000200F98007061800081618000E91207008C
:1048B00070079800D0618000E1618000E512070078
:1048C000000F9800B0618000C1618000E112070014
:1048D000100F980062004700100278006000470047
:1048E000100052004180DE00CF80DE000081EB002E
:1048F000AF1F0700600F9800710F98006A02570001
:1049000034007800A4007800821F7800831F7800AC
:104910006E099000FE099000922007004F01BE0032
:10492000CC120700600798006C0057001000780058
:10493000300798006C00570010007800E602400035
:1049400066024700148012000F003D00620047001D
:10495000901F780066024700941F780060004700AF
:10496000901F780004007800901F78006BFF07000C
:104970008F00B100140020006600470010084200BC
:104980009A24040000000000F0FF2F00300F980070
:10499000F0FF2F00400F98006200470010007800E1
:1049A00020079800640047009002780060024700EA
:1049B000148052006E0034006C0047001002780032
:1049C00042012000110009000202D8000100780015
:1049D000600250000E003A007A004700901F7800F5
:1049E000E4024700951F78006C025700140078001D
:1049F00065004000801F780005007800901F780057
:104A000004007800901F78005FFF0700AF00B1003E
:104A10006C00470010027800A2002000110009007D
:104A20000202D800010078006002500014003A0031
:104A30006C004700100278004201200011000900BC
:104A40000202D80001007800600250000C00320021
:104A50007A004700901F780064024700941F780096
:104A60006A004700901F780004007800901F7800CB
:104A700068004700901F780043FF0700AF00B100B7
:104A80006E004700900278006C02470014805200CC
:104A90000E003A0010002000801F7800E40247005A
:104AA000951F78006C0257001400780065004000E4
:104AB000801F780005007800901F780004007800BF
:104AC000901F780030FF0700AF00B100F5FF2F0006
:104AD00076024700148012000D003A006C00470077
:104AE00090027800700247001480520008003D00D8
:104AF0006C00470090027800720247001480520058
:104B0000030034006400470010007800300F980064
:104B1000F5FF2F0076024700148012000C003200CF
:104B2000F5FF2F00780247001480120008003A00B9
:104B30006C00470090027800700247001480520019
:104B4000030034006400470010007800400F980014
:104B5000140020006C0047001008420014002000E0
:104B60006400470010081200D22404000000000076
:104B7000F5FF2F0076024700148012000700320074
:104B8000F5FF2F00780247001480120003003A005E
:104B90006000470010007800400F9800F5FF2F00DC
:104BA000760247001480120010003200F5FF2F003B
:104BB00078024700148012000C0032003000200000
:104BC000801F780076004700901F7800740247002D
:104BD000941F780078004700901F78000400780048
:104BE000901F7800E8FE0700AF00B1000080FA00D7
:104BF000000006000800FA0060004700D1612F00A5
:104C00000400090031587800300020003007980077
:104C1000E0072000801F7800B0182000801F780077
:104C2000670007004F00B1006A005700B01F78000E
:104C3000A01F7800905D2F00801F78008C1807005F
:104C40006F00B1006A00570030017800A0017800C1
:104C5000D0618000E1618000002007000000E000DA
:104C60000200350000002000010037001000200085
:104C70000000E0000F003A006A00570030017800A1
:104C8000A0017800B0618000C1618000B01F070002
:104C90000000E00002003C0000002000010037009E
:104CA000100020000000E00002003A00622604002C
:104CB0000000000010002000300798006626040065
:104CC000000000003000200030079800500720004E
:104CD000801F7800801B2000801F7800405E2F001E
:104CE000801F7800621807006F00B1005007200095
:104CF000801F780060182000801F7800E05E2F0081
:104D0000801F78005A1807006F00B100B00720001C
:104D1000801F780090172000801F7800805F2F0090
:104D2000801F7800521807006F00B10010082000A3
:104D3000801F780060182000801F780020602F00FE
:104D4000801F78004A1807006F00B100100820008B
:104D5000801F7800801B2000801F7800C0602F001B
:104D6000801F7800421807006F00B1006000470004
:104D7000801F7800231807002F00B100660047004D
:104D8000901F780060612F00801F7800381807009E
:104D90004F00B10010002000801F78002017200075
:104DA000801F78006A005700B01F7800A01F7800AD
:104DB0008EFE07008F00B1000080FA0000000600A0
:104DC0000000FA006A005700901F78006800570042
:104DD000901F780020622F00801F780024180700A1
:104DE0006F00B1000080FA00000006000600FA0023
:104DF0006A03570070012000CF80DE003602780081
:104E0000A60278000000E900030035008502D10009
:104E10000482D300FBFF3700F00F20000002620085
:104E200024079800F0072000000252002407980091
:104E30006000520013003D006A0257003400780001
:104E4000A40078000200200003002000831F070058
:104E50000000E000020035000000200001003700E3
:104E6000100020000000E0000300320000002000DD
:104E700001F82B002B00370000002000010020006B
:104E800028003700640047001002780078005200C4
:104E9000030036003EB89700CEB8970021003700D7
:104EA0003EB89700CEB897006A1107000081EB006A
:104EB0003F1E0700000F78001107980000037800DC
:104EC000810378006A02570034007800A40078005B
:104ED0000601780087017800601F07000000E000ED
:104EE0000200350000002000010037001000200003
:104EF0000000E00009003200600047003002780046
:104F0000A00278000200200003F8230004007800CB
:104F100085007800131F0700020037001E0078008C
:104F20009E0090000080FA00000006000400FA00D5
:104F30006E005700100078004201DD006C00570041
:104F40001001410032007800A2007800000F7800C4
:104F5000110798001EB897000000E000130032000F
:104F60003EB89700CEB897001E0178009E019000D1
:104F70006A1E07006E01570012017800610151009E
:104F800012BF9F004212DD006C0157001202420066
:104F900034017800A4017800351F0700000F780065
:104FA00011079800AA270400000000001E007800E6
:104FB0009E0090000080FA00000006000A00FA003F
:104FC00000002000200798006A0257003400780093
:104FD000A400780002002000030020001F1F07002B
:104FE0000000E00002003500000020000100370052
:104FF000100020000000E000070032000400200044
:10500000050028006A00570010186A0010906A0016
:1050100010002000200798003EB89700CEB89700F7
:1050200032982F0023E223003C1E070030BF9F0070
:1050300041BF9F00801F7800811F78006BFF070031
:105040004F00B10030079800410798006A025700EE
:1050500034007800A4007800821F7800831F780055
:105060003E019000CE019000BE1E07004F01BE0021
:105070000200200003082400281E070030BF9F0004
:1050800041BF9F00000278008102780000002000EC
:10509000010024000401780085017800EF1E07005C
:1050A0000000E00002003500000020000100370091
:1050B000100020000000E000110032006A005700DC
:1050C00030027800A00278000200200003002400D3
:1050D0000400780085007800A21E070030BF9F0002
:1050E00041BF9F002E0090000000E000020032004F
:1050F0000000200001003700100020002007980069
:105100006A00570030027800A002780000002000FA
:1051100001F823000401780085017800CF1E070004
:105120000000E00002003500000020000100370010
:10513000100020000000E0000A00320006002000FD
:10514000070024006A02570034017800A4017800A7
:105150000600780087007800821E070030BF9F009D
:1051600041BF9F003EB89700CEB897003EB9970068
:10517000CEB99700E91D0700000F780011079800CD
:1051800044002000841F780004632F00841F7800EF
:10519000801F7800811F780064FF07008F00B10036
:1051A0003EB99700CEB99700DC1D070030BF9F00C5
:1051B00041BF9F0030002000801F780040642F0016
:1051C000801F780060004700B01F7800A01F7800A3
:1051D00056FF07008F00B1000001780081017800C0
:1051E0003EB89700CEB89700571F070030BF9F000A
:1051F00041BF9F002E0090000000E0000800320038
:105200006A00570030027800A002780000002000F9
:105210000100280000006A0081806A000200370057
:105220003EB89700CEB897000080FA000000060054
:105230000000FA006A00570030027800A0027800EF
:10524000B0FD20009104240004017800850178005D
:10525000821E07000000E000020035000000200070
:1052600001003700100020000000E0000D003200B7
:105270006A00570030027800A002780042BE2C007D
:10528000630924000400780085007800351E0700BB
:10529000801F7800811F780048FF07004F00B10091
:1052A0000C0037006A00570030027800A002780036
:1052B000B0FD200091FC23000401780085017800F6
:1052C0006B1E0700801F7800811F78003BFF0700DE
:1052D0004F00B1000080FA00000006000600FA004E
:1052E0006000470041652F00050009003158780033
:1052F0006E005700901F78006C005700901F7800D8
:105300006A005700901F780068005700901F7800CF
:10531000070007008F00B10060004700801F780081
:10532000B81607002F00B1000080FA000000060048
:105330000000FA00010920006A00570010804000B8
:10534000801F7800010F2000680057001080400087
:10535000801F7800A0652F00801F7800C41607000A
:105360006F00B100010920006E005700108040005E
:10537000801F7800010F20006C0057001080400053
:10538000801F780040662F00801F7800B816070045
:105390006F00B1000080FA00000006000600FA006D
:1053A00060004700E1662F000400090031587800D2
:1053B0006E005700901F78006C005700901F780017
:1053C0006A005700901F780068005700901F78000F
:1053D000D7FF07008F00B10060004700801F7800F2
:1053E000881607002F00B1000080FA0000000600B8
:1053F0000C00FA0080638000CF80DE000081EB00AB
:10540000EB1C0700B2FD200093042400431D07009D
:105410000200200043332400CB1E0700801F7800C9
:10542000811F7800E5FE07004F00B1000200200058
:1054300023352C00391D07002007980031079800FC
:10544000000178008101780000002000C12D2400B7
:10545000021E07000000E0000200350000002000EE
:1054600001003700100020000000E00006003200BC
:1054700000002000C12D240020079800310798006B
:10548000662A040000000000640047003001780034
:10549000A001780000002000C12D2C00AC1D0700E9
:1054A0000000E00002003C00000020000100370086
:1054B000100020000000E000040032000000200086
:1054C000C12D2C00200798003107980070638000E0
:1054D000CF80DE000081EB00B51C07000200200039
:1054E000432B2400E21D0700B2FD2000930424009A
:1054F0000A1D07000200200043332400921E07000B
:10550000801F7800811F7800ACFE07004F00B100BB
:105510002E019000BE019000001D0700CD0F070076
:10552000100798002E009000BE009000020020009E
:1055300003042400F91C07000200200003002400DB
:10554000811E070040079800510798007063800093
:10555000CF80DE000081EB00951C070002002000D8
:10556000432B2400C21D0700B2FD20009304240039
:10557000EA1C07000200200043332400721E0700CB
:10558000801F7800811F780029FF07004F00B100BD
:105590004E019000DE019000E01C0700AD0F0700F7
:1055A000000F7800E4E120001401500007003A00E9
:1055B000620047001002780002E220001200520050
:1055C00002003A00162B040000000000200EF80034
:1055D0001E0EF80000002000801F78000000200050
:1055E000801F78003DFF07008F00B1006002470078
:1055F00014007800F0708800620147001200780003
:105600000071880002007800901F78000400780084
:10561000901F780000002000801F7800000020000C
:10562000801F78005DFF07008F00B100706380006D
:10563000CF80DE000081EB005D1C0700B2FD200082
:1056400093042400B51C070002002000433324000B
:105650003D1E0700801F7800811F780057FE07005D
:105660004F00B10002002000032A2400AB1C0700F9
:10567000780F07001007980070638000CF80DE006D
:105680000081EB004A1C0700B2FD200093042400B7
:10569000A21C070002002000433324002A1E07003A
:1056A000801F7800811F7800E1FE07004F00B100E5
:1056B00002002000032F2400981C0700650F07003C
:1056C000000F780024E220001401500007003A0087
:1056D000620047001002780042E2200012005200EF
:1056E00002003A00BA2B040000000000280EF80067
:1056F000260EF800240EF800220EF800F7FE070030
:105700008F00B100620147001200780004E220001F
:105710001404400028718800E00347001700780057
:10572000E6E1200096024000157188000200780032
:1057300010007800600110000400780010024100A1
:1057400044718800070078001000780060011000A4
:10575000060078001000410030718800841F780036
:10576000801F7800881F7800851F78000BFF0700D6
:105770008F00B1000080FA00000006000000FA006F
:1057800068005700901F78006A005700901F78004B
:1057900030672F00801F7800B51507006F00B1003B
:1057A0000080FA00000006008800FA006000470050
:1057B000918F2F00040009003158780065004700E0
:1057C000E18F2F0004000900315878006A0047007B
:1057D00031902F0004000900315878006F00470015
:1057E00081902F00040009003158780074004700B0
:1057F000D1902F000C0009003158780010022000D1
:1058000000004700A1912F000500090031587800E1
:10581000700220000000470001922F0005000900DF
:1058200031587800D00220000000470061922F001C
:1058300005000900315878003003200000004700BF
:10584000C1922F0005000900315878009003200014
:105850000000470021932F00040009003158780010
:10586000E00320000000470071932F0004000900AE
:10587000315878003004200000004700C1932F0009
:10588000050009003158780090042000000047000E
:1058900021942F000500090031587800F004200001
:1058A0000000470081942F0004000900315878005F
:1058B0004005200000004700D1942F00020009009D
:1058C00031587800700520000000470001952F0036
:1058D0000200090031587800A005200000004700B0
:1058E00031952F000200090031587800D0052000C2
:1058F0000000470061952F00020009003158780030
:10590000000620000000470091952F0002000900CA
:10591000315878003006200000004700C1952F0064
:10592000020009003158780060062000000047009E
:10593000F1952F00020009003158780090062000F0
:105940000000470021962F0002000900315878001E
:10595000C00620000000470051962F0004000900F7
:10596000315878001007200000004700A1962F0052
:105970000300090031587800507080006B0040002F
:10598000801F78001063800061004000801F780055
:10599000E4FA07004F00B100C46F800060005200BD
:1059A0000C003A00E0698000F1698000A90E070050
:1059B000801F7800400DF800420DF80000682F00AD
:1059C000801F78002A1507008F00B100642D0400A5
:1059D00000000000E0698000F16980009D0E070072
:1059E00064DF200014025000343F9800006A8000F9
:1059F000403F9800106A8000503F980060005200BD
:105A000008003D00C403200060072000000047009C
:105A1000100842001400200080072000000047000A
:105A200010081200800720000000470010027800D4
:105A300040DF200010025200443F980060005200F6
:105A400008003D00C403200080072000000047003C
:105A50001008420014002000A007200000004700AA
:105A600010081200A0072000000047001002780074
:105A700020DF200010025200543F980060005200C6
:105A800004003D0084012000A00720000000470022
:105A9000100842006007200000004700901F7800B7
:105AA0008007200000004700901F7800A00720001A
:105AB00000004700901F780060692F00801F780069
:105AC000EB1407008F00B100306380000000E0009D
:105AD0000E003200C46F8000600052000B003200E4
:105AE0004E0DF800500DF80099FA07004F00B10074
:105AF000020EF800040EF8003EFC07004F00B10053
:105B0000F4140700D02E0400000000005070800044
:105B10006B004000801F78007417200020C6200012
:105B200010005200801F78007EFA07004F00B1007D
:105B3000906280000000E000080032004E0DF80086
:105B4000500DF800806A2F00801F7800C8140700ED
:105B50006F00B100C42D040000000000706A8000D6
:105B6000816A8000A2212100F3F123006B1B070052
:105B7000801F7800811F7800606B2F00801F7800E5
:105B8000BB1407006F00B100A4708000B5708000E6
:105B9000D0CC2C00C1E42B000401780085017800F2
:105BA0002E1C07000000E00002003500000020006D
:105BB00001003700100020000000E0001800320053
:105BC000A4708000B5708000D0CC2C00C1E423000C
:105BD0000401780085017800DD1B07000000E0006B
:105BE00002003C00000020000100370010002000EF
:105BF0000000E0000A0032004408200004024700D0
:105C0000000A2000004A78005408200004024700DF
:105C1000000C2000004A7800442E04000000000020
:105C20005408200004024700400C2000004A78007D
:105C3000A0708000B17080000200200003002000EE
:105C4000C31B07000000E00002003C000000200031
:105C500001003700100020000000E00006003200C4
:105C6000440820000402470020082000004A780071
:105C7000442E0400000000004408200004024700F5
:105C800010082000004A7800206080003160800009
:105C9000D26F8000E36F8000201B0700147080002B
:105CA000257080000401780085017800A81B07009A
:105CB0000000E00002003C0000002000010037006E
:105CC000100020000000E000060032001004200058
:105CD000801F7800761407002F00B100742E040096
:105CE000000000007B140700507080007800400026
:105CF000801F78007417200020C62000100052007A
:105D0000801F780007FA07004F00B1009062800002
:105D10000000E00008003200020EF800040EF80057
:105D2000406C2F00801F7800511407006F00B100F5
:105D3000B22E04000000000010708000217080006E
:105D400082942F0013052400F41A0700801F7800A6
:105D5000811F7800006D2F00801F78004414070019
:105D60006F00B1004008200000004700104078009C
:105D70000080FB00801F78005008200000004700D2
:105D8000104078000080FB00801F7800D06D2F004D
:105D9000801F7800361407006F00B1004D14070013
:105DA000406380000000E00014003A00547180005D
:105DB000657180007071800081718000040178003D
:105DC00085017800621B07000000E00002003C0033
:105DD0000000200001003700100020000000E0005B
:105DE0000600320010042000801F780030140700E5
:105DF0002F00B100002F0400000000003514070040
:105E00005070800078004000801F78001063800090
:105E100061004000801F7800C2F907004F00B10008
:105E20002A0EF8002C0EF800606E2F00801F7800FC
:105E30000F1407006F00B100261407005402200061
:105E4000A0E0200010004200801F78001063800056
:105E500061004000801F7800B2F907004F00B100D8
:105E60003605200004D2200014001300380034004E
:105E700000698000CF80DE000081EB004C1A070033
:105E80003232230033B52300A41A0700F4FD2400A6
:105E9000D5EC23000401780085017800311B070050
:105EA000D2CC2C00C3BC2300271C07000400200018
:105EB00005F0230004017800850178006C1B0700C1
:105EC0000087980011879800906280000000E00031
:105ED0000A0032000008200000004700B01F7800D0
:105EE000A01F7800206F2F00801F7800E0130700AC
:105EF0006F00B100A42F0400000000000E8090008D
:105F00009E8090000200200003112400831A0700E5
:105F100002002000030A24000B1C070004002000DC
:105F2000052024000401780085017800501B07003B
:105F3000801F7800811F780010702F00801F78006C
:105F4000CB1307006F00B100B02F04000000000069
:105F500000712F00801F7800C51307002F00B100CB
:105F6000DC1307000403200060C5200010A2B90064
:105F7000000D200004034000A4E02000C007200022
:105F8000000047001408530014638000E00720005D
:105F9000000047006108420094718000A5718000F4
:105FA00000002000010A2400040178008501780027
:105FB0002A1B07000000E00002003500000020005E
:105FC00001003700100020000000E0005B003200FC
:105FD000C007200000004700901F7800E007200065
:105FE00000004700901F78004EF907004F00B100F5
:105FF00094718000A5718000B0718000C171800033
:106000000401780085017800D11A07000000E00043
:1060100002003C00000020000100370010002000BA
:106020000000E0000600320010042000801F78000D
:106030009F1307002F00B100223004000000000071
:10604000A4130700320EF800340EF80090712F00F0
:10605000801F7800861307006F00B100C007200082
:1060600000004700100078006D004000801F78009D
:10607000E007200000004700901F780029F9070082
:106080004F00B1003A0EF8003C0EF80020732F00CC
:10609000801F7800761307006F00B100C007200052
:1060A00000004700100078007A004000801F780050
:1060B000E007200000004700901F780019F9070052
:1060C0004F00B100F47180000572800050628000C2
:1060D000616280000401780085017800DF1A070002
:1060E0000000E00002003500000020000100370041
:1060F000100020000000E000060032001004200024
:10610000801F78006A1307002F00B1008C30040054
:10611000000000006F1307003E0EF800400EF8006C
:10612000E0732F00801F7800511307006F00B1004B
:1061300068130700EE30040000000000C0072000D4
:1061400000004700901F7800E00720000000470093
:10615000901F7800F3F807004F00B100600047007F
:10616000801F7800271307002F00B100C007200010
:1061700000004700100078006D004000801F78008C
:10618000E007200000004700901F7800E5F80700B6
:106190004F00B10065004700801F78001913070009
:1061A0002F00B100C0072000000047001000780059
:1061B0007A004000801F7800E007200000004700C0
:1061C000901F7800D7F807004F00B1006A00470021
:1061D000801F78000B1307002F00B100C46F8000F0
:1061E00060005200C00132000403200060C520009E
:1061F00010A2B900D00D200004024000A0E0200051
:1062000010005200603F9800801F78003418200072
:1062100020C6200010005200801F7800C1F807003F
:106220004F00B100D46F8000E56F80007060800087
:10623000816080000401780085017800441A07001D
:106240000000E00002003C000000200001003700D8
:10625000100020000000E0003E003200906280004C
:106260000000E00008003200FA0DF800FC0DF80014
:10627000B0742F00801F7800FD1207006F00B1007E
:10628000A631040000000000D06F8000E16F8000A4
:10629000A2212100F3F12300A0190700020024002D
:1062A000C3612400281B07000002780081027800E7
:1062B0000000200001F82300040178008501780027
:1062C000661A07000000E000020035000000200010
:1062D00001003700100020000000E0001000320034
:1062E000D06F8000E16F8000A2212100F3F1230034
:1062F0008A19070002002000A3472400121B070090
:10630000801F7800811F780060752F00801F780043
:10631000D71207006F00B100A63104000000000092
:10632000D06F8000E16F800082942F00130524005D
:106330007A190700801F7800811F780030762F00BF
:10634000801F7800CA1207006F00B100B23104004C
:10635000000000006F004700801F7800A9120700AE
:106360002F00B100C0072000000047001000780097
:106370006D004000801F7800B416200020C6200069
:1063800010005200801F780066F807004F00B1002F
:1063900074004700801F78009A1207002F00B10098
:1063A000F46F800005708000006080001160800044
:1063B0000401780085017800281A07000000E00039
:1063C000020035000000200001003700100020000E
:1063D0000000E0000600320010042000801F78005A
:1063E000B31207002F00B100FA31040000000000D2
:1063F000B8120700906280000000E0000800320040
:10640000FE0DF800000EF800F0762F00801F7800D7
:10641000971207006F00B100723204000000000004
:10642000F06F800001708000A2212100F3F12300B1
:106430003A19070002002400C3612400C21A0700B1
:1064400000027800810278000000200001F823009B
:106450000401780085017800001A07000000E000C0
:10646000020035000000200001003700100020006D
:106470000000E00010003200F06F8000017080002A
:10648000A2212100F3F123002419070002002000BB
:10649000A3472400AC1A0700801F7800811F7800F2
:1064A000A0772F00801F7800711207006F00B100E5
:1064B0007232040000000000F06F80000170800064
:1064C00082942F001305240014190700801F780000
:1064D000811F780070782F00801F780064120700F9
:1064E0006F00B1007B1207000403200060C520008C
:1064F00010A2B900F008200004034000A4E020002E
:10650000C00720000000470014085300E60B2000DD
:1065100024C62000E00720000000470014085300B4
:10652000746A8000856A80000000200001F023006A
:106530000401780085017800851907000000E0005B
:1065400002003C0000002000010037001000200085
:106550000000E000A3003200C00720000000470058
:10656000901F780084022000E00720000000470010
:1065700010004200801F780011FA07004F00B100A0
:10658000906280000000E00032003200C00720006E
:10659000000047001000780070004000801F780065
:1065A000E007200000004700901F7800DDF707009B
:1065B0004F00B100420EF800440EF80030792F0071
:1065C000801F78002A1207006F00B100C00720006A
:1065D00000004700100078007D004000801F780018
:1065E000E007200000004700901F7800CDF707006B
:1065F0004F00B100460EF800480EF800F07A2F0068
:10660000801F78001A1207006F00B100A40220005A
:10661000C00720000000470010004200801F7800E3
:10662000E007200000004700901F7800BDF707003A
:106630004F00B1004A0EF8004C0EF800907C2F007D
:10664000801F78000A1207006F00B100AE3304000B
:1066500000000000C0072000000047001000780084
:1066600070004000801F7800E00720000000470015
:10667000901F7800ABF707004F00B1001072800048
:1066800021728000A2212100F3F12300A31807004A
:10669000801F7800811F7800207E2F00801F7800E7
:1066A000F31107006F00B100C00720000000470091
:1066B000100078007D004000801F7800E007200077
:1066C00000004700901F780096F707004F00B100C8
:1066D000307280004172800082942F0013052400E4
:1066E0008E180700801F7800811F7800E07F2F0040
:1066F000801F7800DE1107006F00B100A4022000A7
:10670000C00720000000470010004200801F7800F2
:10671000E007200000004700901F780081F7070085
:106720004F00B1005072800061728000A2212100F0
:10673000F3F123007918070002002000A34724008A
:10674000011A0700801F7800811F780090812F00B8
:10675000801F7800C61107006F00B100947180009F
:10676000A57180000000200001F8230004017800DA
:1067700085017800391907000000E00002003500AB
:106780000000200001003700100020000000E000A1
:106790001000320074032000C007200000004700F2
:1067A00010004200801F7800E00720000000470032
:1067B000901F78005BF707004F00B1004E0EF80005
:1067C000500EF80040832F00801F7800A8110700AA
:1067D0006F00B10010002000907288007434040033
:1067E0000000000094728000610052003E003A00F8
:1067F000C007200000004700100078007000400033
:10680000801F7800E007200000004700901F7800FC
:1068100044F707004F00B1001002200000004700BD
:10682000801F7800771107002F00B100C0072000FB
:1068300000004700100078007D004000801F7800B5
:10684000E007200000004700901F780035F70700A0
:106850004F00B1007002200000004700801F780048
:10686000681107002F00B100A4022000C00720001B
:106870000000470010004200801F7800E007200061
:1068800000004700901F780026F707004F00B10076
:10689000D002200000004700801F78005911070037
:1068A0002F00B10074032000C00720000000470043
:1068B00010004200801F7800E00720000000470021
:1068C000901F780017F707004F00B1003003200039
:1068D00000004700801F78004A1107002F00B10018
:1068E0000000200090728800C46F80006000520099
:1068F000160032002060800031608000D26F80007E
:10690000E36F800005180700147080002570800078
:1069100004017800850178008D1807000000E00070
:1069200002003C00000020000100370010002000A1
:106930000000E00005003A00F467800060005200AB
:10694000020032006435040000000000E4678000AB
:10695000600052005C003A00507080006B00400004
:10696000801F780080072000801F7800EDF6070068
:106970004F00B100D46A80006300520007003D0060
:106980005A0DF800E0842F00801F780038110700AE
:106990004F00B100D8340400000000005A0DF80088
:1069A00050862F00801F7800311107004F00B10082
:1069B000507080006B004000801F7800600E200047
:1069C000801F7800D7F607004F00B10080D4200068
:1069D000104078000080FB00801F7800440DF80014
:1069E000460DF80020872F00801F78002011070037
:1069F0008F00B1005070800078004000801F780048
:106A0000600E2000801F7800C6F607004F00B1001E
:106A100090D42000104078000080FB00801F780098
:106A20004A0DF8004C0DF80000882F00801F7800F8
:106A30000F1107008F00B1005070800078004000F7
:106A4000801F7800E0062000801F7800B5F6070060
:106A50004F00B100E06A8000F16A8000020020006F
:106A6000030020003A1807000000E00002003C008C
:106A70000000200001003700100020000000E000AE
:106A8000080032005C0DF8005E0DF800E0882F0071
:106A9000801F7800F61007006F00B1005C3504001D
:106AA000000000009003200000004700801F7800D5
:106AB000D41007002F00B10010002000A072880041
:106AC000CE35040000000000A47280006100520076
:106AD00032003A00507080006B004000801F780048
:106AE00080072000801F78008EF607004F00B1005D
:106AF000E003200000004700801F7800C11007005D
:106B00002F00B100507080006B004000801F7800A3
:106B1000600E2000801F780082F607004F00B10051
:106B20003004200000004700801F7800B5100700E7
:106B30002F00B1005070800078004000801F780066
:106B4000600E2000801F780076F607004F00B1002D
:106B50009004200000004700801F7800A910070063
:106B60002F00B1005070800078004000801F780036
:106B7000E0062000801F78006AF607004F00B10091
:106B8000F004200000004700801F78009D100700DF
:106B90002F00B10000002000A0728800000020003B
:106BA000303F98000403200060C5200010A2B90007
:106BB000900D200004034000A4E02000C007200046
:106BC0000000470014085300C0082000703F9800E0
:106BD000906A8000A16A80001E0A0700503F98005A
:106BE000C406200004025000543F98006000520088
:106BF00004003D0084162000A0072000000047008C
:106C000010084200A0072000000047001002780092
:106C100062002000110009000202D800503F9800D5
:106C2000640020000480B900503F980076022000E4
:106C300064072000040247001400130090003D0088
:106C4000A007200000004700100078006603400005
:106C5000563F9800841620000400530004003500BD
:106C600084162000A0072000000047001008120032
:106C7000A00720000000470010027800E201200079
:106C8000110009000202D8000100780060025000E3
:106C90000A00320060D92000660720000603470082
:106CA00016024000D0022000004A780010002000A8
:106CB000160B40003C37040000000000A405200033
:106CC000A007200000004700100078001100090014
:106CD0000400D80001007800600250001200320069
:106CE000A007200000004700901F7800308A2F0086
:106CF000801F780064D92000600720000000470052
:106D000010004200801F7800880507006F00B10066
:106D100034002000600720000000470010084200F7
:106D2000343704000000000060D92000660720000E
:106D30000603470016024000D0022000004A7800F7
:106D400010002000160B4000E43604000000000094
:106D50004408200004024700E0042000004A7800B4
:106D6000123704000000000044082000040247001D
:106D700050042000004A7800123704000000000090
:106D8000440820000402470030052000004A780033
:106D900012370400000000004408200004024700ED
:106DA00070052000004A780012370400000000003F
:106DB0004408200004024700F0032000004A780045
:106DC0001237040000000000A00720000000470068
:106DD0001002780060005200DDFF3200A60520009E
:106DE000A40720000402470014001300DEFF320055
:106DF000460B2000A40720000402470014001300E3
:106E0000DFFF3200A00720000000470010037800D9
:106E1000E410200004005300DFFF3200D8360400E5
:106E20000000000060D9200066072000060347002C
:106E3000160240004008200000004700104A780079
:106E4000060078001000780061024000343F98008E
:106E500060D9200004024000D0022000004A7800DF
:106E600010002000160B4000C4002000A0072000E6
:106E70000000470010084200163604000000000021
:106E800064D9200060072000000047001002420083
:106E900000002000004A7800906A8000A16A80000B
:106EA0006C090700303F98006400200011000900C1
:106EB0000400D80001007800303F980060025000C4
:106EC00005003A0084DB200000002000004A780022
:106ED000723704000000000094DB20000000200056
:106EE000004A7800E0072000000047001002780008
:106EF000600720000000470010035200363F980052
:106F000094DB200000002000004A7800C007200029
:106F100000004700100078006A004000801F7800E1
:106F2000861F7800A6F707004F00B10090D9200017
:106F3000801F7800808A2F00801F7800CC0F070008
:106F40004F00B1003470800045708000926A80006C
:106F5000A36A80000400780085007800011707000C
:106F60003C090700503F9800C00720000000470080
:106F7000901F7800A4052000E007200000004700D3
:106F800010004200801F78008DF707004F00B1000D
:106F9000A0072000000047001002780060005200A7
:106FA0000B003A00C06F80000000E00008003200D3
:106FB000520DF800540DF800D08A2F00801F780081
:106FC000AB0F07006F00B100F437040000000000B1
:106FD000520DF800540DF800908B2F00801F7800A0
:106FE000A30F07006F00B100BA0F0700C06F800049
:106FF0000000E00024013200206380000000E00077
:1070000001003200FAF80700A00720000000470046
:1070100010037800C4F42F000400530006003D0064
:1070200084162000A007200000004700100842003E
:107030002E38040000000000460B2000A4072000AA
:1070400004024700140013000400340084162000DA
:10705000A0072000000047001008120000002000D8
:10706000403F980080072000000047001002780091
:107070007F0052000C003D0064D9200080072000F2
:10708000000047001002420000022000004A780081
:107090001400200080072000000047001008420074
:1070A000323804000000000064D92000800720006E
:1070B000000047001002420000002000004A780053
:1070C00006FA2F00A4072000040247001400130052
:1070D0002400340006062000A40720000402470014
:1070E000140013001F003D00A4052000A00720008D
:1070F000000047001002420034879800443F980087
:1071000062002000110009000202D800010078008E
:10711000303F9800640020003E809000110009007C
:107120000400D800403F9800600250000B0035007A
:107130008007200000004700100278007F00520006
:1071400006003D0064D920008007200000004700B1
:107150001002420080042000004A7800B638040083
:107160000000000000002000303F98006007200071
:107170000000470010027800E007200000004700F0
:1071800010024200343F9800C00720000000470072
:107190001000780074004000801F7800841F780081
:1071A00007F707004F00B100A007200000004700CC
:1071B000100278006000520008003A0060D92000F8
:1071C000801F7800008C2F00801F7800280F070098
:1071D0004F00B1002239040000000000A007200089
:1071E00000004700100278006700520007003500D9
:1071F00096FF2F00A407200004024700140013008C
:1072000002003C00163904000000000060D9200094
:10721000801F7800F08C2F00801F7800140F07006B
:107220004F00B100223904000000000060D92000A6
:10723000801F7800408D2F00801F78000C0F070002
:107240004F00B100A00720000000470010027800A6
:107250006000520024003A00C007200000004700F0
:10726000100078006A004000801F7800E0072000CE
:10727000000047001000780067005000801F780071
:10728000A8F407004F00B1004005200000004700AF
:10729000801F7800DB0E07002F00B100C007200020
:1072A00000004700100078006A004000801F78004E
:1072B000F40B2000E007200000004700100042000F
:1072C000801F780097F407004F00B1007005200080
:1072D00000004700801F7800CA0E07002F00B10091
:1072E000403A040000000000A00720000000470012
:1072F00010027800600052002E003D00C007200000
:1073000000004700100078006A004000801F7800ED
:10731000E0072000000047001000780067005000E0
:10732000801F78007FF407004F00B10066FA2F003D
:10733000A4072000040247001400130007003D00CA
:10734000A005200000004700801F7800AD0E070058
:107350002F00B100B839040000000000D005200063
:1073600000004700801F7800A60E07002F00B10024
:10737000C007200000004700100078006A004000AD
:10738000801F7800F40B2000E00720000000470079
:1073900010004200801F780062F407004F00B10027
:1073A0000006200000004700801F7800950E0700AF
:1073B0002F00B100A0072000000047001002780055
:1073C000600052002E003400C0072000000047007B
:1073D000100078006A004000801F7800F40B200045
:1073E000E00720000000470010004200801F7800E6
:1073F0004CF407004F00B100A6052000A4072000B0
:107400000402470014001300070034003006200077
:1074100000004700801F78007A0E07002F00B1009F
:107420001E3A040000000000600620000000470033
:10743000801F7800730E07002F00B100C0072000E6
:1074400000004700100078006A004000801F7800AC
:10745000E00720000000470010007800670050009F
:10746000801F78002FF407004F00B1009006200025
:1074700000004700801F7800620E07002F00B10057
:10748000C43B040000000000206B80000000E0000E
:10749000BD003200B06280006B024000643F980083
:1074A00000002000206B8800841F7800B0002000BE
:1074B000801F7800B1F807004F00B10000002000E5
:1074C000303F98006007200000004700100278005D
:1074D0006C00520038003D006007200000004700AB
:1074E000100078004202DD0060D620000400400059
:1074F0006203400024032000160012000600310041
:10750000540820000402470000092000004A7800C7
:10751000BE3A0400000000006007200000004700A1
:10752000100078004202DD0060D620000400400018
:1075300062024000100320001402100072002000BC
:10754000110009000282D800040920000002420054
:1075500050082000000047000448780004437800E9
:107560006409200004405300040036005408200041
:107570000402470060092000004A780050082000FB
:1075800000004700104078000080FB00801F78005A
:10759000908D2F00801F7800350E07004F00B1003E
:1075A000140020006007200000004700100842007F
:1075B000623A040000000000C007200000004700FD
:1075C0001000780061004000801F7800B0002000AB
:1075D000801F780069F807004F00B100000020000C
:1075E000303F98006007200000004700100278003C
:1075F0006C0052002E003D00600720000000470094
:10760000100078004202DD0060D620000400400037
:107610006203400014032000160012000600390027
:10762000540820000402470060092000004A780046
:107630003A3B040000000000600720000000470003
:10764000100078004202DD0060D6200004004000F7
:107650006200400010027800720020001100090052
:107660000282D800060920005408200004024700C6
:10767000004A4300500820000000470010407800F6
:107680000080FB00801F7800608E2F00801F780034
:10769000F70D07004F00B100140020006007200024
:1076A0000000470010084200F23A04000000000009
:1076B000C007200000004700100078006200400072
:1076C000801F7800B0002000801F78002BF8070092
:1076D0004F00B100C006200000004700801F780066
:1076E000C80D07002F00B10000002000303F9800B7
:1076F0006007200000004700100278006C00520074
:1077000021003D00600720000000470010007800C5
:107710004202DD0060D62000040040001002780024
:10772000600052000D00320060072000000047009A
:10773000100078004202DD0060D620000400400006
:10774000901F7800308F2F00801F7800C80D070031
:107750004F00B100B83B04000000000010072000FB
:1077600000004700801F7800A60D07002F00B10021
:1077700014002000600720000000470010084200AD
:10778000783B0400000000000080FA0000000600C2
:107790000600FA0060004700E1962F00040009008F
:1077A0003158780060004700801F7800950D070071
:1077B0002F00B1000080FA00000006000600FA0069
:1077C00080012000000F7800B262800030002000AD
:1077D0000090B900F00140002307980068015700AD
:1077E0001200780010079800128011000700340082
:1077F000C00D2000000F78006400470010007800E2
:10780000610140006200470010081100620047005B
:1078100010017800D00020000090B90010079800F7
:107820007A00400010079800801F78006000470031
:10783000901F780030972F00801F78008C0D070074
:107840006F00B1000080FA00000006005200FA004C
:1078500060004700B1C82F000300090031587800CC
:1078600064004700F1C82F00030009003158780078
:107870006800470031C92F00030009003158780023
:107880006C00470071C92F000300090031587800CF
:1078900070004700B1C92F00060009003158780078
:1078A0007700470021CA2F000800090031587800EE
:1078B0000002200000004700B1CA2F0003000900A9
:1078C000315878004002200000004700F1CA2F0024
:1078D00004000900315878009002200000004700A1
:1078E00041CB2F000300090031587800D00220005E
:1078F0000000470081CB2F000500090031587800B7
:107900003003200000004700E1CB2F0003000900F6
:1079100031587800700320000000470021CC2F0070
:107920000300090031587800B00320000000470030
:1079300061CC2F000200090031587800E0032000DC
:107940000000470091CC2F00040009003158780056
:107950003004200000004700E1CC2F0002000900A5
:1079600031587800600420000000470011CD2F003E
:107970000400090031587800B004200000004700DE
:1079800061CD2F000100090031587800D00420009B
:107990000000470081CD2F00040009003158780015
:1079A00068005700901F780084FF07002F00B10087
:1079B000680057001001780061E5200011005100B7
:1079C00006003A00A0042000801F7800380D070050
:1079D0002F00B100F03C0400000000003D0D070046
:1079E0005240040000000000000CF800020CF800F7
:1079F00000982F00801F780060D92000801F780039
:107A00004A0207008F00B100664104000000000038
:107A1000040CF800060CF80080992F00801F7800F5
:107A200060D92000801F7800400207008F00B1005D
:107A30006641040000000000080CF8000A0CF80081
:107A4000009B2F00801F780060D92000801F7800E5
:107A5000360207008F00B1006641040000000000FC
:107A60000C0CF800809C2F00801F780060D920004B
:107A7000801F78002D0207006F00B10066410400EE
:107A8000000000000E0CF800100CF800E09D2F0024
:107A9000801F780060D92000801F78002302070033
:107AA0008F00B1006641040000000000120CF800D5
:107AB000140CF800609F2F00801F780060D9200010
:107AC000801F7800190207008F00B1006641040092
:107AD00000000000160CF800180CF800E0A02F00C1
:107AE000801F780060D92000801F78000F020700F7
:107AF0008F00B10066410400000000001A0CF8007D
:107B00001C0CF80060A22F00801F780060D92000B4
:107B1000801F7800050207008F00B1006641040055
:107B2000000000001E0CF800200CF800E0A32F005D
:107B3000801F780060D92000801F7800FB010700BB
:107B40008F00B1006641040000000000220CF80024
:107B5000240CF80060A52F00801F780060D9200059
:107B6000801F7800F10107008F00B100664104001A
:107B700000000000260CF800280CF800E0A62F00FA
:107B8000801F780060D92000801F7800E70107007F
:107B90008F00B10066410400000000002A0CF800CC
:107BA0002C0CF80060A82F00801F780060D92000FE
:107BB000801F7800DD0107008F00B10066410400DE
:107BC000000000002E0CF800300CF800E0A92F0097
:107BD000801F780060D92000801F7800D301070043
:107BE0008F00B1006641040000000000320CF80074
:107BF000340CF80060AB2F00801F780060D92000A3
:107C0000801F7800C90107008F00B10066410400A1
:107C100000000000360CF800380CF800E0AC2F0033
:107C2000801F780060D92000801F7800BF01070006
:107C30008F00B10066410400000000003A0CF8001B
:107C40003C0CF80060AE2F00801F780060D9200047
:107C5000801F7800B50107008F00B1006641040065
:107C6000000000003E0CF800400CF800E0AF2F00D0
:107C7000801F780060D92000801F7800AB010700CA
:107C80008F00B1006641040000000000460CF800BF
:107C9000480CF80060B12F00801F780060D92000E8
:107CA000801F7800A10107008F00B1006641040029
:107CB00000000000420CF800440CF800E0B22F0075
:107CC000801F780060D92000801F7800970107008E
:107CD0008F00B10066410400000000004A0CF8006B
:107CE0004C0CF80060B42F00801F780060D9200091
:107CF000801F78008D0107008F00B10066410400ED
:107D000000000000716280006180500004003A00B1
:107D10006000470080007800943E040000000000EE
:107D2000640047008000780001007800801F780020
:107D3000E0B52F00801F780060D92000801F7800F8
:107D40007A0107006F00B1006641040000000000E6
:107D5000816280006180500004003A0068004700A2
:107D600080007800BA3E0400000000006C0047006C
:107D70008000780001007800801F780040B72F0055
:107D8000801F780060D92000801F780067010700FD
:107D90006F00B100664104000000000090628000A6
:107DA0000000E0000400320070004700800078000E
:107DB000E03E0400000000007700470080007800EB
:107DC00001007800801F7800A0B82F00801F780085
:107DD00060D92000801F7800540107006F00B100B7
:107DE0006641040000000000540CF800D0B92F00D8
:107DF000801F780060D92000801F78004B010700A9
:107E00006F00B1006641040000000000B062800015
:107E10000000E000050032000002200000004700E2
:107E2000800078001C3F0400000000004002200099
:107E3000000047008000780001007800801F780073
:107E400030BB2F00801F780060D92000801F780091
:107E5000360107006F00B100664104000000000019
:107E6000580CF80060BC2F00801F780060D92000FB
:107E7000801F78002D0107006F00B10066410400EB
:107E800000000000C06F80000000E000050032002C
:107E9000900220000000470080007800583F040056
:107EA00000000000D00220000000470080007800A1
:107EB00001007800801F7800C0BD2F00801F78006F
:107EC00060D92000801F7800180107006F00B10002
:107ED00066410400000000005A0CF8005C0CF80039
:107EE000F0BE2F00801F780060D92000801F78002E
:107EF0000E0107008F00B100664104000000000081
:107F00005E0CF800600CF80050C02F00801F780055
:107F100060D92000801F7800040107008F00B100A5
:107F20006641040000000000620CF800D0C12F0080
:107F3000801F780060D92000801F7800FB000700B8
:107F40006F00B10066410400000000004063800043
:107F50000000E00005003200300320000000470070
:107F600080007800BC3F0400000000007003200087
:107F7000000047008000780001007800801F780032
:107F800030C32F00801F780060D92000801F780048
:107F9000E60007006F00B100664104000000000029
:107FA000206380000000E00005003200B0032000E4
:107FB0000000470080007800E63F04000000000059
:107FC000E0032000000047008000780001007800F6
:107FD000801F780090C42F00801F780060D9200097
:107FE000801F7800D10007006F00B10066410400D7
:107FF00000000000306380000000E0000500320057
:108000003004200000004700800078001040040089
:10801000000000006004200000004700800078009D
:1080200001007800801F7800F0C52F00801F7800C5
:1080300060D92000801F7800BC0007006F00B100ED
:108040006641040000000000C07280000000E000F3
:1080500005003200B00420000000470080007800D6
:108060003A40040000000000D00420000000470057
:108070008000780001007800801F780050C72F0032
:10808000801F780060D92000801F7800A7000700BB
:108090006F00B1006641040000000000664104006A
:1080A00000000000680057009000780060805000D9
:1080B0004DFE32006800570090007800618050004B
:1080C00053FE320068005700900078006280500034
:1080D00059FE32006800570090007800638050001D
:1080E0005FFE320068005700900078006480500006
:1080F00064FE3200680057009000780065805000F0
:108100006AFE3200680057009000780066805000D8
:1081100070FE3200680057009000780067805000C1
:1081200076FE3200680057009000780068805000AA
:108130007CFE320068005700900078006980500093
:1081400082FE320068005700900078006A8050007C
:1081500088FE320068005700900078006B80500065
:108160008EFE320068005700900078006C8050004E
:1081700094FE320068005700900078006D80500037
:108180009AFE320068005700900078006E80500020
:10819000A0FE320068005700900078006F80500009
:1081A000A6FE3200680057009000780070805000F2
:1081B000ACFE3200680057009000780071805000DB
:1081C000B2FE3200680057009000780072805000C4
:1081D000B8FE3200680057009000780073805000AD
:1081E000BEFE320068005700900078007480500096
:1081F000C4FE32006800570090007800758050007F
:10820000D3FE32006800570090007800768050005E
:10821000E2FE32006800570090007800778050003E
:10822000F1FE32006800570090007800788050001E
:10823000F6FE320068005700900078007980500008
:1082400007FF320068005700900078007A805000E5
:108250000CFF320068005700900078007B805000CF
:108260001DFF320068005700900078007C805000AD
:1082700023FF320068005700900078007D80500096
:1082800029FF320068005700900078007E8050007F
:108290002EFF320068005700900078007F80500069
:1082A0003FFF320002022000E800570011001100D9
:1082B00050FF320012022000E800570011001100A8
:1082C00061FF32004E4004000000000060D9200031
:1082D000801F7800CB0A07002F00B1000080FA0051
:1082E000000006000200FA0000002000000F7800E5
:1082F00012022000E00047001100110009003C00BC
:1083000060004700901F780050FD07002F00B1006B
:1083100011002000600047001088400078410400F0
:10832000000000000080FA00000006000200FA00D1
:10833000E00047006A00570080087800811F78003D
:10834000901F780068005700901F7800D007070042
:108350006F00B1000080FA00000006000000FA0083
:10836000A2072000E80057001100110007003E009E
:1083700012062000E8005700110011000300390028
:10838000F1FD2F0068005700108860004EB897007C
:108390000080FA00000006000200FA000000200041
:1083A000000F7800680057009000780060004700D8
:1083B000108040009040780060C0500013003200F0
:1083C000711080000020200000806000C900DE00E5
:1083D0000100E00002003200E04104000000000063
:1083E00068005700100078006001470092004000CC
:1083F000114078000080FB008010880010002000F1
:1084000012094000D2410400000000000080FA0080
:10841000000006000C00FA0020002000000F780089
:108420000000200030079800680057009000780096
:1084300066004700108040009040780060C0500007
:108440000C003200680057001000780066014700F9
:1084500012004000904078008180FB0060004700DF
:108460001088680010002000120940001442040027
:108470000000000060004700901F7800D0CD2F0062
:10848000801F780062004700801F7800A7FF070068
:108490006F00B1000000200030079800E2004700A4
:1084A00066004700108040009040780060C0500097
:1084B00011003200E20047006600470050079800B4
:1084C0001080400040079800104078000080FB00BA
:1084D000801F7800A1FF07002F00B100CE009000A0
:1084E00080487800110020005E0090001088400055
:1084F0004E4204000000000062004700801F780028
:1085000068005700901F780020CE2F00801F780051
:1085100060D92000801F780084FF07008F00B10021
:1085200060D92000801F78009BFF07002F00B1005A
:108530000080FA00000006002A00FA0060004700F0
:10854000F1CE2F000E000900315878006F0047006F
:10855000E1CF2F0001000900315878007100470079
:1085600001D02F0001000900315878007300470046
:1085700021D02F0016000900315878006000470014
:10858000801F7800A3FF07002F00B1004EB89700AE
:108590000000E000060032006F004700801F7800F6
:1085A0009CFF07002F00B100E04204000000000023
:1085B00071004700801F780096FF07002F00B10070
:1085C00073004700801F780092FF07002F00B10062
:1085D0000080FA00000006000000FA00F1EF2F0012
:1085E00060082000108860004EB897000000E0008E
:1085F0000500320001102000E00820001088700003
:108600000A43040000000000F1EF2F00E008200002
:1086100010886000D1FF2F008021200010886000AA
:108620000080FA00000006000000FA00EA0057008F
:1086300011007800103B8800628040009040780074
:1086400020032000014878006C00570010007800DB
:10865000003B88000C0007000080FA0000000600C4
:108660000000FA0040042400801F78006A005700D0
:10867000B01F7800A01F7800EBFF07006F00B1006B
:108680000080FA00000006000000FA000500FC006F
:108690005C0520003C3B8800AC0A20003C3B880085
:1086A00061E7A80000000000000000000080FA0060
:1086B000000006000000FA006A005700B01F7800B2
:1086C000A01F7800E6FF07004F00B100013B8000CB
:1086D0000000280000806000CF00DE000100E00004
:1086E000020032006643040000000000EA00570068
:1086F00011007800C000880062804000904078003F
:1087000020032000014878006C005700100078001A
:10871000B00088000B0EBB0040002400003B880026
:10872000D9FF0700F1FF2B000076200010886000C1
:108730000080FA00000006000A00FA006A005700F4
:1087400010007800100798004EB9970032007800AA
:10875000A200780020079800310798000000200050
:10876000000F780060004700100278006C0157008D
:10877000120052001D003D001E009000901F780066
:108780006400470040079800B01F7800A01F7800E1
:10879000C8FF07006F00B100220020006200470000
:1087A0001008410022002000CF91DE004E00900012
:1087B0001018410010904900023B80000000280082
:1087C000000061004F01DE000200E0000200320004
:1087D000DC4304000000000012002000600047009D
:1087E00010084100B2430400000000006C00570074
:1087F000100078004100DD004EB99700CF80DE0008
:1088000012194000129148000080FA000000060092
:108810000200FA0000002000000F7800CEB8970098
:108820001100780010417800010320000140510040
:1088300016003900CEB8970011007800104178007A
:10884000910320000140510010003E0060024700EB
:1088500094007800A00020000089B900CEB89700ED
:1088600011007800104078000080FB00800041007B
:1088700000032000008A5000CEB8970010002000AE
:10888000910840000E440400000000001E00780023
:108890000080FA00000006000200FA00680057009D
:1088A00010007800000F78001E00780090407800DB
:1088B00060C050000B0032003EB99700110020004C
:1088C0006A005700108810000200E0000500320026
:1088D000110020006000470010884000544404004C
:1088E000000000006000470090007800680057001A
:1088F000108050000080FA00000006000000FA001E
:1089000002000700D2440400000000000400E00060
:1089100002003A001000070000000600811F7800E6
:108920000100E00002003D0060001000E08018003F
:108930000300E00002003D0060011100E081190029
:10894000050007004F00E00002003B00600010003F
:10895000E080180000000600020007000400BE00CE
:10896000000006006022B800060220000000D000CF
:108970008180D2000482D2008582D2000000A00053
:108980000202520083825A0003003B0002024200AE
:1089900083824A000000A1000603E900F3FF3A00C9
:1089A000000006000080FA00000006000000FA0047
:1089B0000200070024450400000000000400E0005D
:1089C00002003A001000070000000600839F6800C4
:1089D0000100E00002003D0060001000E08018008F
:1089E0000300E00002003D0060011100E081190079
:1089F000050007004F00E00002003B00600010008F
:108A0000E0801800000006006022B8000602200086
:108A10000000D0008180D2000482D2008582D20082
:108A20000000A0000202520083825A0003003B00B3
:108A30000202420083824A000000A1000603E9000E
:108A4000F3FF3A00000006000080FA000000060074
:108A50004C00FA0070778000202798000204200064
:108A6000740057001001610002003200B0788000ED
:108A700020279800740057001000780070016000F3
:108A800003003200E2FF2F0074005700100861005D
:108A90006E0057001001780062005100060035009A
:108AA000440220006E0157001200120002003C0038
:108AB00060450400000000000000200013013700A2
:108AC000740057001000780061016000040032005B
:108AD00000032000004178007445040000000000FD
:108AE0000002200000417800600047000248780042
:108AF0006101470000002000004978007400570021
:108B00001000780062016000290032006C005700FC
:108B100030017800A00178006000510060805900A9
:108B20000D003D0061014700D0022000004978009F
:108B30006C01570032007800A20078006019100024
:108B400060911800120020007000570010081100FA
:108B5000D8450400000000007400570010007800A1
:108B6000640160000800320061014700B00220008B
:108B70000049780012002000700057001008110012
:108B8000D845040000000000740057001000780071
:108B90006801600006003200610147000002200009
:108BA00000497800120020007000570010081100E2
:108BB0000202200074005700100161001000320012
:108BC0006E005700100178007000510005003A0057
:108BD0002200200070005700100811000046040019
:108BE000000000006E00570010017800680051007E
:108BF00003003A0012002000700057001008110016
:108C000000002000302798006C00570030017800E9
:108C1000A001780060005100608059000A003A000D
:108C20006200470064042000040247001401400071
:108C3000000320000049780010002000140A4000C2
:108C40006C460400000000006C0057003001780002
:108C5000A001780060005100608059001E003200C1
:108C60006201470060042000000047005027980080
:108C700010004100402798001EB997008001EB00CA
:108C80002EB89700BEB897000002EB001BFF07004C
:108C90004204200002014700120140004E209000D3
:108CA00012487800120020005E2090001008410059
:108CB0001EB997008001EB002EB89700BEB8970050
:108CC0000002EB0039FF070020BF9F0031BF9F006B
:108CD000244604000000000060042000000047005B
:108CE0001002780072015700120052000400340094
:108CF00060042000000047001000780070B79F005B
:108D00007200570010017800700057001008110021
:108D10007400570010007800710160000E003A00E6
:108D20000EBA9700120020007000570010081100C2
:108D300060005200080034004EB997000002200085
:108D40000049780012002000680057001008410018
:108D500090460400000000001E4090000004E00067
:108D600006003200610147004EB8970012487800B3
:108D70001200200068005700100841000202200085
:108D800074005700100161001D0032006E00570092
:108D9000100178006800510008003A004EB99700B1
:108DA00000032000004978001200200068005700EE
:108DB0001008410000470400000000006E0057004A
:108DC00010017800700051000D003A004EB9970074
:108DD0000003200000497800E802570015007800E1
:108DE0006102400044BF9F0012022000E0EE20001C
:108DF00010004100104A780010002000950A400041
:108E00007400570010007800700160000E003A00F6
:108E10000EBA9700120020007000570010081100D1
:108E20006000520008003400600147004EB897000F
:108E30001248780012002000680057001008410016
:108E400008470400000000007EB2970012002000D6
:108E50007200570010081100620420000201470050
:108E60001200120008003D004EB9970000032000D8
:108E700000497800120020006800570010084100E7
:108E800024470400000000003E2290001200200051
:108E9000600420000000470010081100600052002C
:108EA0000B0034006201470060042000000047000E
:108EB000100141004EB897001248780012002000BF
:108EC00068005700100841004447040000000000FB
:108ED0000EBA970012002000700057001008110011
:108EE00060005200080034004EB9970000022000D4
:108EF0000049780012002000680057001008410067
:108F000068470400000000004EB897000080FA0097
:108F1000000006001E00FA0070778000400F9800E5
:108F200001042000700057009080600002003200B1
:108F3000B0788000400F980000002000600F98007B
:108F400000002000500F98007A0047009000780041
:108F5000668050002E003D007A00470090007800A7
:108F60006080500007003200600047007C0147002D
:108F700092004000A00320008048780010002000EC
:108F800012094000E00347007C03470016814300BC
:108F9000EA025700150078007A024700940040006A
:108FA000114078000080FB004400DE00F80147001B
:108FB0001300400010497800060078001000780087
:108FC00061004000600F98000081430005007800B8
:108FD0009000780004007800108040001040780075
:108FE0000080FB00EF00600003007800108040006C
:108FF0001049780010002000160B400011002000DE
:109000007A00470010884000A447040000000000D8
:109010007000570010007800F00060000F003A0068
:109020002EB99700110020006C0057001088100026
:10903000FC0047001100110008003D00CEB8970069
:1090400000022000804878001100200068005700CE
:1090500010884000104804000000000000002000BC
:10906000500F98007A00470010017800FC0047007C
:10907000110051000D003D00E00047007A0047005C
:10908000908040004EB897001148780011002000F1
:109090006800570010884000110020007A00470047
:1090A0001088400032480400000000002EB99700EC
:1090B000110020006C00570010881000FC004700D1
:1090C0001100110008003D00CEB8970000022000FA
:1090D0008048780011002000680057001088400088
:1090E00056480400000000004EB897000080FA00C7
:1090F000000006002800FA0000002000600F980021
:1091000000002000400F980078004700100278000F
:109110006400520082003D00780047001002780091
:10912000600052000700320060004700FC02470068
:1091300015024000E0022000004A780010002000E4
:10914000950A40006A005700100278007800470036
:1091500010024200144078000080FB00500F98007D
:109160007A004700100278006000520009003A00BF
:1091700060004700FC024700150240007077800045
:10918000104A780010002000950A4000864904002B
:1091900000000000450620007A02470014801200FB
:1091A0003400350060024700341798007C00470007
:1091B0002017980010004200700F9800440620000D
:1091C0007A0047001017980010007800110009007D
:1091D0000400D800E4EE20000417980014024000B8
:1091E0007E089000144878002E109000100078003F
:1091F00061004000700F9800600F98004406200046
:109200001E10900010007800110009000400D80022
:1092100001007800500F9800BE1290007E0A900066
:1092200004824200740F9800A4002000110009007D
:109230000400D8000E129000140240007E08900036
:1092400014487800140020002E10900010084200EE
:109250001E10900010027800A200200011000900EA
:109260000202D80001007800500F980074490400F1
:10927000000000007A004700100278006A005200E7
:1092800019003500600247007C0047001017980065
:1092900010004200001798007A004700700F9800F5
:1092A00010027800A2002000110009000202D8007C
:1092B000E4EE2000140240000E10900014487800E4
:1092C000140020001E109000100842007E0890003C
:1092D00010027800A2002000110009000202D8004C
:1092E00001007800500F9800600047007C034700A1
:1092F00096024000747780007A0047001000420018
:10930000904A780010002000160B40001400200046
:109310007800470010084200844804000000000064
:109320007000570010007800700260000F003A00D3
:10933000AEBA9700140020006C005700100812000D
:109340007C0247001480120008003D004EBA9700CE
:1093500000022000004A7800140020006800570036
:10936000100842009849040000000000000020009E
:10937000400F980078004700900278007C02470078
:10938000148052000D003D00600247007800470045
:10939000100242004EB897001448780014002000D4
:1093A00068005700100842001400200078004700B1
:1093B00010084200BA49040000000000AEBA97004D
:1093C000140020006C005700100812007C024700B7
:1093D0001480120008003D004EBA970000022000E1
:1093E000004A78001400200068005700100842006E
:1093F000DE490400000000004EB897000080FA002B
:10940000000006000000FA003EB89700CEB89700B2
:10941000100007000081EB00E50C07002EB9970053
:1094200000197800011178002EB89700B00178007B
:10943000200278006A01570032007800A20078000C
:109440000301780084017800C60D07000080FA004F
:10945000000006000000FA00020007009E4A040017
:10946000000000000001BE001F0007000470A700FC
:1094700003F0A1006509B100160032000D003500AF
:109480006828E10006003500F0FF2F00F1FF2700FB
:109490000300E00013003B0001002800000005006D
:1094A00000004000818048008502E900FCFF3A008E
:1094B00008003700F88F420002003C008000EB00FB
:1094C000000005008100D1000080D3008502E80083
:1094D000FCFF3A000300E00002003B0060001000C7
:1094E000E080180000000600C70ADE00F107B200A5
:1094F000F50FB20008003200E1CF42000200320056
:109500000170A00024000500810F700001003200EE
:109510000408050044000500810F700002003A00B5
:10952000140005008502E9000000400081C04800E9
:10953000FCFF3B000170A000240005000080FA0041
:10954000000006001000FA006C00570010017800BF
:109550006000510002003D000000200020BF9F007D
:10956000F40420006C0157001200120002003500C4
:10957000E004200020BF9F0000002000000F7800C2
:109580000EB9970000002000000978007200570013
:1095900010007800500798006A01570032007800E8
:1095A000A20078000200200003002000AB0D07009D
:1095B0000000E0000200350000002000010037003C
:1095C000100020000000E000080032000EB99700F3
:1095D000100020000009780002002000030028008D
:1095E0006A00570010186900109069006200470077
:1095F00070079800801F78006A005700B01F78003D
:10960000A01F78007FFF07006F00B10030BF9F00F0
:1096100041BF9F0004052000720157006C00470005
:10962000120842007E0090000001780032007800AD
:10963000A20078000200200003002000870D070030
:109640000000E00002003A000000200001003700A6
:10965000100020000000E000460032000405200059
:10966000720157006C004700120842006201470077
:1096700032007800A20078000200200003002000E1
:10968000760D07000000E00002003A000000200014
:1096900001003700100020000000E000220032002E
:1096A00062004700801F780002002000031224009F
:1096B0001E009000AE009000230E0700801F78006F
:1096C000811F78004FFF07006F00B100300798003E
:1096D000410798006C0147001201780061015100B8
:1096E0007207980062079800F2282C0053CF2300DD
:1096F0005F0D07000200200003122400870C070002
:1097000054FF0700040320007E019000044940003C
:109710007E00900012002000600047001008410009
:10972000364B0400000000000205200072005700C4
:10973000100241006C014700120012000B003100C2
:109740006E0190005E009000124878001200200028
:109750006A00470010084100120020006C0047001A
:1097600010084100944B0400000000000E4C04005F
:10977000000000006A01570032007800A200780063
:109780000200200003002000F10C07000000E000B0
:1097900002003C0000002000010037001000200003
:1097A0000000E0001D0032003EB89700CEB89700E0
:1097B0000200200003122400580C07003007980014
:1097C0004107980000017800810178000000200026
:1097D00001F82300DE0C07000000E00002003C005E
:1097E0000000200001003700100020000000E00011
:1097F0000A0032006601470032007800A2007800BB
:1098000030BF9F0041BF9F00120020006000470052
:1098100010081100D44B0400000000007200570033
:10982000100278006C0157006C00470012084200DB
:1098300074005700100178006000510004003A00E5
:1098400060004700100178006C00470010084100DC
:109850001EB99700600047001000780000097800EA
:109860006C0047001002780072015700120052008D
:10987000050031007EB1970000002000004978000B
:109880007EB09700690037006A0047001002780038
:109890006C0147001200520020003E00020520002B
:1098A00072005700100241006A01470012001200C6
:1098B0001A0031003EB89700CEB897000200200091
:1098C00003122400150C070030BF9F0041BF9F000A
:1098D00066014700821F7800801F7800811F780092
:1098E000C8FE07006F00B10030BF9F0041BF9F005E
:1098F0003E009000CE009000D6FE0700040320003A
:109900005E01900004494000120020006A004700F8
:1099100010084100444C0400000000000205200033
:1099200072005700100241006C0147001200120043
:1099300007003900F20420007200570010014100B6
:1099400000002000004978007EB097003700370003
:109950006C00470010007800500798006E019000DE
:1099600050002000124940006E0090001042780024
:109970009203200002405200280036006E01900041
:1099800000032000004978006C00470010027800B6
:109990007201570012005200090036006C004700A7
:1099A0001000780061015000620798000200780002
:1099B00010407800614940000A4D0400000000009A
:1099C0006E01900010032000004978001EB9970036
:1099D00010002000120940007400570010017800A8
:1099E000600051000B003A006A0047001002780046
:1099F0007201570012005200030036005E01900011
:109A00000003200000497800120020006A0047008F
:109A100010084100B44C0400000000005E019000FA
:109A200000002000004978007EB097000080FA0016
:109A3000000006005800FA000000200030079800DF
:109A40006E0057001041780061062000014051006F
:109A50008F003A0000002000801F78006800470057
:109A6000801F780062004700801F78006000470078
:109A7000801F780070005700901F78006A00570020
:109A8000B01F7800A01F7800AEFE0700EF00B10005
:109A9000300798001E0090000000E0000600320031
:109AA000AEB89700D0022000804878001100200056
:109AB0006C00570010884000BE0090001104E000C8
:109AC0005100320060004700900078006080500034
:109AD0002E003C00AEB897000003200080487800BC
:109AE0006C01570012007800E100400021BF9F0088
:109AF000E002200080487800100020001209400099
:109B00000000200020079800600047001000780047
:109B100060011000E4004700110011000B003D003F
:109B2000AEB89700000320008048780011002000A4
:109B30006C005700108840001100200064004700AE
:109B400010884000844D040000000000BE0090001A
:109B50001104E0000B003200BE0090002EB8970008
:109B600011487800110020006C0057001088400058
:109B7000110020006600470010884000A64D040038
:109B800000000000004E0400000000000000200063
:109B900020079800BE0090001104E0001800320079
:109BA0002E01900011002000640047001088400042
:109BB000E00047001100510006003A00AEB89700DF
:109BC000E002200080487800110020006C0057005F
:109BD00010884000BE0090002EB897001148780011
:109BE000110020006C005700108840001100200078
:109BF0006600470010884000CA4D040000000000C5
:109C0000484E040000000000AEB89700000320009A
:109C100080487800110020006C0057001088400038
:109C200070005700900078006080500018003400E9
:109C3000AEB89700E00220008048780011002000B4
:109C40006C0057001088400000002000200798009A
:109C50006400470010017800F00057001100510027
:109C60000B003D00AEB8970000032000804878004C
:109C7000110020006C0057001088400011002000E7
:109C80006400470010884000284E040000000000D7
:109C9000AEB8970000002000804878000080FA00ED
:109CA000000006000200FA00CEB897001104E000A0
:109CB000190032004EB8970010417800E1022000F0
:109CC0000140510001003A003A0037004EB89700B9
:109CD0001041780051062000014051000700320079
:109CE0004EB8970010417800510420000140510007
:109CF00002003200824E0400000000008C4E04007E
:109D0000000000001100200068005700108840008B
:109D1000544E040000000000CEB897001104E0008B
:109D20001B00320068005700901F780005040700F0
:109D30002F00B100000F780060004700900078000D
:109D4000608050000D003400E001470013007800EF
:109D5000E10040006800570010814000900078004A
:109D600003007800108040001049780010002000A7
:109D7000930910009C4E040000000000CEB897002C
:109D8000E002200080487800DA4E04000000000065
:109D9000CEB89700E00220008048780068005700A5
:109DA00010007800E100400041BF9F00000020004B
:109DB000804878000080FA00000006000200FA00E7
:109DC000CEB897001104E0000A0032004EB89700A8
:109DD00010417800E10220000140510005003200EE
:109DE000110020006800570010884000E04E040079
:109DF000000000004EB997001100200068005700D5
:109E0000108840001204E00037003200CEB89700FE
:109E10001104E0000F0032004EB8970010417800A6
:109E200051062000014051000A0032004EB8970050
:109E3000104178005104200001405100050032001B
:109E4000110020006800570010884000064F0400F1
:109E500000000000E800570011007800000F7800B3
:109E600010002000910810004EB8970010417800B3
:109E7000010320000140510005003A0011002000BC
:109E80006800570010881000344F040000000000E4
:109E90004EB8970010417800E102200001405100C7
:109EA00003003A00110020006800570010881000DD
:109EB0006800570010007800E101400043BF9F0098
:109EC0001E0178001100200060004700108840004B
:109ED00092497800CEB897001104E00002003200E9
:109EE000584F0400000000000080FA000000060047
:109EF0005600FA00740057001000780070016000EE
:109F000003003200E2FF2F007400570010086100C8
:109F100074005700100078006101600004003200F6
:109F200000032000004178009C4F04000000000066
:109F300000022000004178000005200000004700DA
:109F400002487800120520000201470000002000AE
:109F5000004978007400570010007800620160002A
:109F6000330032006C01570032007800A200780004
:109F70000200200003002000380B07000000E00072
:109F80000200350000002000010037001000200012
:109F90000000E0000E003200120520000201470020
:109FA000D0022000004978000200200003002800B1
:109FB0006C00570010186900109069001200200012
:109FC0006E00570010081100185004000000000037
:109FD000740057001000780064016000090032002E
:109FE0001205200002014700B0022000004978005D
:109FF000120020006E0057001008110018500400D5
:10A000000000000074005700100078006801600034
:10A010000700320012052000020147000002200064
:10A0200000497800120020006E005700100811004F
:10A0300070005700100178006000510004003D00DE
:10A040006000200000BF9F003E50040000000000A0
:10A0500070005700100178006000510007003A00BE
:10A060007200570010427800720620000240520031
:10A0700002003A001000200000BF9F00700057004F
:10A08000901F780072005700104078000080FB009D
:10A09000801F780060004700801F78006C00570028
:10A0A000B01F7800A01F780062FE0700AF00B1006B
:10A0B0000202200074005700100161000800320005
:10A0C00070005700100178006000510004003A0051
:10A0D00060004700801F7800F2FE07002F00B100EB
:10A0E00072005700104278007206200002405200B1
:10A0F00008003A00020220007400570010016100BD
:10A1000004003A0060004700801F78002BFF070022
:10A110002F00B10060004700801F7800090307008E
:10A120002F00B100102F98006E0157001209100087
:10A130007400570010007800710160000E003A00B2
:10A140001EBA9700120020006E0057001008110080
:10A1500060005200080034004EB997000002200051
:10A1600000497800120020006800570010084100E4
:10A17000A0500400000000001ED090000004E00089
:10A180000700320012052000020147004EB8970078
:10A1900012487800120020006800570010084100A3
:10A1A0007400570010007800700160000F003A0042
:10A1B0001EBA9700120020006E0057001008110010
:10A1C000600052000900340002052000020147002F
:10A1D0004EB897001248780012002000680057001F
:10A1E00010084100D85004000000000000002000CA
:10A1F000202F980040052000000047001002780042
:10A200002205200002014700120052000F003D000D
:10A210006001470040052000000047001001410098
:10A220004EB89700124878001200200068005700CE
:10A2300010084100120020004005200000004700E7
:10A2400010084100FA500400000000001EBA9700F8
:10A25000120020006E00570010081100600052002C
:10A26000080034004EB99700000220000049780031
:10A270001200200068005700100841002651040019
:10A28000000000004EB897000080FA0000000600B1
:10A290001E00FA006000470091D12F00060009005F
:10A2A000315878006800570010007800100F9800AF
:10A2B0003EB997001204E000990232003EB89700C0
:10A2C000904178005202200002C051000800320084
:10A2D0003EB997001E089000124878001200200036
:10A2E000720047001008410086560400000000007C
:10A2F00000002000300F9800120020006A00570074
:10A3000010084100B85104000000000002012000C4
:10A3100076004700100871007C5104000000000026
:10A320004200200076004700100871007C510400B4
:10A330000000000082002000760047001008710035
:10A340007C5104000000000002022000760047005B
:10A35000100871007C510400000000001200200071
:10A3600076004700100871007C51040000000000D6
:10A370003EB8970090417800D202200002C0510000
:10A38000E2FF32003EB8970090417800B202200010
:10A3900002C05100E2FF32003EB8970090417800C1
:10A3A0000202200002C05100E2FF32003EB89700D6
:10A3B000904178003202200002C05100E2FF3200DA
:10A3C0003EB89700904178000203200002C051007F
:10A3D000E2FF3200F0FF2F00400F98003EB89700D8
:10A3E000904178000203200002C051000C003900A7
:10A3F0003EB89700904178009203200002C05100BF
:10A4000007003E006A005700801F780000F907002F
:10A410002F00B100400F98003E52040000000000E1
:10A420003EB8970090417800A202200002C051007F
:10A4300012003A00120020006A0057001008410084
:10A44000AEB997002EB99700200020001209100025
:10A450001300780010017800420F9800600051004E
:10A4600006003D00780147001200780060091000E6
:10A47000020120007600470010087100F0FF2F0055
:10A48000500F98003EB8970090417800E2022000FB
:10A4900002C0510029003A006A00570010007800FD
:10A4A0006100400030BF9F0090417800020320000F
:10A4B00002C051000C0039003EB89700904178006E
:10A4C0009203200002C0510007003E006A005700BE
:10A4D000801F7800CEF807002F00B100500F9800C1
:10A4E00092520400000000003EB8970090417800AE
:10A4F000A202200002C051000A003A00120020000F
:10A500006A00570010084100AEB997002EB99700B5
:10A5100020002000120910001301780012007800BA
:10A52000500F98007A004700100178006000510039
:10A5300002003D0000002000500F9800F0FF2F00A7
:10A54000600F98003EB89700904178008206200086
:10A5500002C051000C0032003EB8970090417800D4
:10A56000C206200002C05100070032003EB897002A
:10A5700090417800C204200002C051000200320065
:10A58000D2520400000000003EB99700124078004B
:10A590000080FB00600F9800120020006A00570046
:10A5A00010084100A0002000000F98002A55040068
:10A5B0000000000076004700100078007001600085
:10A5C0000E003A007800470010007800610150004A
:10A5D000420F980060005100080034001E099000EE
:10A5E000000220000049780012002000720047009D
:10A5F00010084100E252040000000000AEB99700CC
:10A600002EB99700200020001209100013017800D5
:10A610001E089000124878001200200072004700C7
:10A6200010084100780047001000780061015000D8
:10A63000420F980060005100080034001E0990008D
:10A64000000220000049780012002000720047003C
:10A650001008410012530400000000008656040058
:10A6600000000000AEB997002EB99700200020002E
:10A67000120910001300780010017800220F9800D2
:10A680006000510002003A0060004700200F98006F
:10A690007A004700901F780074004700901F7800F0
:10A6A0007DF807004F00B100400798007600470092
:10A6B00010007800700160000F003A00CE09900091
:10A6C00012002000780047001008110068014700C0
:10A6D0001280110008003D001E09900000022000B9
:10A6E0000049780012002000720047001008410065
:10A6F0005E53040000000000000020007007980076
:10A700006E004700900178006801470012805100F8
:10A710000E003D002E0990001E089000124878009F
:10A7200012002000720047001008410012002000B3
:10A730007400470010084100120020006E0047001E
:10A74000100841008053040000000000CE09900072
:10A75000120020007800470010081100680147002F
:10A760001280110008003D001E0990000002200028
:10A7700000497800120020007200470010084100D4
:10A78000A6530400000000008656040000000000EC
:10A79000F3FF2F00780147001280110005003A00F6
:10A7A00040002000400F9800120020007600470073
:10A7B0001008710076004700901F78007A0047006B
:10A7C000901F780078004700901F7800000120005B
:10A7D000801F7800AEB997002EB9970020002000A6
:10A7E0001209100013007800100078008000EB00C0
:10A7F000801F7800811F780072004700901F78004A
:10A8000093F80700EF00B100100F9800865604007F
:10A8100000000000C30620007C01470012801100E8
:10A820000F003A00AEB997002EB997002000200023
:10A8300012091000130078009001780072004700A0
:10A840001001780068005700100051008000EB00F4
:10A850008019780081117800445404000000000041
:10A86000AEB997002EB99700200020001209100001
:10A870001300780090017800720047001001780002
:10A88000680057009009510086560400000000003F
:10A89000020420007600470010087100C306200063
:10A8A0007C0147001280110013003A007600470037
:10A8B000901F78007A004700901F780078004700CA
:10A8C000901F7800AEB997002EB9970020002000A5
:10A8D0001209100013007800901F780072004700E2
:10A8E000901F78008BF90700AF00B100100F98009F
:10A8F0009E5404000000000076004700901F78007E
:10A900007A004700901F780078004700901F780079
:10A91000AEB997002EB99700200020001209100050
:10A9200013007800901F780072004700901F780095
:10A93000F0F90700AF00B100100F98008656040030
:10A940000000000080002000000F9800D85504008F
:10A95000000000000204200076004700100871008B
:10A9600000012000000F9800D855040000000000EE
:10A97000220020007600470010087100D85504001E
:10A9800000000000760047001000780062007000B0
:10A99000801F78003EB9970012407800801F780031
:10A9A0007A004700901F780078004700901F7800D9
:10A9B000AEB997002EB99700400020001209100090
:10A9C00013007800B01F7800A01F780072004700C5
:10A9D000901F780046FD0700EF00B100100F9800AF
:10A9E00086560400000000003EB8970090417800B1
:10A9F0005202200002C05100060032001E099000E1
:10AA00005002200000497800120020007200470028
:10AA1000100841003EB997001204E000080032001F
:10AA20003EB997001E0890001248780012002000DE
:10AA30007200470010084100265504000000000085
:10AA4000120020006A00570010081100865604000A
:10AA5000000000003EB897009041780032062000C8
:10AA600002C05100D3FE32003EB8970090417800FA
:10AA70003207200002C05100FAFE32003EB89700B3
:10AA8000904178000207200002C0510040FF3200D0
:10AA90003EB8970090417800E206200002C05100C5
:10AAA0005CFF32003EB8970090417800120420000D
:10AAB00002C0510076FF32003EB897009041780006
:10AAC0001206200002C0510074FF32003EB8970009
:10AAD00090417800F206200002C0510099FF320038
:10AAE0003EB89700904178008205200002C05100D6
:10AAF00098FF32003EB8970090417800820720000E
:10AB000002C0510096FF32003EB897009041780095
:10AB10004206200002C0510095FF32003EB8970067
:10AB2000904178009206200002C0510090FF320050
:10AB30003EB89700904178005207200002C05100B3
:10AB40008EFF32003EB897009041780052042000FA
:10AB500002C051008BFF32003EB897009041780050
:10AB60007204200002C0510086FF32003EB89700F8
:10AB7000904178005206200002C0510081FF32004F
:10AB80003EB89700904178006206200002C0510054
:10AB90007CFF32003EB8970090417800720620009A
:10ABA00002C0510077FF3200F4540400000000009E
:10ABB000C30620007C014700128011000B003A0000
:10ABC000AEB997002EB9970040002000120910007E
:10ABD0001301780032007800A20078005007980036
:10ABE00061079800665604000000000083062000FC
:10ABF0007C014700128011001C003A0076004700DB
:10AC000010007800620160000C003200AEB99700BD
:10AC10002EB99700100020001209100013017800CF
:10AC2000124078000000FB00CF80DE005007980043
:10AC3000610798003256040000000000AEB997008A
:10AC40002EB997001000200012091000130178009F
:10AC5000124078000080FB008000EB005007980055
:10AC60006107980066560400000000007600470067
:10AC700010007800620160000B003200AEB997004E
:10AC80002EB997002000200012091000130178004F
:10AC900012007800CF80DE0050079800610798000E
:10ACA0006656040000000000AEB997002EB9970068
:10ACB0002000200012091000130178001200780013
:10ACC0008000EB005007980061079800760047006D
:10ACD000901F78007A004700901F780078004700A6
:10ACE000901F780070004700901F78006A004700AE
:10ACF000B01F7800A01F780072004700901F7800F6
:10AD000053F70700EF00B100100F98001200200069
:10AD10006A0057001008410058510400000000006C
:10AD20001E099000000020000049780072004700D2
:10AD30001001780068005700100051000080FA00F0
:10AD4000000006000200FA006800570010007800BA
:10AD5000000F78001E0178001100200060004700FD
:10AD6000108840001204E00002003200AA560400DD
:10AD70000000000060004700900078006800570065
:10AD800010805000610050000080FA0000000600B2
:10AD9000C822A90020C2A9002022AF00CC5604007E
:10ADA00000000000F00F2000201188002002AE00FB
:10ADB000D65604000000000020118000F10F200092
:10ADC0000104E100F3FF3A0020C2A9002022AF00F5
:10ADD000E6560400000000000000EB00201188008F
:10ADE0002002AE00F0560400000000002011800098
:10ADF000F000B200110020000008DD00C822A80009
:10AE0000000006000200FA0068005700901F78005A
:10AE1000CCFF07002F00B100000F7800DCFF070017
:10AE20006001470092001000020036000E57040037
:10AE300000000000C822A9006800570090007800B8
:10AE4000314078000080FB00060032002022AF0075
:10AE5000265704000000000020118800205704003D
:10AE600000000000C822A8000080FA0000000600D0
:10AE70003E00FA00E00047006800570080087800B4
:10AE8000811F7800901F780062004700801F7800C3
:10AE9000FFFC07006F00B10062004700801F7800D0
:10AEA000D8FF07002F00B1000080FA000000060064
:10AEB0000000FA0068005700901F780000D22F00B1
:10AEC000801F7800EAFF07004F00B1000080FA0001
:10AED0000000060050042000801F7800F4FF0700E7
:10AEE0002F00B100000006000A00FA00B0728000D6
:10AEF00010079800C2122000CF91DE00A0E52000CC
:10AF000030021100A082190002D02000320012008D
:10AF100022801A0010003D00B2728000E0C42000C0
:10AF200010014100B27288006000510002003D0033
:10AF300000002000B07288001402200062E52000AA
:10AF4000120012000200340010022000B0728800CB
:10AF5000A063040000000000C2122000CF91DE00B8
:10AF6000A0E5200030024100A082490002D020006C
:10AF70003200120022801A0010003400B2728000E9
:10AF8000E0C4200010015100B2728800600051003E
:10AF900002003D0000002000B07288001402200072
:10AFA00062E52000120012000200340010022000AE
:10AFB000B0728800A06304000000000000002000C0
:10AFC000000F7800C2122000CF91DE00E0E52000E3
:10AFD00030024100A082490082CF200032001200DE
:10AFE00022801A000400340010002000000F7800B6
:10AFF0001258040000000000C2122000CF91DE00B1
:10B00000E0E5200030021100A082190082CF20006C
:10B010003200120022801A0002003D00F0FF2F00D3
:10B02000000F7800600047001001780000C5200084
:10B030001091B900020F780060005100C005320085
:10B040001402200062E52000120012000600320007
:10B0500010002000C072880010022000801F7800BD
:10B06000FAF107002F00B100C662040000000000E2
:10B0700002608000136080000000200001F82300BF
:10B08000F60607000000E000020034000000200087
:10B0900001003700100020000000E0000600320030
:10B0A00060004700100178006000510002003D0080
:10B0B00084580400000000000260800013608000DB
:10B0C00000F82400317C2400A10607000000E00005
:10B0D00002003C00000020000100370010002000AA
:10B0E0000000E00006003200600047001001780018
:10B0F0006000510002003400845804000000000089
:10B1000096580400000000001E007800CF80DE008A
:10B110000081EB00A605070002608000136080003C
:10B12000D306070000608800116088009A6304005D
:10B13000000000002260800033608000A0702D00BD
:10B1400031C22300C50607000000E0000200340001
:10B150000000200001003700100020000000E00087
:10B1600006003200600047001001780060005100C6
:10B1700002003D00E658040000000000226080004C
:10B18000336080000000200001F8230070060700F3
:10B190000000E00002003C00000020000100370039
:10B1A000100020000000E0000600320060004700B0
:10B1B000100178006000510002003400E6580400DD
:10B1C00000000000FE580400000000001E0078008F
:10B1D000CF80DE000081EB0075050700A2702D0016
:10B1E00033C22300CD050700226080003360800059
:10B1F0009F06070020608800316088009A63040081
:10B20000000000004260800053608000D0CC2C0021
:10B21000C1E42300910607000000E00002003400B2
:10B220000000200001003700100020000000E000B6
:10B2300006003200600047001001780060005100F5
:10B2400002003D004E5904000000000042608000F2
:10B250005360800030332300F11924003C060700BE
:10B260000000E00002003C00000020000100370068
:10B27000100020000000E0000600320060004700DF
:10B280001001780060005100020034004E590400A3
:10B290000000000066590400000000001E00780055
:10B2A000CF80DE000081EB0041050700D2CC2C00EE
:10B2B000C3DC2300990507004260800053608000D2
:10B2C0006B06070040608800516088009A630400A4
:10B2D0000000000062608000610051000600340040
:10B2E00060004700100178006000510002003D003E
:10B2F000945904000000000054092000C2C020003E
:10B300001200120006003D006000470010017800A6
:10B310006000510002003400945904000000000055
:10B320009C590400000000006000470010017800F4
:10B33000C0C02000100841009A6304000000000013
:10B3400072608000836080000000200001F823000C
:10B35000420607000000E000020035000000200067
:10B3600001003700100020000000E000060032005D
:10B3700060004700100178006000510002003D00AD
:10B38000EC590400000000007260800083608000BF
:10B3900000F82400317C2400ED0507000000E000E7
:10B3A00002003C00000020000100370010002000D7
:10B3B0000000E00006003200600047001001780045
:10B3C0006000510002003400EC590400000000004D
:10B3D000FE590400000000001E007800CF80DE004F
:10B3E0000081EB00F204070072608000836080003F
:10B3F0001F06070070608800816088009A6304005F
:10B400000000000092608000A3608000D0CC2C007F
:10B41000C1DC2300110607000000E0000200350037
:10B420000000200001003700100020000000E000B4
:10B4300006003200600047001001780060005100F3
:10B4400002003D004E5A040000000000926080009F
:10B45000A3608000D0CC2C00712C2400BC05070018
:10B460000000E00002003C00000020000100370066
:10B47000100020000000E0000600320060004700DD
:10B480001001780060005100020034004E5A0400A0
:10B4900000000000665A0400000000001E00780052
:10B4A000CF80DE000081EB00C1040700D2CC2C006D
:10B4B000C3DC23001905070092608000A3608000B0
:10B4C000EB05070090608800A16088009A63040083
:10B4D00000000000B0608000C16080000200200019
:10B4E000030020009A0507000000E00002003C0075
:10B4F0000000200001003700100020000000E000E4
:10B500000600320060004700100178006000510022
:10B5100002003D00B65A040000000000B260800046
:10B52000C36080000000200041242400880507003B
:10B530000000E00002003C00000020000100370095
:10B54000100020000000E00006003200600047000C
:10B55000100178006000510002003400B65A040067
:10B5600000000000C85A0400000000001E0078001F
:10B57000CF80DE000081EB008D040700B260800008
:10B58000C3608000BA050700B0608800C160880011
:10B590009A63040000000000D2608000E360800035
:10B5A000D0CC2C00C1DC2300AC0507000000E0007B
:10B5B00002003500000020000100370010002000CC
:10B5C0000000E00006003200600047001001780033
:10B5D0006000510002003D00185B04000000000004
:10B5E000D2608000E3608000D0CC2C00712C24005D
:10B5F000570507000000E00002003C0000002000AA
:10B6000001003700100020000000E00006003200BA
:10B610006000470010017800600051000200340013
:10B62000185B040000000000305B04000000000014
:10B630001E007800CF80DE000081EB005C04070074
:10B64000D2CC2C00C3DC2300B4040700D2608000FD
:10B65000E360800086050700D0608800E160880014
:10B660009A63040000000000F26080000361800023
:10B67000D0CC2C00C1DC2300780507000000E000DE
:10B6800002003500000020000100370010002000FB
:10B690000000E00006003200600047001001780062
:10B6A0006000510002003D00805B040000000000CB
:10B6B000F260800003618000D0CC2C00712C24004B
:10B6C000230507000000E00002003C00000020000D
:10B6D00001003700100020000000E00006003200EA
:10B6E0006000470010017800600051000200340043
:10B6F000805B040000000000985B04000000000074
:10B700001E007800CF80DE000081EB0028040700D7
:10B71000D2CC2C00C3DC230080040700F260800040
:10B720000361800052050700F06088000161880015
:10B730009A63040000000000106180002161800015
:10B740000200200003002000010507000000E000C7
:10B7500002003C0000002000010037001000200023
:10B760000000E00006003200600047001001780091
:10B770006000510002003D00E85B04000000000092
:10B780001261800023618000000020004124240019
:10B79000EF0407000000E00002003C000000200071
:10B7A00001003700100020000000E0000600320019
:10B7B0006000470010017800600051000200340072
:10B7C000E85B040000000000FA5B040000000000D9
:10B7D0001E007800CF80DE000081EB00F40307003C
:10B7E000126180002361800021050700106188003C
:10B7F000216188009A63040000000000326180002B
:10B80000436180000000200001F8230013050700B9
:10B810000000E000020035000000200001003700B9
:10B82000100020000000E000060032006000470029
:10B83000100178006000510002003D004A5C0400E5
:10B8400000000000326180004361800000002000A1
:10B85000612C2400BE0407000000E00002003C0050
:10B860000000200001003700100020000000E00070
:10B8700006003200600047001001780060005100AF
:10B88000020034004A5C0400000000005C5C04001C
:10B89000000000001E007800CF80DE000081EB0079
:10B8A000C30307003261800043618000F004070099
:10B8B00030618800416188009A6304000000000044
:10B8C0005261800063618000D0CC2C00C1DC230079
:10B8D000E20407000000E000020035000000200044
:10B8E00001003700100020000000E00006003200D8
:10B8F00060004700100178006000510002003D0028
:10B90000AC5C0400000000005261800063618000B4
:10B91000D0CC2C00712C24008D0407000000E00026
:10B9200002003C0000002000010037001000200051
:10B930000000E000060032006000470010017800BF
:10B940006000510002003400AC5C04000000000004
:10B95000C45C0400000000001E007800CF80DE0000
:10B960000081EB0092030700D2CC2C00C3DC230043
:10B97000EA0307005261800063618000BC04070095
:10B9800050618800616188009A6304000000000033
:10B9900072618000836180000000200001F82300B4
:10B9A000AE0407000000E0000200350000002000A7
:10B9B00001003700100020000000E0000600320007
:10B9C00060004700100178006000510002003D0057
:10B9D000145D04000000000072618000836180003B
:10B9E00000002C0091472400590407000000E000EB
:10B9F00002003C0000002000010037001000200081
:10BA00000000E000060032006000470010017800EE
:10BA10006000510002003400145D040000000000CA
:10BA2000265D0400000000001E007800CF80DE00CC
:10BA30000081EB005E03070072618000836180007B
:10BA40008B04070070618800816188009A6304009C
:10BA50000000000092618000A361800000002000CF
:10BA600001F823007D0407000000E000020035001B
:10BA70000000200001003700100020000000E0005E
:10BA8000060032006000470010017800600051009D
:10BA900002003D00765D040000000000926180001D
:10BAA000A361800000002C009147240028040700B7
:10BAB0000000E00002003C00000020000100370010
:10BAC000100020000000E000060032006000470087
:10BAD000100178006000510002003400765D04001F
:10BAE00000000000885D0400000000001E007800D7
:10BAF000CF80DE000081EB002D0307009261800003
:10BB0000A36180005A04070090618800A161880049
:10BB10009A63040000000000B2618000C3618000ED
:10BB20000000200001F823004C0407000000E000A2
:10BB30000200350000002000010037001000200046
:10BB40000000E000060032006000470010017800AD
:10BB50006000510002003D00D85D040000000000BC
:10BB6000B2618000C361800000002C009147240076
:10BB7000F70307000000E00002003C000000200086
:10BB800001003700100020000000E0000600320035
:10BB9000600047001001780060005100020034008E
:10BBA000D85D040000000000EA5D04000000000011
:10BBB0001E007800CF80DE000081EB00FC02070051
:10BBC000B2618000C361800029040700B061880071
:10BBD000C16188009A63040000000000D261800007
:10BBE000E36180000000200001F823001B0407002F
:10BBF0000000E000020035000000200001003700D6
:10BC0000100020000000E000060032006000470045
:10BC1000100178006000510002003D003A5E04000F
:10BC200000000000D2618000E361800000002C0071
:10BC300091472400C60307000000E00002003C001A
:10BC40000000200001003700100020000000E0008C
:10BC500006003200600047001001780060005100CB
:10BC6000020034003A5E0400000000004C5E040054
:10BC7000000000001E007800CF80DE000081EB0095
:10BC8000CB020700D2618000E3618000F803070067
:10BC9000D0618800E16188009A6304000000000020
:10BCA000F2618000036280000000200001F82300A0
:10BCB000EA0307000000E000020035000000200059
:10BCC00001003700100020000000E00006003200F4
:10BCD00060004700100178006000510002003D0044
:10BCE0009C5E040000000000F2618000036280009E
:10BCF00000002C0091472400950307000000E0009D
:10BD000002003C000000200001003700100020006D
:10BD10000000E000060032006000470010017800DB
:10BD200060005100020034009C5E0400000000002E
:10BD3000AE5E0400000000001E007800CF80DE0030
:10BD40000081EB009A020700F2618000036280002C
:10BD5000C7030700F0618800016288009A6304004D
:10BD6000000000003262800043628000000020007A
:10BD700001F82300B90307000000E00002003500CD
:10BD80000000200001003700100020000000E0004B
:10BD9000060032006000470010017800600051008A
:10BDA00002003D00FE5E04000000000032628000E0
:10BDB0004362800000002000612C2400640307001F
:10BDC0000000E00002003C000000200001003700FD
:10BDD000100020000000E000060032006000470074
:10BDE000100178006000510002003400FE5E040083
:10BDF00000000000105F0400000000001E0078003A
:10BE0000CF80DE000081EB00690207003262800013
:10BE10004362800096030700306288004162880018
:10BE20009A63040000000000126280002362800018
:10BE30000000200001F82300880307000000E00054
:10BE40000200350000002000010037001000200033
:10BE50000000E0000600320060004700100178009A
:10BE60006000510002003D00605F0400000000001F
:10BE70001262800023628000000020003133240021
:10BE8000330307000000E00002003C000000200037
:10BE900001003700100020000000E0000600320022
:10BEA000600047001001780060005100020034007B
:10BEB000605F040000000000725F040000000000EA
:10BEC0001E007800CF80DE000081EB003802070002
:10BED0001262800023628000650307001062880000
:10BEE000216288009A630400000000005262800012
:10BEF0006362800000002000011224005703070045
:10BF00000000E000020035000000200001003700C2
:10BF1000100020000000E000060032006000470032
:10BF2000100178006000510002003D00C25F040073
:10BF300000000000526280006362800000C02300A5
:10BF4000C1612400020307000000E00002003C0081
:10BF50000000200001003700100020000000E00079
:10BF600006003200600047001001780060005100B8
:10BF700002003400C25F040000000000D85F04002B
:10BF800000000000A2002000600047001090B900EF
:10BF9000CF80DE000081EB000502070052628000C6
:10BFA000636280003203070050628800616288008B
:10BFB0009A6304000000000072628000600051007B
:10BFC0000600340060004700100178006000510056
:10BFD00002003D0004600400000000007262800066
:10BFE0006000510006003D0060004700100178002D
:10BFF00060005100020034000460040000000000F2
:10C000000A60040000000000600047001000780093
:10C01000706288009A630400000000008262800061
:10C0200060005100060034006000470010017800F5
:10C030006000510002003D00366004000000000076
:10C04000826280006000510006003D0060004700F1
:10C0500010017800600051000200340036600400D6
:10C06000000000003C600400000000006000470089
:10C0700010007800806288009A63040000000000CD
:10C0800092628000600051000600340060004700AA
:10C09000100178006000510002003D00686004005B
:10C0A00000000000926280006000510006003C0029
:10C0B0006000470010017800600051000200340069
:10C0C00068600400000000007060040000000000D0
:10C0D000600047001001780020C5200010084100D2
:10C0E0009A63040000000000A2628000600051001A
:10C0F0000600340060004700100178006000510025
:10C1000002003D009E60040000000000A462800068
:10C11000823E20000200520006003D006000470001
:10C120001001780060005100020034009E6004009D
:10C1300000000000A660040000000000600047004E
:10C140001001780040C52000100841009A630400E7
:10C1500000000000B2628000600051000600340060
:10C1600060004700100178006000510002003D00AF
:10C17000D260040000000000B26280006000510044
:10C1800006003C006000470010017800600051008C
:10C1900002003400D260040000000000DE600400F1
:10C1A00000000000600047001001780060C520001A
:10C1B0001008410076ED07004AF007009A6304007A
:10C1C00000000000C26280006000510006003400E0
:10C1D00060004700100178006000510002003D003F
:10C1E0000C61040000000000C4628000C212200044
:10C1F0000200520006003D00600047001001780078
:10C2000060005100020034000C61040000000000D6
:10C210001461040000000000600047001001780075
:10C2200080C52000100841009A630400000000004F
:10C2300060004700100178006000510006003400E3
:10C2400000002000C06F880010002000801F7800D0
:10C25000B9F007002F00B1009A630400000000004D
:10C26000D2628000E3628000C05A2C007172230009
:10C270007A0207000000E000020035000000200004
:10C2800001003700100020000000E000060032002E
:10C2900060004700100178006000510002003D007E
:10C2A0007C61040000000000D2628000E362800034
:10C2B0000000200001F82300250207000000E00034
:10C2C00002003C00000020000100370010002000A8
:10C2D0000000E00006003200600047001001780016
:10C2E00060005100020034007C6104000000000086
:10C2F00094610400000000001E007800CF80DE0082
:10C300000081EB002A010700C25A2C00737223003F
:10C3100082010700D2628000E362800054020700BD
:10C32000D0628800E16288009A6304000000000087
:10C33000F262800003638000F026210031A8230010
:10C34000460207000000E000020035000000200067
:10C3500001003700100020000000E000060032005D
:10C3600060004700100178006000510002003D00AD
:10C37000E461040000000000F262800003638000BA
:10C380000000200001F82300F10107000000E00098
:10C3900002003C00000020000100370010002000D7
:10C3A0000000E00006003200600047001001780045
:10C3B0006000510002003400E4610400000000004D
:10C3C000FC610400000000001E007800CF80DE0049
:10C3D0000081EB00F6000700F226210033A82300BD
:10C3E0004E010700F2628000036380002002070014
:10C3F000F0628800016388009A6304000000000076
:10C4000012638000600051000600340060004700A5
:10C41000100178006000510002003D002A62040013
:10C42000000000008402200022C62000120012003A
:10C4300006003D00600047001001780060005100D8
:10C44000020034002A62040000000000346204008C
:10C4500000000000126380006000470010004100EF
:10C4600010638800507088009A6304000000000088
:10C4700060004700100078006100500002003200A8
:10C4800000002000010037001000200040638800F9
:10C490009A6304000000000060004700100078006C
:10C4A000610050000200320000002000010037004F
:10C4B0001000200020638800801F780046F00700ED
:10C4C0002F00B1009A6304000000000060004700E4
:10C4D00010007800610050000200320000002000CF
:10C4E0000100370010002000306388009A630400C8
:10C4F000000000006000470010017800600051005B
:10C500001E00340000C02F00F10720003007980003
:10C510004107980000002000200798000402200036
:10C52000640147001200120011003D006400470042
:10C53000100078004201DD0080F12000020140007F
:10C5400062004100901F7800921F7800660047004B
:10C55000801F780078F007006F00B1001200200003
:10C5600064004700100841008E62040000000000D3
:10C5700000002000C07288005AEF07009A63040090
:10C58000000000009A63040000000000B272800006
:10C5900060005100B6FA3200B272800061005100B2
:10C5A000E4FA3200B27280006200510015FB3200E2
:10C5B000B27280006300510046FB3200B27280000C
:10C5C000640051005EFB3200B272800065005100D1
:10C5D0008CFB3200B272800066005100BDFB32005D
:10C5E000B272800067005100EBFB3200B272800033
:10C5F000680051001CFC3200B272800069005100DA
:10C600004DFC3200B27280006A0051007BFC3200A7
:10C61000B27280006B005100A9FC3200B27280003F
:10C620006C005100DAFC3200B27280006D005100E3
:10C6300008FD3200B27280006E00510036FD3200FB
:10C64000B27280006F00510064FD3200B27280004F
:10C650007000510092FD3200B272800071005100F2
:10C66000C0FD3200B272800072005100EEFD320057
:10C67000B2728000730051001CFE3200B272800062
:10C68000740051004CFE3200B272800075005100FF
:10C6900062FE3200B27280007600510078FE3200F5
:10C6A000B2728000770051008FFE3200B2728000BB
:10C6B00078005100A7FE3200B2728000790051006C
:10C6C000C0FE3200B27280007A005100D8FE320003
:10C6D000B27280007B005100E1FE3200B272800035
:10C6E0007C00510012FF3200B27280007D005100C8
:10C6F00043FF3200B27280007E0051005CFF3200C6
:10C70000B27280007F00510063FF320004022000FB
:10C7100062E52000120012006CFF320014022000BB
:10C7200062E520001200120072FF3200C2620400B3
:10C7300000000000560EF80044EC07002F00B10086
:10C74000620047001002780062E5200012005200EB
:10C750000700320062004700901F78003BEC0700A2
:10C760002F00B100560EF80038EC07002F00B10082
:10C77000D8F907000080FA00000006000000FA0067
:10C780004EB89700BEB897000000E00004003200E9
:10C79000FA3F0900000000000000E900FAFF37003E
:10C7A00001800900000000000080FA00000006007F
:10C7B0000000FA00020007008A6404000000000084
:10C7C0000200E00006003A000005EB000100E00076
:10C7D0000F003E000000E000270032000C00370090
:10C7E000010578000100E0000400350008003C006D
:10C7F0000000E0002000320005003700600010005B
:10C80000E080180002003B0001F02C001A00370005
:10C810000004BE006011B8006B0920000982CF003F
:10C82000020039000882CF000441B0006942520082
:10C830000E00320008003B0082817100610164003B
:10C840008904D1000884D3008B05E8000442E80085
:10C85000F9FF3A00050037000804440089844C00C1
:10C860008B05E9000442E900FBFF3A0003000700E2
:10C870000AF0A70001F0A0000000060081002000DF
:10C88000618055000B003D000B00200061FE2F0071
:10C890000100E1001D00340082817100610164002B
:10C8A0008904D1000884D3000000E800FAFF3A00B0
:10C8B000710020006100640003007000020060004D
:10C8C0000900320061044400E0844C000988A5009E
:10C8D000050032008B05E8006808E10002003A001C
:10C8E0008904D1000884D300F20F20000258E1002F
:10C8F00005003D00C75DDD00F907B20089807500C5
:10C9000008007800000006000BF827008B00780074
:10C91000000005000080FA00000006000000FA0098
:10C9200002000700A465040000000000889FBE000C
:10C930008A9FBE008C1F780030000700370033004C
:10C9400003866C006450E100240032006420E100A2
:10C95000270032006150E100220032006120E10036
:10C96000210032008B854200EB07B1000134B80092
:10C97000003AB8000804420089844A00013AB8002D
:10C980000030B8008880400009014A0004003300EC
:10C990000000400081804800020149008B05E90049
:10C9A000C909DD008301700001003200130020007E
:10C9B000C814DE004814DD004709DE001200B20092
:10C9C000C808DE00088470002400070001F0A10000
:10C9D0000CF0A70001F0A000190037006120E10071
:10C9E0001B0032000801BE000200BE00F7FF370046
:10C9F0006150E100FCFF3A00150037000004BE0062
:10CA00003C0007000003BE000405BE000200BE009B
:10CA100038000700844F7500000006000200BE00C9
:10CA20006450E100050036006420E1000200360099
:10CA30000968A30001003A000800BE000160A000E0
:10CA40004F0678004F05BE004F04BE0000000600F0
:10CA5000F0FF2F00F1FF2700F9FF370081002000D1
:10CA6000618055000B003D000B00200061FE2F008F
:10CA70000100E1001D003400828171006101640049
:10CA80008904D1000884D3000000E800FAFF3A00CE
:10CA9000710020006100640003007000020060006B
:10CAA0000900320061044400E0844C000988A500BC
:10CAB000050032008B05E8006808E10002003A003A
:10CAC0008904D1000884D300F20F20000258E1004D
:10CAD00005003D00C75DDD00F907B20089807500E3
:10CAE00008007800000006000BF827008B00780093
:10CAF00000000500C70ADE00F107B200F50FB20022
:10CB000008003200E1CF4200020032000170A000B4
:10CB100024000500810F70000100320004080500A8
:10CB200044000500810F700002003A001400050067
:10CB30008502E9000000400081C04800FCFF3B0086
:10CB40000170A000240005000080FA00000006002B
:10CB50000000FA00F4FF2F00070007000080FA0031
:10CB6000000006000000FA0003F0A20040000700E9
:10CB70000080FA00000006000000FA000200070032
:10CB80002A66040000000000841F780014000700DB
:10CB90004F00780011003300F0FF2F00838F6C00EE
:10CBA00006003B00040565000A00A70008003700E6
:10CBB00009F0A6001000200008003700820F540082
:10CBC000838F5C00030039001000200001003E004C
:10CBD0000000200009F0A7000000EA0000000600A5
:10CBE0000004BE00060007000003BE000405BE00EE
:10CBF0000200BE0002000700844F7500000006001E
:10CC0000C70ADE00F107B200F50FB20008003200DB
:10CC1000E1CF4200020032000170A00024000500B4
:10CC2000810F700001003200040805004400050077
:10CC3000810F700002003A00140005008502E9002F
:10CC40000000400081C04800FCFF3B000170A000D4
:10CC5000240005000080FA00000006000000FA0031
:10CC600014002000C4FF07000080FA000000060046
:10CC70000000FA0002000700A067040000000000A6
:10CC8000889FBE008A9FBE008C1F78005900070055
:10CC9000600033006450E1004F0032006420E10086
:10CCA0005200320003826C0007003B000905D000EF
:10CCB0000306D000820F54000C065D00020039000C
:10CCC0000200320089017800030678008582550051
:10CCD00004003D000003FD008103FD008502EA0021
:10CCE0008B854200840F720002003B006000100040
:10CCF000E08018006011B8000005EB007A28E10020
:10CD00000A00390006007800C75DDD00F707B200B1
:10CD1000878075002D003700828171000A0178003C
:10CD2000610560008180D1000080D3008502E900A8
:10CD3000F9FF3B00060440008784480002003B00E6
:10CD400060041400E0841C000988A300070032007E
:10CD50008A81710082817100610164008904D100BF
:10CD60000884D3008B05E800170037000978A3007A
:10CD700013003A000B00E000130034008B05E900BB
:10CD80000804440089844C000A4474000978A30014
:10CD90000D003A000B00E000070034008B05E900AD
:10CDA0000804440089844C0001003A000B00200074
:10CDB0000978A300F7FF32000001EB000200370002
:10CDC000828171000A017800220007000CF0A700A0
:10CDD00001F0A000180037006420E10002003A00D2
:10CDE000838F6C00180033000801BE000200BE00F3
:10CDF000110037000004BE003C0007000003BE0025
:10CE00000405BE000200BE0038000700844F750014
:10CE1000000006000200BE006450E100050036007C
:10CE20006420E100020036000968A30001003A0016
:10CE30000800BE000160A0004F0678004F05BE004C
:10CE40004F04BE0000000600F0FF2F00F1FF270096
:10CE5000F9FF370081002000618055000B003D0084
:10CE60000B00200061FE2F000100E1001D003400D6
:10CE700082817100610164008904D1000884D300BB
:10CE80000000E800FAFF3A00710020006100640031
:10CE900003007000020060000900320061044400D9
:10CEA000E0844C000988A500050032008B05E800ED
:10CEB0006808E10002003A008904D1000884D30028
:10CEC000F20F20000258E10005003D00C75DDD00C3
:10CED000F907B2008980750008007800000006009C
:10CEE0000BF827008B00780000000500C70ADE0061
:10CEF000F107B200F50FB20008003200E1CF4200A6
:10CF0000020032000170A00024000500810F7000B3
:10CF1000010032000408050044000500810F700084
:10CF200002003A00140005008502E90000004000FC
:10CF300081C04800FCFF3B000170A00024000500F8
:10CF40000080FA00000006000000FA00020007005E
:10CF5000D668040000000000889FBE008A9FBE00C3
:10CF60008C1F78003E0007004500330003866C00EC
:10CF70006450E1002E0032006420E10033003200F2
:10CF80006150E1002F0032006120E10031003200E9
:10CF900085855500EB07B00009002000080420003B
:10CFA000050037000804440089844C000A00310061
:10CFB0000603430087834B000001530081815B001F
:10CFC000F8FF33000203BE000800A000080444007C
:10CFD00089844C00F6FF3900C639DD0083017300F7
:10CFE00001003200130020008904D1000884D3001E
:10CFF0000998A300050032000800A7000300A00064
:10D000008904D1000884D3008B05E8008904D1008D
:10D010000884D3000001EB000281D2002800070041
:10D0200001F0A1000CF0A70001F0A0001D003700E6
:10D030006420E1001F0032000801BE000200BE00B3
:10D04000F7FF37006120E1001A0032006000B800ED
:10D05000F3FF37000000200001F82700F0FF370041
:10D060000004BE003C0007000003BE000405BE0033
:10D070000200BE0038000700844F75000000060063
:10D080000200BE006450E100050036006420E100AB
:10D09000020036000968A30001003A000800BE0043
:10D0A0000160A0004F0678004F05BE004F04BE008F
:10D0B00000000600F0FF2F00F1FF2700F9FF370006
:10D0C00081002000618055000B003D000B00200016
:10D0D00061FE2F000100E1001D003400828171001B
:10D0E000610164008904D1000884D3000000E800D5
:10D0F000FAFF3A0071002000610064000300700034
:10D10000020060000900320061044400E0844C0029
:10D110000988A500050032008B05E8006808E100D9
:10D1200002003A008904D1000884D300F20F2000E5
:10D130000258E10005003D00C75DDD00F907B200BF
:10D140008980750008007800000006000BF82700B1
:10D150008B00780000000500C70ADE00F107B2006E
:10D16000F50FB20008003200E1CF420002003200A9
:10D170000170A00024000500810F70000100320042
:10D180000408050044000500810F700002003A0009
:10D19000140005008502E9000000400081C048003D
:10D1A000FCFF3B000170A000240005000080FA0095
:10D1B000000006000000FA00020AB80080027800B1
:10D1C0000200B80081004200032AB800810042003A
:10D1D0000080FA00000006000F802000E0BF200061
:10D1E000000188004440A80000002000A001880041
:10D1F00080EC2000E1DC2F00D700090031587800D6
:10D20000B400FA006000470021D42F000E0009008E
:10D21000315878006F00470011D52F003100090008
:10D2200031587800100420000000470031D82F004A
:10D230001F00090031587800100620000000470048
:10D2400031DA2F001800090031587800A0072000BB
:10D2500000004700C1DB2F000300090031587800AF
:10D26000E00720000000470001DC2F000500090056
:10D2700031587800400820000000470061DC2F0092
:10D2800007000900315878000000200060879800EE
:10D2900000002000108F980000772000400E8800CA
:10D2A00000002000C0168800E4FF2F00A02D200001
:10D2B00010086200E0E02000801F780010002000CD
:10D2C000801F78002DFD07004F00B10014002000E2
:10D2D000A02D200010087200002C21000100200069
:10D2E000801F7800811F780061CD07004F00B100DA
:10D2F00004402000C02020001008720000102E0002
:10D3000001002000801F7800811F7800F1CD070008
:10D310004F00B100040028006021200010087200B6
:10D3200080F920005063880060EA2000CF80DE0092
:10D33000406888005168880060EA200001002000F1
:10D34000206888003168880060EA20000100200021
:10D35000C0678800D167880060EA200001002000D3
:10D36000006888001168880000002000100E880006
:10D37000701A2600200E880080002800000E880009
:10D3800060EA2000D00E8800D00E8000C00E880019
:10D39000C00E8000B00E880000002000A06788004A
:10D3A000000020009067880000002000B06788001F
:10D3B00022CE070038CE070000002000CF80DE001C
:10D3C000A0688800B1688800003A800070006000A2
:10D3D0004402DE000400E00032003A0000002000B9
:10D3E00001002000106F8800216F880000002000DD
:10D3F00001002000D06E8800E16E8800000020004F
:10D4000001002000F06E8800016F880000002000FD
:10D41000B06F880000002000A06F8800000020008E
:10D42000906F8800000020000100200070728800CA
:10D4300081728800000020000100200050728800E6
:10D440006172880000002000010020003072880016
:10D450004172880000002000010020001072880046
:10D460002172880000002000CF80DE001069880053
:10D470002169880000002000C06F8800A0C52F002F
:10D48000F107200040979800519798000000200075
:10D49000CF80DE0060979800719798000000200010
:10D4A000008F98000000200080708800000020009D
:10D4B0007070880000002000C0708800000020000C
:10D4C0009070880000002000CF80DE000081EB001B
:10D4D000B7FC0700507188006171880000002000CF
:10D4E000CF80DE0070738800817388000000200008
:10D4F0000100200050738800617388000000200044
:10D500000100200030738800417388000000200073
:10D5100001002000107388002173880000002000A3
:10D5200001002000F07188000172880000002000D6
:10D5300001002000E06A8800F16A880000002000F5
:10D5400001002000A0708800B17088000000200059
:10D5500001002000D0708800E170880000002000E9
:10D5600001002000006B8800116B88000000200083
:10D570000100200010708800217088000000200049
:10D5800001002000906A8800A16A88000000200045
:10D5900001002000706A8800816A88000000200075
:10D5A00001002000206A8800316A88000000200005
:10D5B00001002000506A8800616A88000000200095
:10D5C00001002000009798001197980000002000AB
:10D5D00001002000608F9800718F980000002000EB
:10D5E00001002000F06F880001708800000020001A
:10D5F0000100200030708800417088000000200089
:10D6000001002000D06F8800E16F8800000020003A
:10D61000006A880000002000106A880000002000D6
:10D6200001002000408F9800518F980000002000DA
:10D6300001002000E0698800F169880000002000F6
:10D6400090688800000020008068880000002000AA
:10D6500070688800000020006068880084D4200082
:10D6600000022000004A780094D42000000220002C
:10D67000004A780074D2200000022000004A78009E
:10D6800000002000C072880000002000308F980049
:10D6900000002000208F98000000200060708800AB
:10D6A00000002000D06A880000002000206B880065
:10D6B00000002000A0728800000020009072880006
:10D6C00000002000E068880000002000B0728800A0
:10D6D00000002000E06788000000200060879800BC
:10D6E000C008200000004700100278006C005200C3
:10D6F00016003D00C608200006034700160078000B
:10D700004202DD0060D6200004024000000020003C
:10D71000000A780006007800100078004202DD0060
:10D7200060D620000400400062024000000020009B
:10D73000000A780014002000C00820000000470004
:10D7400010084200706B0400000000000000200080
:10D750000071880000002000F070880000002000A8
:10D760004071880000002000207188000000200027
:10D770003071880000002000107188000000200037
:10D780007063880000002000806388001000200083
:10D79000906E880010002000F067880064D220009E
:10D7A00040002000004A780000102000801F780010
:10D7B00000002000801F780000002000801F7800FB
:10D7C00000002000801F780000002000801F7800EB
:10D7D00020002000801F780000002000801F7800BB
:10D7E00000022000801F7800D4CD07000F01B10097
:10D7F00000C02F00F1072000209798003197980073
:10D80000000020006087980006022000C408200065
:10D81000040247001400130014003D00C00820005B
:10D8200000004700100078004202DD0080F1200077
:10D830000402400062004200901F7800941F7800AC
:10D84000400A200000004700801F780006D0070033
:10D850006F00B10014002000C00820000000470045
:10D8600010084200046C04000000000010638000F7
:10D87000507088006460800060005200080035002D
:10D88000A6D72000CFB3DE0004D020003400130060
:10D8900024801B0002003500286D040000000000F9
:10D8A00000002000012424003061880041618800CC
:10D8B0000000200001222400D0608800E160880080
:10D8C0000000200001172400F0608800016188003A
:10D8D000000020000112240090608800A1608800F0
:10D8E00000002000011024001061880021618800E0
:10D8F0000000200001102400B0608800C160880092
:10D9000000002000010A2400506188006161880045
:10D91000000020004123240010628800216288005A
:10D92000000020000112240030628800416288005B
:10D93000B00420006060880000002600A16624007A
:10D9400070608800816088006066260061FA2300AC
:10D9500040608800516088001000200070628800DC
:10D96000100020008062880000002000812C24002C
:10D97000706188008161880000002000012224007D
:10D9800090618800A161880000002000011A240035
:10D99000B0618800C161880000002000813C240043
:10D9A000D0618800E161880000002000812424000B
:10D9B000F06188000162880000002800414D2400C9
:10D9C000506288006162880090C22500F1D823006F
:10D9D0002060880031608800000020006149240038
:10D9E00000608800116088001000200090628800AC
:10D9F00080072000A062880000002000B06288003C
:10DA000050002000C062880060BA290041A42300B1
:10DA1000D0628800E1628800207C210061DA230066
:10DA2000F062880001638800F000200050708800D8
:10DA3000F0002000106388000000200020638800B0
:10DA40000000200030638800000020004063880050
:10DA500000002000010E2400707188008171880090
:10DA600000002000010E2400B0718800C171880000
:10DA700060688000CF80DE000081EB004CFB070077
:10DA8000B2FA2C0053CD2300A4FB0700009F98009E
:10DA9000119F980050718800617188007068800043
:10DAA000CF80DE000081EB0041FB070012362C0026
:10DAB00033CD230099FB070090718800A171880085
:10DAC0000E9890009E9890000002780081027800E5
:10DAD00000002000811024000401780085017800F6
:10DAE0001BFC07000000E00002003C0000002000DA
:10DAF00001003700100020000000E00006003200A6
:10DB000000002000010E24007071880081718800DF
:10DB1000946D0400000000000000200001122400A9
:10DB2000707188008171880094718000A5718000F7
:10DB30000000200081102400040178008501780095
:10DB400003FC07000000E00002003C000000200091
:10DB500001003700100020000000E0000600320045
:10DB600000002000010E2400B0718800C1718800FF
:10DB7000EC6D04000000000094718000A57180002D
:10DB8000D0CC2C00C1142400040178008501780059
:10DB9000EFFB07000000E00002003C000000200056
:10DBA00001003700100020000000E00006003200F5
:10DBB0000000200001122400B0718800C1718800AB
:10DBC000EC6D04000000000000002000011524009E
:10DBD000B0718800C1718800406080005160800091
:10DBE000A06E8800B16E880060608000C06E880002
:10DBF0006460800080DD200061084200E06A20004F
:10DC0000801F7800700B2000801F7800DBFA07006F
:10DC10004F00B100DEE60700560CF80060D22F007E
:10DC2000801F780092F407004F00B10060004700A9
:10DC3000801F780073F407002F00B100E046200039
:10DC4000801F7800A0072000801F7800CBFA070013
:10DC50004F00B1009FF407006F004700801F78005D
:10DC600068F407002F00B1001004200000004700F6
:10DC7000801F780063F407002F00B100E01E210030
:10DC8000801F7800801E2000801F7800BBFA0700EC
:10DC90004F00B1002000200060879800C0082000DD
:10DCA00000004700100278006000520018003400A5
:10DCB000C0082000000047001000780061005000FC
:10DCC00060879800801F7800F0D22F00801F7800B6
:10DCD00060D92000801F780094E907006F00B10030
:10DCE00060D92000801F780013D207002F00B100F8
:10DCF000E0CE2200801F7800404C2000801F78007A
:10DD00009EFA07004F00B1004E6E040000000000B4
:10DD10009FE6070004402000E02020001008720069
:10DD200004002800C0202000100872001008200005
:10DD3000801F7800A1CC07002F00B1005001200007
:10DD4000801F78009DCC07002F00B100000220004A
:10DD5000801F780099CC07002F00B100F4DF2F005E
:10DD60004008200010086200D4FF2F00E0202000AF
:10DD7000100862001006200000004700801F780095
:10DD8000EDD107002F00B100A6CC070060025000C3
:10DD900002003500C46E040000000000B9CC07008A
:10DDA0000004E00003003A000060FE00CE6E0400B4
:10DDB00000000000E08E2000801F7800400F20004F
:10DDC000801F78006DFA07004F00B10070E6070071
:10DDD00040F40700A007200000004700801F7800E3
:10DDE0008CE907002F00B100E0462000801F78007A
:10DDF000A0072000801F780060FA07004F00B100E4
:10DE0000003A8000700060004402DE000400E00080
:10DE10000600320000002000801F7800C6E90700DD
:10DE20002F00B1001E6F0400000000001000200051
:10DE3000801F7800C0E907002F00B100000020001B
:10DE4000003A8800E0462000801F7800A0072000EC
:10DE5000801F780049FA07004F00B100E00720005A
:10DE600000004700801F78006AE907002F00B1001A
:10DE70004008200000004700801F780065E9070087
:10DE80002F00B100000020006087980000002000F3
:10DE9000108F9800640CF800CFE907002F00B10044
:10DEA00078CC07000004E000C50132000060FE00ED
:10DEB0005CCC07007087980060025000BE013500FE
:10DEC00046052000C4082000040247001400130087
:10DED0000600340000002000608798000000200049
:10DEE000108F9800DC72040000000000BA72040079
:10DEF0000000000000002000608798001000200053
:10DF0000108F9800DC7204000000000020E7200061
:10DF1000C60820000603470016024000000020004B
:10DF2000004A780010002000160B4000DC7204004C
:10DF30000000000024E72000C00820000000470087
:10DF40001002420000002000004A78002009200052
:10DF50000000470010027800600052007201320099
:10DF600000002000108F980020E72000801F78001C
:10DF70006BCE07002F00B100600250006A01340030
:10DF8000046B8000156B8000126F8000236F80008F
:10DF90000400780085007800F2FA0700107088000D
:10DFA00021708800800920000000470030027800BE
:10DFB000A0027800E0698000F16980000401780027
:10DFC0008501780025FB07000000E00002003A0010
:10DFD0000000200001003700100020000000E000D9
:10DFE0008E003200800920000000470030027800D7
:10DFF000A0027800E0698000F169800004017800E7
:10E000008501780015FB07000000E00002003500E4
:10E010000000200001003700100020000000E00098
:10E020000B00320080092000000047003002780019
:10E03000A0027800020020000327240004007800DA
:10E0400085007800C7FA0700408F9800518F98002C
:10E050001400200040092000000047001008420082
:10E060001400200060092000000047001008420052
:10E070001670800027708000C40920000402470049
:10E0800034017800A4017800060078008700780049
:10E09000B4FA0700A0708800B1708800966A80000A
:10E0A000A76A8000040A20000402470034017800B7
:10E0B000A40178000600780087007800A9FA07001C
:10E0C000D0708800E170880000027800810278003A
:10E0D000000020004133240004017800850178000D
:10E0E000DEFA07000000E00002003500000020001A
:10E0F00001003700100020000000E0000B0032009B
:10E10000D4708000E570800002002000433B2400B2
:10E11000040078008500780092FA0700D07088002B
:10E12000E1708800C470040000000000D47080001A
:10E13000E57080000000200041332C0004017800CD
:10E140008501780082FA07000000E00002003C0030
:10E150000000200001003700100020000000E00057
:10E1600009003200D4708000E570800000002000BB
:10E17000413B24000401780085017800BCFA0700C7
:10E18000D0708800E1708800E6698000F76980003F
:10E19000840920000402470034017800A4017800BB
:10E1A00006007800870078006EFA0700009F98004C
:10E1B000119F98000001780081017800D0708000E4
:10E1C000E170800060FB0700D0708800E17088007B
:10E1D0000E9990009E999000A0708000B170800010
:10E1E00059FB0700A0708800B1708800E0698000CA
:10E1F000F1698000408F9800518F98001070800066
:10E2000021708000608F9800718F9800906A800064
:10E21000A16A80000097980011979800C46F800051
:10E220006000520003003A00DAD007009472040044
:10E230000000000000002000801F780064D5070067
:10E240002F00B100D46A8000630052003600340011
:10E25000746A8000856A80001072800021728000DC
:10E2600004017800850178007CFA07000000E000D6
:10E2700002003500000020000100370010002000DF
:10E280000000E00004003200706A8000816A8000B3
:10E290001072880021728800F46F80000570800081
:10E2A000507280006172800004017800850178005E
:10E2B0006AFA07000000E0000200350000002000BC
:10E2C00001003700100020000000E00004003200D0
:10E2D000F06F8000017080005072880061728800C9
:10E2E00014708000257080003072800041728000C0
:10E2F000040178008501780058FA07000000E0006A
:10E30000020035000000200001003700100020004E
:10E310000000E000040032001070800021708000D6
:10E320003072880041728800F467800060005200FB
:10E330000C003A00E46780006000520009003A00D7
:10E340004009200000004700901F780010002000C6
:10E35000801F780063D607004F00B100C071040031
:10E36000000000004009200000004700901F7800D6
:10E3700000002000801F78005AD607004F00B1002F
:10E3800000002000208F9800C462800060005200CE
:10E390006500340060092000000047001003780089
:10E3A00084C52000140053005F00350000002000E9
:10E3B000308F9800746A8000856A80000000200019
:10E3C00001F02300040178008501780023FA07009A
:10E3D0000000E000020034000000200001003700CF
:10E3E000100020000000E00007003A0000092000B3
:10E3F0000000470010027800600052000200320066
:10E400009472040000000000800A20000000470011
:10E4100030037800A003780044FF2F00F5072000A8
:10E420000400530005805B003F003E0000242400F0
:10E43000F1002000026A8000CF91DE005DFB070042
:10E4400066D5200036024000A6824800049F98004E
:10E45000159F980000102E00515F2000126A800066
:10E46000CF91DE0053FB07000E9A90009E9A900019
:10E470000002420081824A00C00A200000004700DA
:10E480001018420010904A000009200000004700C8
:10E49000100278006000520018003A0020002000AE
:10E4A000CF80DE00840A200004024700141A100006
:10E4B0001492180010002000801F7800000920002E
:10E4C00000004700801F7800841F78009AE807004A
:10E4D0006F00B10020002000801F7800C00A2000DB
:10E4E00000004700801F7800800A200000004700DD
:10E4F000801F780090E807006F00B100000920003D
:10E50000000047001000780061004000008F980074
:10E51000801F7800800A200000004700801F7800DC
:10E52000B3D707004F00B100DC7204000000000008
:10E53000200920000000470010027800600052000F
:10E540000A00320020E72000C6082000060347002A
:10E5500016024000E008200000004700104078004C
:10E56000004A780010002000160B4000DC72040006
:10E570000000000046022000E408200004024700DA
:10E58000140013005BFE3200E0082000000047008A
:10E59000100278006D0052005CFE3200E00820009E
:10E5A00000004700100278006A00520061FE32004D
:10E5B0009872040000000000506F0400000000008A
:10E5C00060D220001042780061405200AA00390059
:10E5D000EFF107000608200006025000A6003900EF
:10E5E00064D2200000002000004A780060688000AB
:10E5F000CF80DE000081EB006DF80700B2FA2C003E
:10E6000053CD2300C5F80700547180006571800068
:10E61000040178008501780095F9070002002000C8
:10E620000300240048FA07005071880061718800D7
:10E6300070688000CF80DE000081EB005CF807008E
:10E6400012362C0033CD2300B4F8070094718000FB
:10E65000A5718000040178008501780084F9070025
:10E66000020020000300240037FA070090718800A0
:10E67000A1718800F0688000CF80DE000081EB008F
:10E680004BF80700F262800003638000A3F80700E4
:10E69000D0718800E1718800000278008102780062
:10E6A000707280008172800004017800850178001A
:10E6B0006AF907000000E0000200350000002000B9
:10E6C00001003700100020000000E00004003200CC
:10E6D000D0718000E17180007072880081728800C2
:10E6E00010698000216980000001EB0030F807000C
:10E6F000D2628000E362800088F80700F071880031
:10E700000172880006AF2000CFB3DE0044D02000A5
:10E710003400130024801B0014003D00C06F8000F3
:10E720000000E00011003200E46780006100520048
:10E7300007003A0000002000E06788001000200079
:10E74000206B880012E40700B27304000000000090
:10E7500000002000F067880010002000906E880004
:10E7600011DC07003A7404000000000010002000D3
:10E77000F0678800C63E2100CFB3DE0044D0200001
:10E780003400130024801B000400340060EA2000E1
:10E79000CF80DE002068880031688800C62521000F
:10E7A000CFB3DE0044D020003400130024801B00CF
:10E7B00008003400946E80006100520003003A00AB
:10E7C000F3E3070000002000906E88003A74040014
:10E7D0000000000046192100CFB3DE0044D0200025
:10E7E0003400130024801B0017003400946E800056
:10E7F0006100520003003A00E5E30700000020003A
:10E80000906E8800E4678000600052000B003A00C0
:10E8100010002000E0678800006880001168800018
:10E82000D0728800E1728800C0678000D1678000E4
:10E83000F072880001738800AAE60700AAF10700B9
:10E840003A74040000000000E46780006100520098
:10E8500005003A0000002000E0678800CCE30700D4
:10E860003A7404000000000010002000906E880040
:10E87000CDDB070046F10700506F040000000000E8
:10E880000080FA00FFFF37003235FF00312CFF0017
:10E890003338FF003430FF003000FF000000FF007D
:10E8A0000000FF000000FF000000FF000000FF006C
:10E8B0000000FF000000FF000000FF000000FF005C
:10E8C0000000FF003C0AFF002530FF003130FF0050
:10E8D0006C75FF000A00FF002538FF002E36FF0090
:10E8E000662CFF002538FF002E36FF00662CFF0047
:10E8F0002564FF000A00FF004750FF00524DFF0053
:10E900004300FF004750FF004747FF004100FF0062
:10E910004750FF004753FF005600FF005049FF00DB
:10E920004E47FF000050FF004F4EFF00470AFF0018
:10E930000047FF004554FF004C4FFF004700FF0019
:10E940003E0AFF000053FF006574FF007469FF007A
:10E950006E67FF002048FF004F4DFF004520FF007D
:10E96000252DFF003364FF000048FF004F4DFF00DE
:10E970004520FF006E6FFF007420FF007365FF00ED
:10E980007400FF000000FF000000FF00C4FFFF0054
:10E990007F3FFF0080EFFF00FFBEFF0090E1FF0020
:10E9A000A93EFF00EC82FF0076BEFF0082ADFF00B3
:10E9B0002B3EFF000E3CFF00C3BDFF0087D1FF00D0
:10E9C000133DFF004178FF00D3BBFF000000FF00B4
:10E9D000803FFF001872FF00313FFF00F0FDFF0095
:10E9E000753EFF004758FF00633DFF005895FF004C
:10E9F0001D3CFF0082C4FF00AE3AFF00A878FF0074
:10EA00002139FF00EF93FF008037FF00A092FF0045
:10EA1000A735FF004656FF001534FF00063CFF00F7
:10EA20000442FF007D9FFF006A42FF005C90FF00F0
:10EA30000142FF00604DFF00BB40FF0051ECFF00B2
:10EA4000473EFF00DE8DFF001FBBFF00063CFF00BE
:10EA50000442FF00C059FF008B42FF007404FF0016
:10EA60004442FF00F99BFF004F41FF000000FF0000
:10EA7000803FFF001B5BFF003958FF00001BFF00B9
:10EA80005B37FF00396DFF004155FF00544FFF0019
:10EA90005049FF004C4FFF005400FF001B5BFF007C
:10EAA000307AFF001B5BFF002564FF003B25FF0061
:10EAB0006478FF000025FF002336FF002E31FF00A1
:10EAC000661BFF005B31FF007A00FF001B5BFF004D
:10EAD0002564FF003B25FF00642EFF007200FF004D
:10EAE0001B5BFF002564FF003B25FF00642DFF003A
:10EAF0007200FF001B5BFF002564FF003B25FF0049
:10EB0000642DFF007200FF001B5BFF002564FF0007
:10EB10003B25FF00642DFF007200FF001B5BFF0020
:10EB20002564FF003B25FF00642DFF007200FF00FD
:10EB30001B5BFF002564FF002F72FF00001BFF001E
:10EB40005B21FF007200FF001B5BFF002564FF00DC
:10EB50003B25FF00642EFF007200FF001B5BFF00DF
:10EB60002564FF003B25FF00642DFF007200FF00BD
:10EB70001B5BFF00302FFF007200FF001B5BFF00DC
:10EB80002564FF003B25FF00642EFF007200FF009C
:10EB90001B5BFF002564FF003B25FF00642DFF0089
:10EBA0007200FF001B5BFF002564FF002F72FF0057
:10EBB0000025FF002336FF002E31FF00661BFF00FB
:10EBC0005B31FF007A00FF001B5BFF002564FF0044
:10EBD0003B25FF00642EFF007200FF001B5BFF005F
:10EBE0002564FF003B25FF00642DFF007200FF003D
:10EBF0001B5BFF002564FF003B25FF00642DFF0029
:10EC00007200FF001B5BFF002564FF003B25FF0037
:10EC1000642DFF007200FF001B5BFF002564FF00F6
:10EC20003B25FF00642DFF007200FF001B5BFF000F
:10EC30002564FF002F72FF00001BFF005B21FF0017
:10EC40007200FF001B5BFF00347AFF001B5BFF00BC
:10EC50002564FF003B25FF006478FF0000FFFF00F4
:10EC6000ECF3FF004A48FF003595FF0095C7FF0011
:10EC700017C1FF00DC45FF00FDDBFF006DC3FF0097
:10EC800072B3FF003340FF002B34FF000148FF0048
:10EC90007F9DFF00B045FF00E7FFFF00D942FF0066
:10ECA0000000FF00803FFF001B5BFF00302FFF00D4
:10ECB0007200FF001B5BFF002564FF003B25FF0087
:10ECC000642EFF007200FF001B5BFF002564FF0045
:10ECD0003B25FF00642DFF007200FF001B5BFF005F
:10ECE0002F72FF00001BFF005B30FF007A1BFF004C
:10ECF0005B25FF00643BFF002564FF004800FF0028
:10ED00002530FF003264FF003A25FF003032FF005B
:10ED1000641BFF005B34FF007A25FF003032FF00E8
:10ED20006420FF005554FF004300FF002530FF0022
:10ED30003264FF003A25FF003032FF00641BFF0001
:10ED40005B34FF007A25FF003032FF006400FF00D3
:10ED50002523FF00362EFF003166FF001B5BFF00FE
:10ED6000317AFF006B70FF006800FF002523FF0071
:10ED7000362EFF003166FF001B5BFF00317AFF007B
:10ED80006D70FF006800FF002523FF00362EFF0096
:10ED90003166FF001B5BFF00317AFF006D00FF0052
:10EDA0002523FF00362EFF003166FF001B5BFF00AE
:10EDB000317AFF006674FF00001BFF005B30FF002C
:10EDC0007A25FF006325FF006300FF002523FF0075
:10EDD000352EFF003266FF001B5BFF00317AFF001B
:10EDE0005600FF001B5BFF00307AFF002535FF0057
:10EDF0002E30FF00661BFF005B31FF007A43FF00EF
:10EE0000001BFF005B30FF007A25FF00352EFF005E
:10EE10003066FF001B5BFF00317AFF004600FF00F9
:10EE20001B5BFF00307AFF001B5BFF003758FF00C1
:10EE30000025FF002335FF002E32FF00661BFF0078
:10EE40005B31FF007A56FF001B5BFF003639FF0085
:10EE50006D1BFF005B34FF007A20FF004558FF0068
:10EE60005400FF002523FF00352EFF003166FF0010
:10EE70001B5BFF00317AFF004100FF002535FF00DA
:10EE80002E30FF00661BFF005B31FF007A6DFF0034
:10EE90004168FF000025FF00352EFF003066FF00AF
:10EEA0001B5BFF00317AFF006D00FF002523FF0090
:10EEB000352EFF003266FF001B5BFF00317AFF003A
:10EEC0006D6CFF000025FF00352EFF003066FF004F
:10EED0001B5BFF00317AFF006674FF000025FF0016
:10EEE000352EFF003066FF001B5BFF00317AFF000C
:10EEF0006D00FF002523FF00352EFF003266FF0066
:10EF00001B5BFF00317AFF006D6CFF000025FF00E6
:10EF1000352EFF003066FF001B5BFF00317AFF00DB
:10EF20006674FF00001BFF005B34FF007A53FF0094
:10EF30005045FF004544FF00201BFF005B30FF00F1
:10EF40007A25FF002336FF002E31FF00661BFF00ED
:10EF50005B31FF007A6BFF007068FF00001BFF0051
:10EF60005B34FF007A20FF002041FF004C54FF007B
:10EF7000201BFF005B30FF007A25FF002336FF00D7
:10EF80002E31FF00661BFF005B31FF007A6DFF0032
:10EF9000001BFF005B34FF007A52FF00414EFF0070
:10EFA0004745FF00201BFF005B30FF007A25FF0074
:10EFB000362EFF003066FF001B5BFF00317AFF003A
:10EFC0006D00FF001B5BFF00347AFF005350FF0011
:10EFD0004545FF004420FF001B5BFF00307AFF0027
:10EFE0002523FF00362EFF003166FF001B5BFF006C
:10EFF000317AFF006D70FF006800FF001B5BFF00AF
:10F00000347AFF002020FF00414CFF005420FF0015
:10F010001B5BFF00307AFF002523FF00362EFF0028
:10F020003166FF001B5BFF00317AFF006674FF0052
:10F03000001BFF005B34FF007A52FF00414EFF00CF
:10F040004745FF00201BFF005B30FF007A25FF00D3
:10F050002336FF002E32FF00661BFF005B31FF00EE
:10F060007A6DFF006C00FF001B5BFF00347AFF002D
:10F070002043FF005552FF005220FF001B5BFF00A2
:10F08000307AFF002523FF00362EFF003166FF0097
:10F090001B5BFF00317AFF004100FF001B5BFF009C
:10F0A0003635FF006D25FF003264FF001B5BFF005B
:10F0B0003639FF006D1BFF005B34FF007A20FF0034
:10F0C0005341FF005453FF000025FF003264FF004E
:10F0D0001B5BFF00347AFF002053FF004154FF0008
:10F0E0005300FF002523FF003130FF002E36FF00C4
:10F0F000661BFF005B34FF007A25FF006300FF0002
:10F100002523FF003130FF002E36FF00661BFF0075
:10F110005B34FF007A25FF006300FF001B5BFF00EC
:10F12000347AFF004844FF004F50FF00201BFF00CF
:10F130005B30FF007A25FF00232DFF00362EFF00F5
:10F140003166FF000025FF003033FF006400FF0040
:10F150002025FF007320FF00001BFF005B37FF002E
:10F16000346DFF002530FF00332EFF003066FF00B6
:10F170000025FF003033FF002E30FF006600FF0047
:10F18000201BFF005B37FF00316DFF002573FF0080
:10F190001B5BFF003639FF006D20FF000020FF00E1
:10F1A0002573FF002000FF002025FF007320FF00D3
:10F1B00000C4FF002563FF001B5BFF00347AFF00E3
:10F1C000201BFF005B30FF007A00FF00C425FF001A
:10F1D000631BFF005B34FF007A20FF001B5BFF0016
:10F1E000307AFF000025FF003032FF006420FF006E
:10F1F000001BFF005B38FF005800FF001B5BFF0097
:10F200003658FF00001BFF005B37FF005800FF006F
:10F210001B5BFF003758FF00001BFF005B34FF0043
:10F220007A4CFF004F53FF00201BFF005B30FF00B4
:10F230007A00FF001B5BFF003132FF005800FF0027
:10F240001B5BFF003132FF005800FF001B5BFF001B
:10F250003132FF005800FF001B5BFF003132FF001E
:10F260005800FF001B5BFF003958FF00001BFF0028
:10F270005B35FF005800FF001B5BFF003131FF00D2
:10F280005800FF001B5BFF003131FF005800FF00FA
:10F290001B5BFF003958FF0000C0FF00A000FF000B
:10F2A000C0A0FF0000C3FF00BF00FF00C480FF003C
:10F2B00000C0FF00A000FF00C480FF0000C3FF00EB
:10F2C000BF00FF00C0A0FF00001BFF005B34FF0079
:10F2D0007A00FF002D2DFF002000FF001B5BFF00C8
:10F2E000324AFF00001BFF005B31FF007A1BFF006A
:10F2F0005B25FF00643BFF002564FF007800FF00F2
:10F30000204DFF004158FF005241FF004E47FF00D3
:10F310004520FF002020FF00201BFF005B30FF0086
:10F320007A25FF00362EFF003066FF002000FF0028
:10F33000204CFF004F57FF00414CFF005452FF008C
:10F340004154FF00494FFF00201BFF005B30FF00CE
:10F350007A25FF00362EFF003266FF002000FF00F6
:10F360002056FF00414CFF004944FF004844FF0085
:10F370004F50FF002020FF00201BFF005B30FF00EC
:10F380007A25FF00362EFF003166FF002000FF00C7
:10F39000204DFF00494EFF005641FF004C49FF0041
:10F3A0004420FF002020FF00201BFF005B30FF00F7
:10F3B0007A25FF003664FF002000FF002053FF0085
:10F3C000484FFF005748FF004F4DFF00454CFF00DE
:10F3D000494DFF00201BFF005B30FF007A25FF0036
:10F3E000362EFF003066FF002000FF002052FF0095
:10F3F0004F43FF004C49FF004D49FF005420FF00E0
:10F400002020FF00201BFF005B30FF007A25FF005B
:10F41000362EFF003166FF002000FF002052FF0063
:10F420004F43FF005354FF004550FF004741FF008A
:10F43000494EFF00201BFF005B30FF007A25FF00D4
:10F44000362EFF003066FF002000FF002041FF0045
:10F450005052FF004F43FF004741FF00494EFF005D
:10F460002020FF00201BFF005B30FF007A25FF00FB
:10F47000362EFF003166FF002000FF002052FF0003
:10F480004F54FF004C49FF004D49FF005420FF003E
:10F490002020FF00201BFF005B30FF007A25FF00CB
:10F4A000362EFF003166FF002000FF002052FF00D3
:10F4B0004F54FF005354FF004550FF004741FF00E9
:10F4C000494EFF00201BFF005B30FF007A25FF0044
:10F4D000362EFF003066FF002000FF002041FF00B5
:10F4E0005052FF004F54FF004741FF00494EFF00BC
:10F4F0002020FF00201BFF005B30FF007A25FF006B
:10F50000362EFF003166FF002000FF002053FF0071
:10F510005045FF004544FF004C4FFF00574CFF0093
:10F52000494DFF00201BFF005B30FF007A25FF00E4
:10F53000362EFF003166FF002000FF002043FF0051
:10F540005255FF004953FF004541FF004C54FF0056
:10F550002020FF00201BFF005B30FF007A25FF000A
:10F56000362EFF003066FF002000FF002043FF0022
:10F570005255FF004953FF004553FF005045FF001F
:10F580004544FF00201BFF005B30FF007A25FF0091
:10F59000362EFF003066FF002000FF00204DFF00E8
:10F5A000494EFF00414CFF005420FF002020FF0087
:10F5B0002020FF00201BFF005B30FF007A25FF00AA
:10F5C000362EFF003066FF002000FF00204DFF00B8
:10F5D0004158FF00414CFF005420FF002020FF0055
:10F5E0002020FF00201BFF005B30FF007A25FF007A
:10F5F000362EFF003066FF002000FF00204DFF0088
:10F600004158FF005350FF004545FF004420FF00D4
:10F610002020FF00201BFF005B30FF007A25FF0049
:10F62000362EFF003066FF002000FF00204DFF0057
:10F630004158FF00414CFF005443FF004847FF0082
:10F640002020FF00201BFF005B30FF007A25FF0019
:10F65000362EFF003066FF002000FF00204DFF0027
:10F660004158FF004844FF004743FF004847FF0060
:10F670002020FF00201BFF005B30FF007A25FF00E9
:10F68000362EFF003066FF002000FF00204DFF00F7
:10F690004148FF005741FF00524EFF00494EFF0016
:10F6A0004720FF00201BFF005B30FF007A25FF0092
:10F6B000362EFF003066FF002000FF002045FF00CF
:10F6C0004C45FF005345FF005256FF004F44FF00DA
:10F6D0004952FF00201BFF005B30FF007A25FF002E
:10F6E0003673FF002000FF002052FF004452FF004D
:10F6F0005345FF005256FF004F44FF004952FF00A0
:10F70000201BFF005B30FF007A25FF003673FF00EF
:10F710002000FF002055FF004E49FF005453FF001A
:10F720002020FF002020FF002020FF002020FF00DD
:10F730002538FF007320FF000020FF00414DFF002F
:10F740005053FF005A45FF00524FFF002020FF009A
:10F750002020FF001B5BFF00307AFF002536FF00F2
:10F760006420FF000020FF005649FF004445FF00D1
:10F770004F4DFF004F44FF004520FF002020FF00B9
:10F780002025FF003873FF002000FF00204CFF0001
:10F790004F47FF005045FF005249FF004F44FF0014
:10F7A0002020FF00201BFF005B30FF007A25FF00B8
:10F7B0003664FF002000FF002048FF004F4DFF008F
:10F7C000454CFF004F43FF002020FF002020FF009A
:10F7D0002020FF002538FF007320FF000020FF00DD
:10F7E0004D41FF00484DFF00554CFF005420FF00E5
:10F7F000201BFF005B30FF007A20FF002537FF0051
:10F800002E35FF006620FF000020FF00414DFF0065
:10F81000504DFF00554CFF005420FF002020FF00FA
:10F820002020FF001B5BFF00307AFF002536FF0021
:10F830002E33FF006620FF000020FF005341FF0031
:10F840004645FF005A4FFF004E45FF002020FF00B5
:10F850002020FF001B5BFF00307AFF002536FF00F1
:10F860006420FF000020FF00564FFF004C54FF00B3
:10F87000314CFF004F57FF004152FF004E20FF0068
:10F880001B5BFF00307AFF002536FF007320FF006E
:10F890000020FF004452FF004157FF00484FFF0087
:10F8A0005249FF005A4FFF004E20FF001B5BFF0034
:10F8B000307AFF002536FF007320FF000020FF0094
:10F8C0004452FF004157FF002048FF005544FF000D
:10F8D0002020FF002020FF001B5BFF00307AFF008C
:10F8E0002536FF007320FF000020FF005341FF007A
:10F8F0005645FF002043FF004F4EFF004649FF00E2
:10F900004720FF001B5BFF00307AFF002536FF0019
:10F910007320FF00004EFF004F52FF000052FF0017
:10F920004556FF00004EFF004F52FF000052FF00FF
:10F930004556FF00004DFF004554FF005249FF00AF
:10F940004300FF00494DFF005045FF005249FF00B2
:10F95000414CFF000050FF00414CFF00004EFF00F3
:10F960005453FF004300FF005345FF005400FF00C5
:10F97000554EFF005345FF005400FF004F46FF0067
:10F980004600FF00204FFF004E00FF004F4EFF00DB
:10F990000020FF004F46FF004600FF004F4EFF00D3
:10F9A0000020FF004F46FF004600FF002A00FF0036
:10F9B000444FFF004E45FF000025FF003032FF009E
:10F9C0007800FF002450FF004D54FF004B25FF003E
:10F9D000732AFF002573FF000D0AFF000033FF00AC
:10F9E0003134FF002C30FF002C31FF002C30FF00A1
:10F9F0002C31FF002C30FF002C00FF003100FF00F5
:10FA00003000FF002C30FF002C30FF002C30FF00B6
:10FA10002C30FF002C30FF002C30FF002C30FF007A
:10FA20002C30FF002C30FF002C30FF002C30FF006A
:10FA3000003CFF004E55FF004C4CFF003E00FF0015
:10FA40001B5BFF002564FF006D00FF001B5BFF00D8
:10FA50003136FF003B25FF006476FF000047FF00C2
:10FA60005053FF002F4FFF005344FF002053FF006F
:10FA70005441FF005254FF005550FF002025FF0065
:10FA80006400FF001B5BFF003231FF003B30FF00D2
:10FA9000761BFF005B33FF00323BFF003176FF0037
:10FAA000001BFF005B31FF007A1BFF005B32FF0091
:10FAB0003B35FF004844FF007261FF00676FFF00A5
:10FAC0006E4FFF005344FF002056FF00342EFF000E
:10FAD0003866FF002033FF002F38FF002F32FF0071
:10FAE0003030FF003820FF002863FF002920FF008E
:10FAF0004461FF006E69FF00656CFF002057FF0046
:10FB00006565FF00001BFF005B33FF003B35FF0016
:10FB1000484DFF006F64FF006966FF006965FF00E4
:10FB20006420FF006279FF002054FF006F72FF0025
:10FB3000696EFF002053FF006567FF007374FF00CC
:10FB4000726FFF000057FF006169FF007469FF00DA
:10FB50006E67FF002066FF006F72FF002047FF0006
:10FB60005053FF002064FF006174FF006120FF001C
:10FB70002E2EFF002E00FF003030FF003000FF006F
:10FB80003330FF00312CFF003200FF003232FF0023
:10FB9000302CFF003230FF003000FF003031FF001A
:10FBA0003233FF003435FF003637FF003839FF00AD
:10FBB0006162FF006364FF006566FF006768FF0025
:10FBC000696AFF006B6CFF006D6EFF006F70FF00D5
:10FBD0007172FF007374FF007576FF007778FF0085
:10FBE000797AFF0000FFFF00C80EFF003031FF00F0
:10FBF0003233FF003435FF003637FF003839FF005D
:10FC00004142FF004344FF004546FF004748FF00D4
:10FC1000494AFF004B4CFF004D4EFF004F50FF0084
:10FC20005152FF005354FF005556FF005758FF0034
:10FC3000595AFF0000FFFF00F00EFF00000CFF000C
:10FC40000200FF00040CFF000200FF00080CFF0090
:10FC50000200FF000C0CFF000100FF000E0CFF0073
:10FC60000200FF00120CFF000200FF00160CFF0054
:10FC70000200FF001A0CFF000200FF001E0CFF0034
:10FC80000200FF00220CFF000200FF00260CFF0014
:10FC90000200FF002A0CFF000200FF002E0CFF00F4
:10FCA0000200FF00320CFF000200FF00360CFF00D4
:10FCB0000200FF003A0CFF000200FF003E0CFF00B4
:10FCC0000200FF00420CFF000200FF00460CFF0094
:10FCD0000200FF004A0CFF000200FF004E0CFF0074
:10FCE0000100FF00500CFF000100FF00520CFF005C
:10FCF0000100FF00540CFF000100FF00560CFF0044
:10FD00000100FF00580CFF000100FF005A0CFF002B
:10FD10000200FF005E0CFF000200FF00620CFF000B
:10FD20000100FF00640CFF000100FF00660CFF00F3
:10FD30000100FF00680CFF000100FF000000FF0051
:10FD40000000FF000000FF000000FF00FFFFFF00B9
:0200000401F009
:10000000F6FF0000F4FF00007F7A0000FFFFFF0012
:0C001000FFFFFF00FFFF0000FFFF0000EB
:00000001FF
